:020000040000FA
:107800005469616E59696E673130300000000000C4
:1078100054593230302E303830303030625F747925
:10782000424154333247313339474B3634464200B4
:1078300043414E5F5354440000000000000000002C
:1078400043414E5F43485F300000000000000000ED
:1078500043414E5F3530304B6270730000000000D2
:107860009407000014070000DF070000000000007C
:020000040000FA
:10800000D82F0020E9800000F1800000F3800000FC
:108010000000000000000000000000000000000060
:10802000000000000000000000000000FB800000D5
:108030000000000000000000FF8000003DCE0100B5
:108040004115010085150100B5150100E515010078
:10805000151601004516010075160100A516010050
:10806000D516010005170100391701004D17010051
:108070005D17010091170100A1170100B117010060
:10808000E51701002918010071180100B918010055
:108090000119010049190100591901008D19010048
:1080A000C1190100F1190100251A0100591A010036
:1080B000691A0100791A0100AD1A0100E11A0100E4
:1080C000EF72E8FF03B40148019001BD897F0020F1
:1080D0000448854600F02CFA0048004701100200D1
:1080E000C046C046D82F0020164880471648004793
:1080F000FEE7FEE7FEE7FEE7FEE7FEE7FEE7FEE758
:10810000FEE7FEE7FEE7FEE7FEE7FEE7FEE7FEE747
:10811000FEE7FEE7FEE7FEE7FEE7FEE7FEE7FEE737
:10812000FEE7FEE7FEE7FEE7FEE7FEE7FEE7FEE727
:10813000FEE7FEE7FEE7FEE7FEE7FEE7FEE7FEE717
:10814000FEE7000081D40100D180000030B50B466D
:10815000014600202022012409E00D46D5409D4221
:1081600005D31D469540491B2546954040191546A7
:10817000521E002DF1DC30BD70B5002425460028CC
:1081800001DA01244042002901DA01254942FFF7C2
:10819000DDFFAC4200D04042002C00D0494270BD0F
:1081A000F0B51FB40646002082B005464024019178
:1081B00000901BE0019922460F46304600F066F918
:1081C000049A059B801A994110D3104619462246FD
:1081D00000F04CF9361A8F41019722460120002108
:1081E000009F00F043F938184D4100902046641E6E
:1081F0000028DFDC019B00982946324607B0F0BD1D
:10820000F0B51FB486B0002000900190029006984F
:10821000069980B204900798090C020400141143D7
:1082200007900027089D099806913E463C4603901A
:108230000398A9B20204000C039004982D0C154376
:1082400048430021224600F011F9C719714110344A
:108250000E46402CECDB3846029A00F007F9009AF3
:10826000019B8018009059410298019110300290B2
:108270004028CCDB00980BB0F0BD03460B439B07B6
:1082800003D009E008C9121F08C0042AFAD203E08B
:108290000B780370401C491C521EF9D27047D2B2B1
:1082A00001E00270401C491EFBD270470022F6E735
:1082B00010B513460A4604461946FFF7F0FF20465C
:1082C00010BD30B504460020034600E05B1C93421D
:1082D00003D2E05CCD5C401BF8D030BD0321001D13
:1082E000401E037812021A43491EF9D51046704702
:1082F000034603220870000A491C521EFAD518468C
:108300007047024670B54A40D30FDB0740002DD0BE
:108310004A002AD0010E140E000212020919400A66
:10832000520A8418E50104465443000A120A2E0436
:108330005043A4194219200CC543AA18120C012558
:10834000AD03521C521912047F39240400D0521C70
:10835000104301D44000491EC2B20C06C0092018C7
:10836000401C4008802A02D003E0002070BD400875
:108370004000002900DA0020184370BD70B50246A5
:108380004A40D50F40004A00ED0740085208002837
:1083900014D0002A12D0C40DD30D41020120C00513
:1083A0005202490A520AE41A091812187D349142FD
:1083B00001D3641C00E04900002C01DA002070BDEC
:1083C0000023914201D3891A034340084900002841
:1083D000F7D100290AD0914202D10121C90705E055
:1083E000914201D2012101E00121C943E005C018F9
:1083F000401900F05CF870BD10B5002296231146BC
:1084000000F05DF810BDC20FD207400040080BD04D
:10841000C10D0723DB01C91840020905400A1143B9
:10842000C208400711437047002001467047000012
:1084300010B5002904DB0124E40740428C412146A9
:10844000002B04DB1C460123DB075242A341994267
:1084500000D1904210BD00000122D207002800DBAD
:10846000101A002900DB511A8842704710B5202AE3
:1084700004DB0146203A9140002010BD91402023AA
:108480009C1A0346E3401943904010BD10B5202AC2
:1084900004DB0846203AD040002110BD0B46D340F3
:1084A000D0402024A21A91400843194610BD00294B
:1084B00004DA401C490001D140084000704770B404
:1084C0000024050C05D11024000402D1002921D07C
:1084D0001124050E01D100020834050F01D100015D
:1084E000241D850F01D18000A41C002801DB400061
:1084F000641C002908D020252E1B0D46F540A14004
:1085000000D001212943084301061B1B000ADB1D83
:1085100002D5002070BC7047DB05181880180029B0
:10852000F8DA401C4900F5D170BC400840007047A3
:10853000064C0125064E05E0E36807CC2B430C3CB6
:1085400098471034B442F7D3FFF7C6FD0824020061
:108550003824020070B58C180578401C6B075B0F3F
:1085600001D10378401C2A1106D10278401C03E097
:1085700006780E70401C491C5B1EF9D12B0705D4F0
:108580000023521E0DD40B70491CFAE70378401CDF
:10859000CB1A921C03E01D780D70491C5B1C521E07
:1085A000F9D5A142D8D3002070BD70B507F080FA8C
:1085B0000524204618F0DEFC0025284607F06EFA58
:1085C000204618F0D7FC0126304607F045FA204631
:1085D00018F0D0FC284607F03FFA204618F0CAFCF5
:1085E000304607F05BFA204618F0C4FC70BDB0B509
:1085F00007F05EFA0524204618F0BCFC0125284649
:1086000007F04CFA204618F0B5FC284607F024FA8B
:10861000204618F0AFFC002007F01EFA204618F0A4
:10862000A9FCB0BDF0B581B007F030FA052018F014
:10863000A1FC08270026012007F00EFA0524204699
:1086400018F098FC204618F095FC07F015FA05463E
:10865000204618F08FFC002007F0FEF9204618F0A5
:1086600089FC76002E437F1E3806E4D1F0B201B0BB
:10867000F0BD70B50446002007F0EEF907F018FAD7
:10868000052018F077FC0826E0B2C00907F006FACA
:108690000525284618F06EFC012007F0DDF9284674
:1086A00018F068FC002007F0D7F9284618F062FCA3
:1086B000284618F05FFC6400761E3006E4D10520E1
:1086C00018F058FC012070BDF0B583B0019314463A
:1086D0000E460746012038430290032504E000F0CF
:1086E0008EF86D1E280631D000F067F83846FFF787
:1086F000C0FF00F0A7F80028F1D13046FFF7B9FF1E
:1087000000F0A0F80028EAD100F057F80298FFF72F
:10871000B0FF00F097F80028E1D1019802280BD3B0
:10872000451E0026FFF77EFF2070FFF73EFF641C0A
:10873000761CF0B28542F5DCFFF774FF2070FFF77E
:1087400056FF00F05CF8202003B0F0BD102003B00D
:10875000F0BDF0B583B01C46009201910290032554
:1087600004E000F04CF86D1E280623D000F025F838
:108770000298FFF77EFF00F065F80028F1D101981C
:10878000FFF777FF00F05EF80028EAD1002C0CD04C
:108790000026009F3878FFF76CFF00F053F80028A0
:1087A000DFD1761C7F1CA642F4D300F028F8082005
:1087B00003B0F0BD102003B0F0BDB0B507F078F9FC
:1087C0000524204618F0D6FB0125284607F044F979
:1087D000204618F0CFFB284607F060F9204618F035
:1087E000C9FB0025284607F059F9204618F0C2FBBE
:1087F000284607F031F9642018F0BCFBB0BDB0B5D5
:1088000007F056F90524204618F0B4FB0025284649
:1088100007F022F9204618F0ADFB284607F03EF994
:10882000204618F0A7FB0125284607F015F9204639
:1088300018F0A0FB284607F031F9642018F09AFBE5
:10884000B0BD0000B0B507F021F90524204618F0AE
:1088500091FB012007F000F9204618F08BFB0B4D2F
:1088600007F00AF9044607F0F1F8002C02D06D1E5B
:108870002804F5D10525284618F07CFB002007F0D8
:10888000EBF8284618F076FB2046B0BD33210000F7
:10889000034801780B2901D8491C01707047C04674
:1088A000C72B002070B584B0002503950295019573
:1088B000009507F0CBF80F20C6430E4C1036F1B2EE
:1088C000A0206A461023FFF744FF204618F052FB11
:1088D000204618F04FFB912EF0D3A020B0216A461D
:1088E0001023FFF736FF204618F044FB02480580AE
:1088F00004B070BD581B0000BA2B002070B50229CF
:1089000002D2EB24E0B270BD891EEB250022134693
:1089100005E0401C5B1CDDB2A94225460EDB047855
:108920006C40154604E034466E1C072D3546F0D2E7
:108930006608E407F7D09A246640F4E7E0B270BD19
:10894000F0B58BB00691044640780AA90870A27869
:1089500012021018E27823791B029A1812041018D8
:10896000020ECA70030C8B70050A4D7004900195BD
:1089700028180293C018039280182178C943401820
:108980006179A27912025118E279237A1B029A18AE
:10899000120452188018110A4018110C4018059240
:1089A000110E4018A17AE27A12025118227B099422
:1089B000637B1B029A18120452188018110A40187F
:1089C000110C401808900092100E079000263346B4
:1089D000304606E039409940C9B208435B1C082B79
:1089E0000ED001273A469A403446314602E0641CD4
:1089F000042CEFD00AAD2D5D2A42F8D0491CF6E7D1
:108A00000899079A8918C9B2099CA27B914212D190
:108A1000617A88420FD110212046FFF76FFF069A36
:108A20000399D17002999170019951700499117054
:108A3000059B009C19E010212046FFF75FFFE17BBA
:108A400088420BD1069A049911700399D17002994A
:108A5000917001995170059B009C06E00023069AD5
:108A6000D3709370537013701C4614721371210EDF
:108A7000D172210C9172210A5172190ED171190C07
:108A80009171190A51710BB0F0BDF0B58DB055223E
:108A90000270002747720B784370CA790592027200
:108AA0008A790492C2714A79039282710A79029298
:108AB0004271CA7A089242738A7A019202734E7A9C
:108AC000C6720C7A84720CAA13704D782D02EB18C2
:108AD0008D78C978090249190904CB18190E01715A
:108AE0001D0CC57009931B0A0B90837038460A91C0
:108AF000D170079595700693537031020919089A41
:108B00001202019BD218120451180891039909020C
:108B1000029A8918059A1202049BD218120451185D
:108B200005913D463A4605E02640AE4032436D1C75
:108B3000082D0ED001242146A9400346064602E036
:108B40005B1C042BF0D00CAFFF5C3942F8D0761CD4
:108B5000F6E70B9B5A720998069940180799401836
:108B60000A994018059A8018110A4018110C4018EB
:108B7000110E4018089A8018110A4018110C40185C
:108B8000110E40185638987310211846FFF7B6FE9C
:108B90000DB0F0BDF0B58FB00446FF20E070A070BE
:108BA00060700F20C04302900F302070704818F0A2
:108BB000E1F970490868632801D8642008606E4FA5
:108BC000002038806D4E0190308008E00B99814282
:108BD00022D338881030388080B2A1286DD206F0B8
:108BE00035FF3978A02003AA1023FFF76DFD3080F0
:108BF0002028EED103AD0BA92846FFF7A1FEE97BA3
:108C00008842E6D128785528E3D15D4801780029CB
:108C10000298DBD10846D9E73888A0284DD8C0B2E1
:108C20000021019105E006F011FF3988C8B2A129A1
:108C300043D2C1B2A02003AA1023FFF745FD308024
:108C4000398810313980202837D103AD07A928464B
:108C5000FFF776FEE97B8842E5D128785528E2D1F6
:108C6000474800780028029900D1014607988842B9
:108C7000D9D240490A68962151430B9A824208D9B9
:108C80000818904219D30BA90E222046FFF7F5FAD7
:108C9000C9E78918814210D307A90E222046FFF7A1
:108CA000ECFA0BA80A99818107980B9008980C9010
:108CB00009980D9038880190B5E72078617809020D
:108CC0000818A178E2781202511809040818401C0B
:108CD00024D1002001903880A020B02103AA1023C5
:108CE000FFF7F2FC3080202818D103AD0BA92846ED
:108CF000FFF726FEE97B884210D1287855280DD150
:108D00001F480078002800D102900B9802998842F1
:108D100004D20BA90E222046FFF7AFFA2078617823
:108D200009020818A178E2781202511809040818FB
:108D3000401C0CD10020E072A07260722072E071C1
:108D4000A07160712071E070A07060702070019857
:108D500038802078617809020818A178E278120238
:108D60005118090408180749086030880FB0F0BD91
:108D700070110100B42B0020BA2B0020B02B002072
:108D8000B32B0020C02B0020F0B581B00091064627
:108D9000214800250570002A2ED01446C036631BDA
:108DA00071190F2008401022101A834200D3034685
:108DB0001A480278102A01D0042A1AD1C809FE27BD
:108DC00007405F2F13D80127B8436038C0B29E32E6
:108DD00082420CD3009A5219C9B2DFB23B46FFF768
:108DE00073FC0F490880ED19A542D8D304E0082090
:108DF00000E004200A49088009480188002004296D
:108E000002D0082900D0012003490870411E884182
:108E1000400001B0F0BDC046C62B0020B22B0020A0
:108E2000C42B00200A4A012313700A4A10700A4A10
:108E300011600A4A00211160042801D1052189012D
:108E4000102801D11D208101054801807047C046CE
:108E5000B32B0020B22B0020B42B0020C02B00200D
:108E6000B82B0020F0B587B09B4D00262E709B4B91
:108E70001B688B4224D19B4C2188202925D102904C
:108E800000920196984C00272760984D984E2878BC
:108E9000062809D806F0DAFD2068401C2060B042A0
:108EA000F5D38F48042101802F70924C2088010750
:108EB000029B34D08A4820210180874D019E0BE01F
:108EC000012040028649088006E003A8FFF762FE01
:108ED0002080834880210180814800883F2807DD69
:108EE000894988420BDC402812D0802810D010E03D
:108EF00004280DD008280AD0202809D009E0012133
:108F00004A02904204D0C902884201D001E0012601
:108F10002E702878411E8841400007B0F0BDA1287E
:108F2000019E00D32780009A012A6B4D1ED1187B29
:108F3000012856D1DF719F715F711F711F73587BBC
:108F4000012804D1DF729F725F721F725F7303AFDB
:108F500038461946FFF799FDF8732088002846D057
:108F60001038C1B2A02003AA102344E0002AB3D1D4
:108F7000614801780029AFD0027018785978090249
:108F800008189978DA7812025118090408185B4910
:108F90000978002901D00F21C943884233D22746DE
:108FA00003AC20461946FFF770FDE0733978A02026
:108FB00010232246FFF7CDFB029A49490880082872
:108FC0008AD1388810303880107851780902081812
:108FD0009178D2781202511809040818484908609B
:108FE0007AE7597B012911D10128A3D0A7E7A02056
:108FF00003AA10230146FFF7ACFB394908803E481D
:109000000099017068E70120C0025BE73D480078E5
:10901000012812D103AC20461946FFF736FDE07354
:10902000A020B02110232246FFF793FB2C49088093
:109030000828E4D133480770E1E718785978090225
:1090400008189978DA7812025118090408182C497E
:109050000968224A12685118884203D220484021E8
:109060000180CCE725490978002901D00F21C943A7
:1090700088422DD203AF384619461C46FFF705FD3E
:10908000F8731C480178A02010233A46FFF761FBD3
:10909000134908800828B2D1164908881030088082
:1090A0002078617809020818A178E2781202511834
:1090B000090408181249086008490A681521514333
:1090C000FFF744F800299AD101200E49087096E76D
:1090D0000120C00291E7C046CC2B0020B42B002019
:1090E000CA2B0020B02B0020D02B0020C72B002043
:1090F000818D5B00BA2B0020BC2B0020B32B0020FD
:10910000C02B0020C82B0020FF010000F0B585B067
:1091100006462E4C0025257010182D4B1B889842B2
:1091200035D20192029103952A4D002004902860C7
:10913000294C2A4F2078052809D806F087FC286892
:10914000401C2860B842F5D32548042101800498CA
:109150002070244801780122102901D0042918D157
:10916000C036F309603B1002DCB26409052C174CD1
:10917000039D11D39343DAB29E3191420CD3F1B2E5
:109180000198C3B21046029AFFF7E3FA04E02020E8
:1091900002E090020D4C039D114908801F2809DD53
:1091A00020280CD001210A02904208D0890288426E
:1091B00005D005E0042802D0082801D1012525703A
:1091C0002078411E8841400005B0F0BDCC2B002026
:1091D000B82B0020D02B0020C72B0020818D5B00F6
:1091E000CA2B0020B22B0020F0B585B00446002029
:1091F0000190042C6FD20CF083FA002801D10CF0FE
:10920000FFFA0020009000BF0098401C00900CF076
:1092100077FA03900398002803D0484900988842C1
:10922000F2D30398002856D1042145480CF04AFA9D
:109230004448454908802101444A515C4900404A5C
:10924000505A41490A880121090300F059F9029056
:109250000120049020013D4940184078002801D1A8
:1092600000264BE02001394940184078012802D1FE
:109270003548068842E020013449401840780228E9
:109280002AD12001401805792901304A515C490052
:109290002B4A505A2C490A880121090300F030F961
:1092A000064628012A4943182801284940180289FE
:1092B000280140180021C7683046B84706462801F3
:1092C000224BC018C2882801C0188178304600F0AF
:1092D0008BF8064612E02DE020011C49401840782A
:1092E000032804D0200140184078132804D120011D
:1092F00016494018868801E0002004900498002850
:1093000018D0200112494318200110494018028941
:10931000200140183146C7680298B84701902001E3
:109320000A4BC018C2882001C0188178019800F04B
:109330005BF80190019805B0F0BD000050C300003B
:10934000180100208813000010010020A41A020058
:10935000E41A0200F8B507460C46154600200090B6
:10936000002C00D1F8BD01211C4801751C48007873
:1093700088431B490870084680780821084318492B
:10938000887000208871084600780121084314493C
:10939000087008460772002617E0114800788021FF
:1093A00008430F49087000BF0E48007D0028FBD01D
:1093B00000200C4908750A48C0892880AD1C08485F
:1093C000C189009808180090761CA642E5D3214672
:1093D0000098FEF7BBFE80B2C4E700004061004089
:1093E000005004404060004010B50346012908D1F8
:1093F000094CA41A9C4202D99C18A0B20BE0064862
:1094000009E0022906D1934202DD9C1AA0B202E0D3
:10941000002000E0184610BDFFFF000010B5044614
:109420000121202002F0F4F80020324908700121C7
:1094300031480175002031490875152017F01CFCD2
:109440002C488078E17808432A498870084680785B
:1094500021780843274988702078802806D108465B
:109460000079E17949000843224908712148807850
:10947000E17A08431F498870A078002803D1084684
:10948000007908710FE0A078012806D11948007909
:10949000602108431749087105E0164800798021CA
:1094A0000843144908711348807921790843114908
:1094B000887108468079617908430E498871207A5D
:1094C000C872607A88720846007838218843094952
:1094D0000870084600786178C9000843054908709B
:1094E000A07A0873084600780121084301490870F2
:1094F00010BD00000050044040610040406000404A
:10950000F8B504460E461746002E01D100250FE09F
:10951000A64201DC3D460BE00094009C20467843C7
:10952000009031460098FEF711FE0090009885B239
:109530002846F8BD0146042904D28A00024BD218FD
:10954000508800E0002070474C2300200146042989
:1095500003D28A00024B985C00E0002070470000B4
:109560004C230020FFB587B004460898844203DAF4
:109570000A988068002802D12448019042E00898A7
:10958000001B82B20292002625460A9880680021BC
:109590002F463A463346049605910690FEF730FE74
:1095A00005460E46002328463146029AFEF7F8FD8E
:1095B00005460E46304600210A46494050400143C8
:1095C00002D0124801901DE003950A98C068039DDF
:1095D000A84202D30020019014E00A98C1680398C1
:1095E000401A039009990398FEF7B0FD0390039881
:1095F000000C0004002802D00448019002E0039807
:1096000080B2019001980BB0F0BD0000FFFF000098
:1096100010B5084800788021884306490870012168
:1096200005480175002005490875152017F024FB31
:1096300010BD000000500440406100404060004008
:10964000F8B505460E4614461F4621462846FEF745
:1096500093FD80B2F8BD0000FFB587B006460A98BA
:109660004068002801D1029035E00A9801684068FE
:1096700008180390002534460021274603980695D4
:109680000491059038462946049B059AFEF7B8FDDB
:1096900004460D460A984068024600230190204681
:1096A0002946FEF77DFD04460D4600232046294647
:1096B000099AFEF775FD04460D46284607492140E4
:1096C000002359405840014303D00448C04302904E
:1096D00001E0A0B2029002980BB0F0BD0000FFFFC5
:1096E00010B5FE4800688079030017F0ABFA070553
:1096F0009ED8F5F4F3F2F100F848006840790300D1
:1097000017F0A0FA0805138A2A8A468A638A13F09A
:10971000CDFA0020F1490968C873F0480068407923
:10972000401CEE49096848717DE0ED494969EB4A02
:109730001268D27A885C13F031FBE84800684079FF
:10974000401CE64909684871E44800684079401CBB
:10975000E2490968487166E00AF030F9002810D142
:1097600013F01CFBDD4800684079401CDB490968A8
:109770004871DA4800684079401CD8490968487146
:1097800005E013F0BDFA0020D449096848714AE0A9
:109790000AF014F9002811D1112013F0FFFACF4874
:1097A00000684079401CCD4909684871CB48006881
:1097B0004079401CC9490968487105E013F0A0FAD6
:1097C0000020C649096848712DE00AF0F7F8002822
:1097D0001BD1C2480068C07A401CC0490968C872E1
:1097E000BE480068C07ABE49097888420DDB002077
:1097F000BA490968C872B94909684862B748006837
:109800008079401CB5490968887113F079FA002005
:10981000B2490968487106E013F072FA0020AF49B6
:109820000968487100BF00BF32E3AC480068407C63
:10983000002817D0AA48C068002803D0A848C168EB
:10984000192088470020A54909684862A348006894
:109850008079401CA1490968887100209F490968E6
:1098600048711BE09D480068406A282807D29B4841
:109870000068406A401C9949096848620EE000206F
:10988000964909684862954800688079401C934968
:10989000096888710020914909684871F8E28F4889
:1098A00000684079030017F0CDF9080518A42FA42B
:1098B0004CA480A413F0FAF9002088490968C87301
:1098C000864800684079401C84490968487197E0DF
:1098D000D4E2C7E230E25DE194E0814949697F4A20
:1098E0001268D27A885C13F059FA7C480068407993
:1098F000401C7A4909684871784800684079401CE2
:109900007649096848717BE00AF058F8002811D1BF
:10991000012013F043FA714800684079401C6F49F8
:10992000096848716D4800684079401C6B490968B6
:10993000487105E013F0E4F90020684909684871AE
:109940005EE00AF03BF8002828D164490968C97A2A
:1099500024225143634A12688918604A1268D27BF4
:10996000885C13F01BFA5D480068C07B401C5B49B3
:109970000968C87359480068C07B242814D3574825
:1099800000684079401C554909684871534800688F
:109990004079401C51490968487105E013F0B0F95D
:1099A00000204E49096848712AE00AF007F80028AB
:1099B00018D14A480068C07A401C48490968C872F2
:1099C00046480068C07A4649097888420ADB002088
:1099D00042490968C872414800688079401C3F4983
:1099E0000968887113F08CF900203C4909684871B6
:1099F00006E013F085F9002038490968487100BF76
:109A000000BF45E2354800684079030017F01AF9B5
:109A10000A0614B92BB948B978B995B913F046F9C3
:109A200000202E490968C8732C4800684079401C02
:109A30002A4909684871ABE029494969274A1268EF
:109A4000D27A885C13F0AAF9244800684079401C57
:109A5000224909684871214800684079401C1F4923
:109A60000968487194E009F0A9FF002811D14A2043
:109A700013F094F9194800684079401C17490968A7
:109A80004871164800684079401C144909684871BB
:109A900005E013F035F9002010490968487177E0B6
:109AA00009F08CFF002824D1FF2013F077F90B4830
:109AB0000068C07B401C09490968C87307480068F2
:109AC000C07B24281BD3054800684079401C03490B
:109AD0000968487101480068407905E000080020E5
:109AE000982B0020FC070020401CEA4909684871B7
:109AF00005E013F005F90020E6490968487147E0E0
:109B000009F05CFF002811D1FF2013F047F9E1486C
:109B100000684079401CDF4909684871DD480068E9
:109B20004079401CDB490968487105E013F0E8F80A
:109B30000020D849096848712AE009F03FFF002851
:109B400018D1D4480068C07A401CD2490968C8724C
:109B5000D0480068C07AD049097888420ADB0020E2
:109B6000CC490968C872CB4800688079401CC94953
:109B70000968887113F0C4F80020C6490968487163
:109B800006E013F0BDF80020C2490968487100BF23
:109B900000BF7DE1BF4800684079030017F052F82C
:109BA0000C0715C32CC349C366C382C39FC313F0FC
:109BB0007DF80020B7490968C873B6480068407945
:109BC000401CB44909684871B4E0B3494969B14AD5
:109BD0001268D27A885C13F0E1F8AE4800684079E8
:109BE000401CAC4909684871AA4800684079401C8B
:109BF000A849096848719DE009F0E0FE002811D1EC
:109C0000772013F0CBF8A34800684079401CA149A5
:109C1000096848719F4800684079401C9D4909685F
:109C2000487105E013F06CF800209A490968487102
:109C300080E009F0C3FE002811D10C2013F0AEF82B
:109C4000944800684079401C9249096848719148DD
:109C500000684079401C8F490968487105E013F09D
:109C60004FF800208B490968487163E009F0A6FEAF
:109C7000002810D113F092F8864800684079401C03
:109C8000844909684871834800684079401C8149CB
:109C90000968487105E013F033F800207D49096830
:109CA000487147E009F08AFE002811D1132013F013
:109CB00075F8784800684079401C76490968487111
:109CC000744800684079401C72490968487105E091
:109CD00013F016F800206F49096848712AE009F06E
:109CE0006DFE002818D16B480068C07A401C694995
:109CF0000968C87267480068C07A6749097888426D
:109D00000ADB002063490968C872624800688079EC
:109D1000401C60490968887112F0F2FF00205D491B
:109D20000968487106E012F0EBFF00205949096804
:109D3000487100BF00BFABE056480068407903009F
:109D400016F080FF080513872A874787638712F07C
:109D5000ADFF00204F490968C8734E48006840793C
:109D6000401C4C49096848717AE04B494969494AA5
:109D70001268D27A885C13F011F84648006840797E
:109D8000401C444909684871424800684079401CB9
:109D900040490968487163E009F010FE002811D1BC
:109DA000492012F0FBFF3B4800684079401C3949CC
:109DB00009684871374800684079401C354909688E
:109DC000487105E012F09CFF002032490968487193
:109DD00046E009F0F3FD002810D112F0DFFF2D4816
:109DE00000684079401C2B4909684871294800687F
:109DF0004079401C27490968487105E012F080FF4E
:109E000000202449096848712AE009F0D7FD00289C
:109E100018D120480068C07A401C1E490968C872E1
:109E20001C480068C07A1C49097888420ADB002077
:109E300018490968C872174800688079401C15499C
:109E40000968887112F05CFF0020124909684871A6
:109E500006E012F055FF00200E490968487100BF66
:109E600000BF15E000200B4909688871094909689D
:109E70004871062007490968C87009E012F040FFE0
:109E8000002004490968487102490968887100BFC7
:109E900000BF10BD00080020982B002010B56A48B4
:109EA00000684079030016F0CDFE090610C627C6EB
:109EB00044C6608EC60012F0F9FE6348006840791F
:109EC000401C614909684871BCE0604949695E4AC3
:109ED0001268D27A885C12F061FF5B4800684079B2
:109EE000401C594909684871574800684079401C2E
:109EF000554909684871A5E009F060FD002811D1B5
:109F00007F2012F04BFF504800684079401C4E49BA
:109F1000096848714C4800684079401C4A49096802
:109F2000487105E012F0ECFE0020474909684871CD
:109F300088E009F043FD002810D112F02FFF4248BD
:109F400000684079401C4049096848713E480068F3
:109F50004079401C3C490968487105E012F0D0FE88
:109F600000203949096848716CE009F027FD002894
:109F700022D135480068C07A401C33490968C8724C
:109F800031480068C07A3149097888420FDB0020E7
:109F90002D490968C8722C4800684079401C2A493C
:109FA00009684871002028490968486208E00020D3
:109FB00025490968487103E0002023490968487170
:109FC00012F09EFE3EE020480068407C002816D03B
:109FD0001E48C068002803D01C48C1681920884763
:109FE00000201949096848621749096848711649EB
:109FF00009688871052014490968C8701AE0124878
:10A000000068406A282807D20F480068406A401C50
:10A010000D49096848620DE000200B490968486253
:10A020000949096848710849096888710520064985
:10A030000968C87006E012F063FE00200249096852
:10A04000487100BF00BF10BD00080020982B002001
:10A0500010B50024F7480068807A01287ED1F548C1
:10A060000068C07900287AD0F2480068807900281A
:10A0700004D0012874D0022873D191E1ED48006822
:10A08000007B24286ED2EB480068C07901287AD181
:10A09000002475E0E7480068C07A24214843E64977
:10A0A00009684018E3490968097B415CE148006898
:10A0B000C07A24225043E14A12688018DD4A1268AF
:10A0C000127B805C814229D0DA480068C07A242162
:10A0D0004843DA4909684018D6490968097B415C58
:10A0E000D4480068C07A24225043D34A12688018AA
:10A0F000D04A1268127B8154CE480068407B2428E5
:10A1000005D3CC480068007BCA4909684873C94830
:10A110000068007BC7490968887308E0C548006883
:10A12000407B242803D20120C24909688871C148B4
:10A130000068007B401CBF4909680873BD4800687F
:10A14000007B242808D3BB480068407B242803D226
:10A150000120B84909688871B64805E0D3E1CDE12E
:10A1600069E0BAE138E00EE00068007B242804D200
:10A17000B04800688079012800D103E0601CC4B2B7
:10A18000242C87D356E0002413E0AA480068C07A44
:10A1900024214843A94909684018015DA548006881
:10A1A000C07A24225043A44A126880180155601CCA
:10A1B000C4B2242CE9D300209E49096848732320A7
:10A1C0009C490968887301209A490968887124208C
:10A1D0009849096808732DE00020964909680873BA
:10A1E00094480068C07A401C92490968C872914836
:10A1F0000068C07A92490978884217DB8D48006868
:10A20000007C012804D102208A490968887106E08F
:10A21000002088490968887186490968C87100204A
:10A2200084490968C8728349096808740020814913
:10A230000968487161E17F4800684079030016F0C1
:10A2400001FD080513A62AA651A68EA6012079496C
:10A250000968087412F02AFD764800684079401CAD
:10A2600074490968487199E075494969714A1268E9
:10A27000D27A885C12F092FD6E4800684079401CEA
:10A280006C49096848716B4800684079401C69490D
:10A290000968487182E009F091FB00281BD16549EB
:10A2A0000968497B491CC8B212F078FD6148006812
:10A2B000407B60490968C8735E4800684079401C6B
:10A2C0005C49096848715B4800684079401C5949FD
:10A2D0000968487105E012F013FD0020554909682E
:10A2E00048715BE009F06AFB00282BD151490968ED
:10A2F000C97A24225143504A126889184D4A12687B
:10A30000D27B885C12F04AFD4A480068C07B401C42
:10A3100048490968C87347480068C07B45490968CF
:10A32000897B88421ADD434800684079401C4149D6
:10A33000096848713F4800684079401C3D490968F8
:10A3400048710BE012F0DCFC3A480068407B394968
:10A350000968C87300203749096848711EE009F090
:10A360002DFB00280CD1334909688871242031491C
:10A370000968C8732F49096848732E4909688873AA
:10A3800012F0BEFC00202B490968487106E012F06B
:10A39000B7FC002027490968487100BF00BFACE046
:10A3A000244800684079030016F04CFC08050F8E25
:10A3B000268E4C8E688E12F079FC1E48006840791B
:10A3C000401C1C490968487185E01D494969194AC2
:10A3D0001268D27A885C12F0E1FC16480068407975
:10A3E000401C144909684871124800684079401CB3
:10A3F0001049096848716EE009F0E0FA002811D1AF
:10A40000492012F0CBFC0B4800684079401C0949F8
:10A4100009684871074800684079401C0549096887
:10A42000487105E012F06CFC00200249096848718F
:10A4300051E0000000080020FC070020F807002081
:10A44000982B002009F0BAFA002810D112F0A6FCCF
:10A450009C4800684079401C9A49096848719948AD
:10A4600000684079401C97490968487105E012F07E
:10A4700047FC00209349096848712CE009F09EFAD6
:10A4800000281AD18F480068C07A401C8D4909689D
:10A49000C8728C480068C07A8B49097888420CDB06
:10A4A000002088490968C872864909688871854909
:10A4B0000968487183490968C87112F021FC0020BD
:10A4C00080490968487106E012F01AFC00207D49B5
:10A4D0000968487100BF00BF0FE012F011FC0020B6
:10A4E0007849096848717749096888717549096828
:10A4F000087374490968C87200BFE2E0002071491E
:10A5000009688872DDE06F480068807A0228F4D11B
:10A510006C480068007A002879D06A480068407961
:10A52000030016F08FFB0B0711BB25BB41545EBB2C
:10A530007590BB0012F0BAFB624800684079401C7D
:10A54000604909684871B7E05F494969087812F0C5
:10A5500025FC5C4800684079401C5A4909684871EC
:10A56000584800684079401C564909684871A3E082
:10A5700009F024FA002810D112F010FC51480068AC
:10A580004079401C4F49096848714E48006840793D
:10A59000401C4C490968487105E012F0B1FB0020ED
:10A5A00048490968487187E009F008FA002807D18E
:10A5B000444800684079401C42490968487103E0FA
:10A5C000002040490968487112F09AFB74E012F0CB
:10A5D0006DFB3C4800684079401C3A490968487165
:10A5E0006AE0394949690978491CC8B212F0D6FBBA
:10A5F000344800684079401C324909684871314844
:10A6000000684079401C2F490968487154E054E0C3
:10A6100009F0D4F900280FD112F01AFB2949096872
:10A620008870012012F08EFB264800684079401C9B
:10A6300024490968487105E012F062FB00202149B5
:10A640000968487138E01F480068807811280CD1EB
:10A6500000201C4909680872AA201A4909688870F4
:10A66000002018490968487011E0164800684078D1
:10A67000401C144909684870124800684078032853
:10A6800005D309F03FFA00200E490968487012F01E
:10A6900037FB00200B49096848710DE012F030FBD0
:10A6A0000020084909684871064909684870AA20CD
:10A6B00004490968887000BF03E000200149096867
:10A6C000887210BD00080020982B002010B50246AB
:10A6D0009000074BC018405C002802D00320C04304
:10A6E00010BD01209300024C1B1958540020F7E7BD
:10A6F0001427002070B5002508E06D1C184885421D
:10A7000002D20BF0A9F801E0002503E00AF0F8FFFF
:10A710000028F2D100BF002406E01248015D0020AD
:10A720000AF0FCFF601CC4B2042CF6D3002408E03D
:10A730000020A1000C4A5054A10089184880601CD8
:10A74000C4B2042CF4D301200849087000204870DA
:10A75000052088700020C87005480649088070BD33
:10A7600050C30000A01A02004C2300201401002056
:10A770008813000010010020F8B58D480078030010
:10A7800016F060FA060405163D5EFDFC0EE10BF0C6
:10A7900037F800208649C87048700846807800283D
:10A7A00002D10320087002E0022081490870FDE018
:10A7B0007F488078002804D07D488078401E7C49FE
:10A7C00088700AF09DFF00280BD10BF019F80020CB
:10A7D0007749C8700846807800280FD10320087098
:10A7E0000CE07348C078401C7149C8700846C078B6
:10A7F000052803D3052008700BF02EF8D6E00AF0E8
:10A800007FFF00280ED104216A480AF05BFF002078
:10A810006749C870487068486849088004206449DE
:10A8200008700CE06248C078401C6149C870084656
:10A83000C078052803D3052008700BF00DF8B5E0AB
:10A840005B49497809015E4A515C4900594A505AAE
:10A850005A490A8801210903FEF752FE009001259A
:10A86000534840780001564940184078002801D1EB
:10A8700000243CE04E48407800015149401840789F
:10A88000012802D14D48048831E049484078000150
:10A890004B4940184078022812D1454949780901AE
:10A8A000474A89180879FEF745FE04464049497829
:10A8B0000901434A89180879FEF748FE054616E063
:10A8C0003B48407800013E4940184078032806D0B4
:10A8D00037484078000140184078132806D13448A2
:10A8E0004078000136494018848800E00025002D9A
:10A8F0002FD02F4840780001324943182C48407827
:10A9000000012F4940180289294840780001401869
:10A910002146C7680098B847064625484078000198
:10A92000274BC018C288224840780001C01881789F
:10A930003046FEF759FD06461D4840788000224902
:10A940004018468001201A49497889001E4A50540F
:10A950000AE000201649497889001B4A8918488076
:10A96000134949788900505411484078401C1049D7
:10A97000487008464078042809D301E013E007E056
:10A980000AF03EFF00200A494870032008700DE0DD
:10A990000AF0B6FE002803D101200549087001E045
:10A9A0000AF05AFF02E0FFF7A5FE00BF00BFF8BDA6
:10A9B000140100201801002088130000100100205D
:10A9C000A41A0200E41A02004C23002010B50AF079
:10A9D00061FE002405E00020A100074A5054601CDD
:10A9E000C4B2042CF7D300200449087005208870F5
:10A9F00003480449088010BD4C23002014010020A6
:10AA0000881300001001002010B50346002000F05C
:10AA1000D7F8002000F03AF9002000F0AFF800204D
:10AA200000F012F9002000F087F8002000F0EAF8AA
:10AA300000BF012000F0A2F8012000F005F9002479
:10AA400021E0002000F09AF8002000F0FDF88020BE
:10AA50001840002806D0012000F0B2F8012000F0D4
:10AA600015F905E0002000F0ABF8002000F00EF929
:10AA700000BF012000F082F8012000F0E5F8580640
:10AA8000030E601CC4B2082CDBDB012000F054F87C
:10AA9000012000F0B7F810BD30B503460C46012088
:10AAA00000F08EF8012000F0F1F8002000F066F8C8
:10AAB000002000F0C9F8002000F03EF8002000F06F
:10AAC000A1F800BF012000F059F8012000F0BCF807
:10AAD000002528E0002000F051F8002000F0B4F834
:10AAE00080201840002803D0012000F069F802E01F
:10AAF000002000F065F880202040002803D00120CD
:10AB000000F0C4F802E0002000F0C0F800BF01200F
:10AB100000F034F8012000F097F85806030E6006A4
:10AB2000040E681CC5B2082DD4DB012000F004F827
:10AB3000012000F067F830BD00B5014600290CD0B7
:10AB40000C480078082290430A4A107008200A4AEC
:10AB50001070052009F0EEFE0BE006480078082290
:10AB60009043044A10700820034A1074052009F02D
:10AB7000E1FE00BD200304408000044000B5014612
:10AB800000290CD00C480078102290430A4A10701B
:10AB900010200A4A1070052009F0CCFE0BE0064890
:10ABA000007810229043044A10701020034A107459
:10ABB000052009F0BFFE00BD2003044080000440D2
:10ABC00000B5014600290CD00C48007804229043BF
:10ABD0000A4A107004200A4A1070052009F0AAFEE3
:10ABE0000BE00648007804229043044A10700420C9
:10ABF000034A1074052009F09DFE00BD20030440A7
:10AC00008000044000B5014600290CD00C48C079F2
:10AC1000022290430A4AD07102200A4AD0710520CC
:10AC200009F088FE0BE00648C07902229043044AEE
:10AC3000D0710220034AD075052009F07BFE00BDCB
:10AC4000200304408000044000B5014600290CD0D8
:10AC50000C48C079400840000A4AD07101200A4AD5
:10AC6000D071052009F066FE0BE00648C079400867
:10AC70004000044AD0710120034AD075052009F034
:10AC800059FE00BD200304408000044000B5014689
:10AC900000290CD00C48C079042290430A4AD07194
:10ACA00004200A4AD071052009F044FE0BE0064852
:10ACB000C07904229043044AD0710420034AD0751D
:10ACC000052009F037FE00BD200304408000044049
:10ACD00010B53221464805F0E9FDF920FFF794FE52
:10ACE0003221444805F0E2FD8820FFF78DFE9020D8
:10ACF000FFF78AFE9820FFF787FE08210846FFF736
:10AD0000CBFEE820FFF780FE12210846FFF7C4FEC5
:10AD1000A020FFF779FE70210846FFF7BDFEA820AE
:10AD2000FFF772FE70210846FFF7B6FEB020FFF76E
:10AD30006BFE70210846FFF7AFFEB820FFF764FEF8
:10AD400000210846FFF7A8FEC020FFF75DFE0021A6
:10AD50000846FFF7A1FEC820FFF756FE002108466F
:10AD6000FFF79AFED020FFF74FFE2F210846FFF78E
:10AD700093FED820FFF748FE2F210846FFF78CFEF0
:10AD8000E020FFF741FE2F210846FFF785FE402017
:10AD9000FFF73AFE00210846FFF77EFE0A20FFF784
:10ADA00033FE002405E000210846FFF775FE601C15
:10ADB000C4B25A2CF7DB00240AE000200E490855E3
:10ADC0000E4908550E4908550E490855601CC4B275
:10ADD0005A2CF2DB8120FFF717FE00200A49086099
:10ADE0000A4908708870C8700871487010BD00006A
:10ADF000C0D40100204E000078200020D220002086
:10AE00002C21002086210020F0000020E8000020F6
:10AE100000B58020FFF7F8FD00BD00000B4800786A
:10AE200000280CD10A480068582805D8084800684E
:10AE3000801C0749086002E00020054908600120E5
:10AE4000024908700020487070470000E8000020A8
:10AE5000F000002000B54E480078002879D04C481A
:10AE60008078030015F0EEFE060450576067768B7D
:10AE7000474800794749085C45490979464A515C89
:10AE8000884216D1424800794449085C4049097912
:10AE9000434A515C88420CD13D48007941490968D8
:10AEA000884222D33A4801793E480068801C81429A
:10AEB0001BD8374800793749085C35490979364A43
:10AEC0005054334800793549085C31490979344A8E
:10AED00050542F48C078002803D004202C49887093
:10AEE00011E001202A4988700DE000202849C8702F
:10AEF00008460079401C0871084600795A2802DB90
:10AF000000200871087041E04020FFF77DFD02201D
:10AF10001F4988703AE01E4A11791079FFF7BCFD8D
:10AF200003201B49887031E00A20FFF76DFD0420E3
:10AF3000174988702AE0164A1279194B995C144A0D
:10AF40001279154B985CFFF7A7FD05201049887012
:10AF50001CE01CE00E480079401C0D4908710846B1
:10AF600000795A2804DB002008710870C87002E0DC
:10AF700001200749C87000200549887006E00020BC
:10AF8000034908708870C870087100BF00BF00BD19
:10AF9000E800002078200020D22000202C21002072
:10AFA00086210020F000002010B501F05FFE01288E
:10AFB0001ED101F049FE1149884212D3072009F041
:10AFC0002FFB002806D04B22D2000021012013F0D5
:10AFD000F3FF12E07D22D2000021012013F0ECFFEC
:10AFE0000BE07D22D2000021012013F0E5FF04E0F8
:10AFF00000221146012013F0DFFF10BDD60B000028
:10B00000002003490872487088704860704700004B
:10B01000240A002058221152704710B5044601211D
:10B02000022000F0F5FA0021022000F0F1FA10BD34
:10B03000014600205322525C10231A40002A08D0F7
:10B040005322525C0C231A409210032A18D1032079
:10B0500016E05422525A0123DB031A40002A0ED074
:10B060005322525C0C231A409210032A05D053221B
:10B07000525C9207920F032A01D1022000E00120C6
:10B0800070470246002058239B5A0B40002B01D0EA
:10B09000012000E00020704710B5002A0AD0562396
:10B0A0001B5A0C0223435624235256231B5A8B430C
:10B0B000235209E056231B5A0C02A3435624235261
:10B0C00056231B5A0B43235210BD0000F8B504460B
:10B0D0000D46012700263448844203D10121022075
:10B0E00000F096FA2878401EA0702088FF210131D8
:10B0F000084320802088400840002080A878401E17
:10B10000C1B25A20015568790007000CE97909029B
:10B110000843A97908435C210853288981B240205B
:10B120000153A868C000C10C42200153A88981B214
:10B1300044200153E868C000C10C46200153288A0E
:10B1400081B2482001532869C000C10C4A20015334
:10B15000A88A81B24C2001536869C000C10C4E20FE
:10B1600001535020005B29790902084350210853FC
:10B170005020005B297988435021085300E0761C59
:10B180005020005B4007400F2979884202D00748D1
:10B190008642F4D15020005B4007400F2979884255
:10B1A00000D000273846F8BD00540440FFFF0000DF
:10B1B00030B5034600201C898C4209DD082A05D2DF
:10B1C00018244C431D682C19A05C02E0002000E00C
:10B1D000002030BD10B5024613898B4205DD1823CF
:10B1E0004B431468E318987C00E0002010BD000079
:10B1F0000146144AC889C007C00F00280AD00120A0
:10B20000C88100E0521EC889C007C00F002801D0C5
:10B21000002AF7D1C889C007C00F00280FD102202B
:10B22000C8810420C881487A400840004872487AA2
:10B23000382398434872002048720120704700204C
:10B24000FCE70000FFFF00000246507A012318438C
:10B250005072507A0B78DB0018435072087A01283C
:10B2600008D1888850814868000C0123DB0318430B
:10B27000908108E0087A002805D150814868800054
:10B28000204B18409081487A012804D1507A4023FD
:10B290001843507206E0487A002803D1507A4023C0
:10B2A00098435072087D002804D0507A80231843B8
:10B2B000507203E0507A8023984350720878002837
:10B2C00011D1C87A1072087B1070487B5070887B4F
:10B2D0009070CB7BD370087C10714B7C5371887C51
:10B2E0009071CB7CD371887A002803D00120C002F2
:10B2F000D08101E00820D081FF200130D0810120E1
:10B3000070470000FC1F0000002904D0427A80230F
:10B310001A43427203E0427A80239A434272704792
:10B3200030B5024600200F4B5024A45A0D022C4386
:10B330005025AC525024A45A8C43AC5200E05B1E02
:10B340005024A45A6407640F8C4201D0002BF6D11C
:10B350005024A45A6407640F002C01D0002000E0A0
:10B36000012030BDFFFF0000827A80231A40802A2E
:10B3700000D0817270470000F0B587B006460C46D9
:10B380000027002006906020875BF807C00F002888
:10B3900002D001216020815355E0FF200002384097
:10B3A0000005000F06902B48864204D10698000144
:10B3B0002949451806E02948864203D1069800012C
:10B3C000274945180420E881A8890121C9030840BC
:10B3D000002809D0012069460872A889C004C00865
:10B3E00069890843019007E0002069460872A8892E
:10B3F0001C49084080100190287A6946C8720020D4
:10B4000003E02A5C03A90A54401C6946C97A8142B8
:10B41000F7DCA088172801DB0020A08061881822B3
:10B42000514322460832881818226946FCF725FF46
:10B430006188481C1721FCF79FFE6180A088401C92
:10B44000A0806020875B022038400028A5D007B08C
:10B45000F0BD000000540440005504400058044072
:10B4600000590440FC1F00000020074908800748DD
:10B470000078002803DD00200449087002E0002065
:10B4800003490880704700008200002087000020E8
:10B4900084000020002001490870704786000020C9
:10B4A00010B5A0210C48FCF701FF0B480B49486080
:10B4B0000B480860052008810A48C860002008740D
:10B4C000084B05220649054800F094FE5521034823
:10B4D00000F00AF810BD0000480900208C08002088
:10B4E0003416020005B80000027C80231A40802A2E
:10B4F00000D001747047000010B502461D4BD08982
:10B50000C007C00F00280AD00120D08100E05B1ED8
:10B51000D089C007C00F002801D0002BF7D1D089F7
:10B52000C007C00F002801D0002010BD507A0124B0
:10B5300020435072507A3824A0435072C87A107257
:10B54000487A00280FD1087B1070487B5070887BA8
:10B550009070CC7BD470087C10714C7C5471887CCA
:10B560009071CC7CD471FF200130D0814000D0811B
:10B57000107ADAE7FFFF0000FFB581B004460D4600
:10B580000020012C03D140262E43304306E0002C3E
:10B5900000D103E0022C01D1C0263043012A06D19C
:10B5A000049E760010273E430643F0B206E0002AD0
:10B5B00000D103E0022A01D130263043134E30700F
:10B5C00076788027BE43114F7E70012C08D1FF2171
:10B5D00000BF0E4EB3781E460E4033468B42F8D164
:10B5E0000A4E76784027BE43084F7E70012A0BD161
:10B5F0000026009603E000BF009E761C0096FF2701
:10B600006937009EBE42F6D905B0F0BD0004024085
:10B61000002905D0054A12780243044B1A7004E051
:10B62000024A12788243014B1A707047200402408C
:10B63000002905D0054A927E0243044B9A7604E025
:10B64000024A927E8243014B9A767047000802407C
:10B6500070B5034614460020002B01D1C0B202E0B1
:10B6600005468035E8B2012902D1051DE8B206E0A1
:10B67000022903D105460835E8B200E0C0B2012C2A
:10B6800002D1851CE8B200E0C0B2084DA870AD78C8
:10B6900001263543054EB570002201E000BF521C63
:10B6A0007D252D01AA42F9D970BD0000000C024091
:10B6B00070B500242448007920210840002801D0DA
:10B6C000224D3FE000F046F80546214800788021F1
:10B6D0000840002836D01E4880780840002801D055
:10B6E0001A4D02E000F036F8054619488078000748
:10B6F000840F022C01DBAD0804E0012C01D16D08A0
:10B7000000E000BF124880788007C00F002801D0F9
:10B710002D0101E00C2045430D4800784007840FBF
:10B72000002C02D1601CC4B207E0032C03D1601CC2
:10B730004006040E01E06006040E21462846FCF790
:10B7400005FD0546284670BD0004024000127A003F
:10B75000000C024000B5C0229178F82211401C4A2A
:10B7600012781143EA2923D00ADC0A46E03A130092
:10B7700015F068FA0A181C20242A2A2A2A161A2ADE
:10B78000ED291FD004DCEB2916D0EC291CD117E0E1
:10B79000F02903D0F82917D10E4817E00E4815E01C
:10B7A0000E4813E00E4811E00E480FE00E480DE081
:10B7B0000E480BE00E4809E00E4807E00E4805E091
:10B7C0000E4803E00E4801E00D4800BF00BF00BD79
:10B7D000201C02400090D003006CDC020048E8010D
:10B7E00000366E010024F400001BB70000127A003E
:10B7F000808D5B0000093D00C0C62D0080841E00C6
:10B8000040420F0070B586B004460025002620682F
:10B810000190A1796846C17261794172002101727B
:10B82000017000BF05E020460830415D03A8415586
:10B830006D1C6846C07AA842F5D80B22D201019946
:10B84000881A914237D007DC2C48081A1FD02321D0
:10B850000901401A48D113E0FF386F38002802D0A0
:10B86000012841D105E069462548FFF745FE064617
:10B870003BE0694622484030FFF73EFE064634E092
:10B8800069461F485030FFF737FE06462DE06946EF
:10B890001B482030FFF730FE06461A48008807286C
:10B8A00005DA18480088401C1649088002E000208C
:10B8B0001449088019E005F073FC002813D01248E1
:10B8C00001780078401C104A1070022906DC694695
:10B8D0000B486030FFF710FE064604E000200A49DE
:10B8E00008700A49087000E000BF00BF002E02D1B6
:10B8F000012006B070BD0020FBE700002002000020
:10B9000080550440840000208000002004010020B5
:10B9100010B5A8210A48FCF7C9FC09480949086084
:10B9200009484860072008810020887207220649DC
:10B93000044800F0AFFA00210248FFF715FD10BDE2
:10B94000A008002080080020C01602000C4A1278CF
:10B9500012060B4B5B781B041A43094B9B781B02A6
:10B960001A43074BDB781A43104642084240D20084
:10B9700083085A401146034A5140034A11607047F8
:10B98000430700200102000048070020F8B50446E4
:10B990000F46A07A4006400E002874D10025ACE086
:10B9A0001820684321680818407C01283CD10121F7
:10B9B0001820684322681018017400260CE0182033
:10B9C0006843216808180830815D182068432268A0
:10B9D00010188155701CC6B2082EF0D30021182013
:10B9E00068432268101801741820684322681018F0
:10B9F0004174182068432268101841611820684378
:10BA00002268101881742C20684361680818406A05
:10BA1000002809D018236B432268D0182C236B43CD
:10BA20006268D218516A884718206843216808184C
:10BA30004069FF21C94388425DD8182068432168C6
:10BA400008184069C119182068432268101841611C
:10BA5000182068432168081841692C2068436268EF
:10BA600010188069814246D318206843216808185D
:10BA7000807C55283FD05521182068432268101833
:10BA80008174002624E03CE01820684321680818EF
:10BA9000805D2C216943626851181031895D08402E
:10BAA0001821694322685118885518206843216875
:10BAB0000818805D2C216943626851180831895D3E
:10BAC000084318216943226851188855701CC6B272
:10BAD000082ED9D32C20684361680818806A002892
:10BAE00009D018236B432268D0182C236B4362685B
:10BAF000D218916A8847681C85B22089A84200DD67
:10BB00004EE7F8BD012001490870704798000020F9
:10BB100010B50446002015F05FFA022850D101202C
:10BB200033490880FFF7A0FC32480078002802D192
:10BB30000120304908702F480078012823D12D4872
:10BB40004078401C2B49487021465A20FCF7FEFAE9
:10BB50002849497888424AD8002026494870084632
:10BB60008078401C8870084680780A2803D300201B
:10BB7000887002200870FFF777FC00F075F800204D
:10BB800015F05AFA33E01B48007802282FD11948E3
:10BB90004078401C1749487021467D20C000FCF7C2
:10BBA000D5FA14494978884221D8002011494870B3
:10BBB000FFF75AFC00F058F8002015F03DFA16E0A7
:10BBC0000C48C078401C0B49C8700846C07804284F
:10BBD00004DB0020C8700870487088700448008832
:10BBE000012804D100200249088000F053F810BD5C
:10BBF0007E0000207800002000B587B0FFF734FCFD
:10BC0000002168460171042141710C4802904110E5
:10BC100003910B49049105910A480690FFF778FEBD
:10BC200001A815F049FA00F09BFB00F033F8002161
:10BC3000054809F00FFF07B000BD0000FFFF1F001F
:10BC4000FFFFFF1F355C01000205000030B5034611
:10BC500000201C898C4204D94D015C686419626023
:10BC600000E0022030BD000010B5002400BF09E054
:10BC70001C20604305494018214682680448FFF7AC
:10BC8000E5FF641C052CF3D310BD00003416020040
:10BC90008C08002010B508207A49C872002008736B
:10BCA0000021784841738173C173017441748174B8
:10BCB000C174002073490875FF20023048600020DD
:10BCC00008720120087000204872012088726E48B6
:10BCD000FFF78EFA6B496C48FFF7B6FA01216A4804
:10BCE000FFF712FB6948674948600020087201208D
:10BCF0000870002048720120887263481030FFF7F6
:10BD000077FA604960481030FFF79EFA01215E48DB
:10BD10001030FFF7F9FA5D48401E5A49486000208C
:10BD2000087201200870002048720120887256486D
:10BD30005030FFF75DFA534953485030FFF784FA0B
:10BD4000012151485030FFF7DFFA5048C1384D49C2
:10BD5000486000200872012008700020487201200D
:10BD6000887249484030FFF743FA46494648403018
:10BD7000FFF76AFA012144484030FFF7C5FAFF2077
:10BD800012304049486000200872012008700020ED
:10BD90004872012088723C486030FFF729FA39491F
:10BDA00039486030FFF750FA012137486030FFF71B
:10BDB000ABFAFF202130334948600020087201208F
:10BDC000087000204872012088722F48A030FFF7C9
:10BDD0000FFA2C492C48A030FFF736FA01212A48E7
:10BDE000A030FFF791FA29488F3826494860002093
:10BDF00008720120087000204872012088722248D1
:10BE0000E030FFF7F5F91F491F48E030FFF71CFA53
:10BE100001211D48E030FFF777FA1D4819494860B5
:10BE200000200872012008700020487201208872EA
:10BE300015482030FFF7DCF9124913482030FFF78E
:10BE400003FA012110482030FFF75EFA1048CB308A
:10BE50000C494860002008720120087000204872D8
:10BE60000120887208483030FFF7C2F905490648BA
:10BE70003030FFF7E9F9012103483030FFF744FA89
:10BE800010BD0000D426002010550440020400001C
:10BE900014070000F0B50B461446436004810021EE
:10BEA00036E0002216E02C254D4346687519AD5C3E
:10BEB00018274F430668F619B5542C254D4346689C
:10BEC0007519AD5C18274F430668F6190836B55446
:10BED000551CEAB2082AE6D3002518274F43066806
:10BEE000F619357418274F430668F6197574182724
:10BEF0004F430668F619B57418274F430668F619BC
:10BF0000F57418274F430668F61975614D1CA9B2E0
:10BF100005898D42C5DC00258572F0BD70B50446EB
:10BF2000606800F02DFE0546E27A23460C33294670
:10BF3000094800F0EDFD09496068884204D00749CE
:10BF4000CB396068884206D1E17AA28890B2224655
:10BF50000C3203F0F5F870BD80080020DF07000008
:10BF6000F8B505460026002704F0DCFE07462C46FF
:10BF7000002C25D000BF03E00020A055701CC6B2E5
:10BF8000082EF9D3207808218843F90008221140AF
:10BF900008432070E079E02188430A490988490173
:10BFA000E02211400843E071E07940094001012F8F
:10BFB00001D1082100E00021C906C90E0843E07143
:10BFC000F8BD000084000020FEB5064600250027CD
:10BFD0000020029004F0A8FF019005F0ADF8009059
:10BFE0003446002C64D033480078012858D100BF73
:10BFF00003E000206055681CC5B2082DF9D304F099
:10C000007FFF00280DD005F0BFF8022809D10621D6
:10C010002948FFF7DFF8552803D004F06BFF00280C
:10C0200003D10020207060700FE0019892307D21D4
:10C03000C900884203D80198923087B201E07D2779
:10C04000FF003804000E2070677005F061F80028CA
:10C050000DD005F09FF8022809D106211648FFF7F8
:10C06000B9F8552803D005F04DF8002803D1002079
:10C07000A070E0701CE0009892307D21C9008842D9
:10C0800004D80098923080B2029002E07D20C00077
:10C09000029002980004000EA0700298E07007E081
:10C0A000002503E000206055681CC5B2082DF9D3B7
:10C0B000FEBD00008600002080080020F8B505467F
:10C0C000002605F06DF807462C46002C20D000BF56
:10C0D00003E00020A055701CC6B2082EF9D3012F32
:10C0E0000AD131202070012060705920A0700820F2
:10C0F000E070002020710BE0022F09D13120207068
:10C10000012060705920A0700820E070012020718B
:10C11000F8BD0000FEB50646002500200290019003
:10C1200001F08EFD074604F02DFE0A210090FCF779
:10C1300023F880B2029004F00DFF01903446002CE9
:10C1400023D012480078012817D100BF03E0002057
:10C150006055681CC5B2082DF9D33802000E607115
:10C160003804000EA071E7710198FF2802DDFF205E
:10C17000A0700AE00198A07007E0002503E000200D
:10C180006055681CC5B2082DF9D3FEBD860000209D
:10C19000FEB50646002400200190002704F0E4FBD1
:10C1A00064210090FBF7E8FF80B20190002001F0CD
:10C1B00069FD87B23546002D18D00D48007801285A
:10C1C0000CD100BF03E000202855601CC4B2082C2D
:10C1D000F9D33804000EA870EF7007E0002403E0E4
:10C1E00000202855601CC4B2082CF9D3FEBD000005
:10C1F00086000020FFB581B004460F4600250026CA
:10C20000002000902760039820810498E0600020BF
:10C21000207400BF9DE01C206843216808586A0113
:10C22000616888501C2068432168081880686A018A
:10C230006168891848601C206843216808184068B4
:10C240006A016168891888601C20684321680818A1
:10C25000C0686A0161688918C8601C206843216849
:10C260000818007C6A016168891808741C206843FA
:10C2700021680818407C6A016168891848741C208C
:10C28000684321680818807C6A016168891888837E
:10C290001C20684321680818C07C6A0161688918FD
:10C2A000887400206A0161688918C8741C2068437A
:10C2B000216808184068002813D01C2068432168B2
:10C2C0000818C07C002805D1401E6A0161688918E1
:10C2D000C8831AE00020C0436A0161688918C883D6
:10C2E00013E01C20684321680818C07C002805D092
:10C2F00000206A0161688918C88306E000206A018D
:10C3000061688918C88301200090002607E0002199
:10C310006A016068801814308155701CC6B26901CA
:10C3200060684018808BB042F1DC1C2068432168B3
:10C330000818406900280AD06B016268D2181046BC
:10C3400014301C236B432268D21851698847681C3B
:10C35000C5B22089A84200DD5DE7009805B0F0BDB8
:10C3600000B58DB068480890002108A801716846A2
:10C37000017708A84171002064498872082108A843
:10C38000C171002004E000220AA90A54411CC8B26D
:10C3900008A9C9798142F6DC5D48FEF729FF07A9A3
:10C3A0005B48FEF751FF5848401C0890002108A840
:10C3B00001716846017708A84171002053498872CD
:10C3C000082108A8C171002004E000220AA90A542B
:10C3D000411CC8B208A9C9798142F6DC4C484030FA
:10C3E000FEF706FF07A94A484030FEF72DFF45201B
:10C3F00000010890002108A801716846017708A88B
:10C400004171002041498872082108A8C1710020AB
:10C4100004E000220AA90A54411CC8B208A9C9793B
:10C420008142F6DC3A485030FEF7E2FE07A9384870
:10C430005030FEF709FF112040010890002108A8A4
:10C4400001716846017708A8417100202F49887260
:10C45000082108A8C171002004E000220AA90A549A
:10C46000411CC8B208A9C9798142F6DC28482030AD
:10C47000FEF7BEFE07A926482030FEF7E5FE0B209A
:10C48000C0010890002108A801716846017708A83A
:10C49000417100201D498872082108A8C17100203F
:10C4A00004E000220AA90A54411CC8B208A9C979AB
:10C4B0008142F6DC16486030FEF79AFE07A9144860
:10C4C0006030FEF7C1FE1048A63002900021684699
:10C4D00001730171417381730821C173002004E06D
:10C4E000002204A90A54411CC8B26946C97B814292
:10C4F000F6DC07481030FEF77BFE01A90448103037
:10C50000FEF7A2FE0DB000BDEE060000D42600200E
:10C5100080550440F0B585B004460F46002500263E
:10C52000207C4006400E55287ED100BF76E169018F
:10C5300060684018807C002877D1690160684018E5
:10C5400040686A01616889188968884209D269016E
:10C55000606840184068C0196A01616889184860BD
:10C560005AE1690160684018C068AF49884208D83C
:10C57000690160684018C068401C6A0161688918D8
:10C58000C860690160684018C07C002821D100267D
:10C5900007E000216A016068801814308155701C22
:10C5A000C6B2690160684018808BB042F1DC1C2083
:10C5B000684321680818406900280AD06B01626846
:10C5C000D218104614301C236B432268D2185169CC
:10C5D00088476901606840580090690160684018A8
:10C5E000017C684601710021417169016068401851
:10C5F000017F68468171690160684018417C684626
:10C60000C171002608E06901606840181430815D3E
:10C6100002A88155701CC6B2690160684018808B01
:10C62000B042F0DCE06801E0FCE01DE0002806D04C
:10C630006846E16888476A0161688918C8746901B9
:10C6400060684018C07C002804D16A0161688918BC
:10C650004860E1E06901606840184068C01B6A01F9
:10C66000616889184860D7E069016068401880688F
:10C670000028EED0690160684018C08B0028E8D01F
:10C68000690160684018C08B6A0161688918C968CF
:10C69000884207D1690160684018C08B6249C9436C
:10C6A00088427DD169016068401840686A0161680C
:10C6B00089188968884209D2690160684018406811
:10C6C000C0196A01616889184860A5E000206A0104
:10C6D000616889184860690160684018C0685249FB
:10C6E000884208D8690160684018C068401C6A0127
:10C6F00061688918C860002607E000216A01606847
:10C70000801814308155701CC6B2690160684018E9
:10C71000808BB042F1DC1C20684321680818406916
:10C7200000280AD06B016268D218104614301C230E
:10C730006B432268D2185169884769016068405884
:10C740000090690160684018017C68460171002111
:10C750004171690160684018017F68468171690113
:10C7600060684018417C6846C171002608E0690194
:10C77000606840181430815D02A88155701CC6B2F3
:10C78000690160684018808BB042F0DCE0680028E6
:10C7900008D06846E16888476A016168891800E046
:10C7A00015E0C874690160684018C07C002804D195
:10C7B0006A016168891848602EE069016068401864
:10C7C0004068C01B6A0161688918486024E01C2029
:10C7D000684321680818406800280FD00020C04333
:10C7E0006A0161688918C8831C2068432168081899
:10C7F00040686A0161688918886008E000206A0161
:10C8000061688918C8836A01616889188860002096
:10C810006A0161688918C860681CC5B22089A8428D
:10C8200000DD84E605B0F0BD0000FFFF7CB500BF71
:10C8300019212B480078FBF789FC044629486043FE
:10C84000294A8118002201200DF082F920460A228F
:10C85000504364300119002201200FF0EBF9012050
:10C860000A2262431219D1B20A22624312190090BD
:10C87000D0B201231A4609F01FFCFF220721002035
:10C8800006F034FF0120009001900B206043024627
:10C890000B2060430146002301200EF0E7FE6F20CD
:10C8A0006043014601200FF06BFC104860430246D4
:10C8B000032101200BF0C6FE002505E001212846DA
:10C8C0000BF0FAFD681CC5B20F2DF7DB21460B22D9
:10C8D00051436431C8B20FF0B7FE0FF0A5FE7CBD26
:10C8E0006F000020672B0000A0860100FCB1010052
:10C8F0000020054908700549087005490870054978
:10C900000870054908707047700000207100002011
:10C910006F0000206E0000206D000020F0B589B08F
:10C9200000BF00BF00BF00BF00BF00BF00BF00BF0F
:10C9300000BF00BF00F088F91E2822D361480078AC
:10C940003C2805DA5F480078401C5E49087002E028
:10C950003C205C4908705B4800781D2805DC5A487B
:10C960000078401C584908700BE0574800780028B0
:10C9700002D15549087004E053480078401E5249DE
:10C980000870032150480078FBF7F6FB4F494843F5
:10C99000039005214C480078FBF7D8FB0890032151
:10C9A00049480078FBF7E8FB0B214843643087B225
:10C9B000454909788A0088180621FBF7DDFBFF212D
:10C9C000F531484386B203213F480078FBF7D4FB9A
:10C9D0000B214843643085B203213B480078FBF7C4
:10C9E000CBFB3B4948433B49401804900321364860
:10C9F0000078FBF7C1FB0B214843C0B2069003212E
:10CA000031480078FBF7B8FB0B214843C0B20590D2
:10CA100003212D480078FBF7AFFB6F21484380B21C
:10CA2000079003210120039A0BF00CFE01200899C6
:10CA30000BF0D2FB01233A461846089909F016FE7E
:10CA4000FF21F5313046FBF797FBC0B2014602905B
:10CA500001200AF0EDFA0022294601200FF0EAF841
:10CA60000022012004990DF073F8012007990FF0BE
:10CA700087FB01200346024600900599069809F0BD
:10CA80001BFBFF220721002006F030FE03210E4889
:10CA90000078FBF771FB0B21484384B20120009022
:10CAA00000232246214601900EF0E0FDFF220321E3
:10CAB000002006F01BFEFF220421002006F016FED7
:10CAC00009B0F0BD7100002070000020FCB1010031
:10CAD000672B0000A0860100002000BF06E00021B7
:10CAE000044A1154044A1154411CC8B25A28F6DBB6
:10CAF00070470000782000202C2100200348007A95
:10CB0000002801D10149487070470000240A002024
:10CB1000FFB581B004460F463D462089A8422DDD71
:10CB20001820684321680818007C002826D10026B8
:10CB300009E00498815D18206843226810180830C5
:10CB40008155701CC6B2082EF3D30121182068430A
:10CB50002268101841742C20684361680818006A24
:10CB600000280BD018236B432268D21810460830D7
:10CB70002C236B436268D218116A884705B0F0BD58
:10CB800001460720124BCA1A994211D008DCCA1F6D
:10CB9000FA3A002A14D0102A0CD01F2A14D10DE022
:10CBA000322A0FD0C02A07D0C12A0DD100200DE0B3
:10CBB00001200BE0022009E0032007E0042005E04B
:10CBC000052003E0062001E0072000BF00BF7047FA
:10CBD0004103000010B504467D21C90061430846A9
:10CBE000322103F063FE10BDFF200B4908700020C6
:10CBF000C0430A4908800A490880FF200949087093
:10CC00000949087009490870002009490860094964
:10CC10000860094908607047540000205600002051
:10CC2000580000205A0000205B0000205C0000201B
:10CC3000480000204C0000205000002001480068FF
:10CC4000704700004C000020014800687047000059
:10CC5000480000200148008870470000560000206E
:10CC600001480078704700005B0000200148007810
:10CC7000704700005400002010B510F06FFC012830
:10CC80002CD100F063F8012000F066F803F072FE8A
:10CC9000044600F043F804F053F8044600F04AF864
:10CCA00004F0A0FA012805D100F03EF8012000F0C0
:10CCB00047F805E0002000F037F8002000F040F8C9
:10CCC00000201349086013480068134988421ED2A7
:10CCD00010480068801C0F49086018E000200D49CA
:10CCE00008600B4800680C49884204D20848006874
:10CCF000801C07490860002000F028F8012000F09F
:10CD00002BF8002000F00AF8002000F013F810BD06
:10CD10004C00002048000020FFFFFF7F01490880F1
:10CD2000704700005600002001490870704700005D
:10CD30005B00002001490880704700005800002077
:10CD400001490870704700005C000020014908702C
:10CD5000704700005400002001490870704700002F
:10CD60005A0000200021014A117170470060004004
:10CD7000002201494A7570470060004000220149C5
:10CD80004A767047006000400021014A11727047E6
:10CD9000006000400021014A1173704700600040AC
:10CDA0000021014A11747047006000400021014ACF
:10CDB00011757047006000400021014A11767047EC
:10CDC00000600040002201494A7370470060004043
:10CDD000002201494A7470470060004010B51C4CA5
:10CDE0001C49206888421ED106221B49201DFBF7E2
:10CDF00068FA002817D11222184920460A30FBF79A
:10CE000060FA00280FD10622154920461C30FBF796
:10CE100058FA002807D10622124920462230FBF793
:10CE200050FA00280DD000F051FF0A480E49086062
:10CE3000074814F00AFA0C4A2C21054814F030FA7D
:10CE400004E02C2221460848FBF717FA10BD000029
:10CE5000000850007AA7A55A590700205F07002054
:10CE6000530700204D070020E42A00200020084935
:10CE70000870084908700120074908700020074918
:10CE80000870074807490860002007490870704784
:10CE90003B0700203A0700203D0700204207002002
:10CEA00025060000740700204C07002070B50446DA
:10CEB00000BF9120604305460A212846FBF746F94A
:10CEC0000546284670BD000070B5A8B00546002490
:10CED0000026A0216846FBF7E9F900F067FD1E492E
:10CEE0000A6814216943505000211B48026814202D
:10CEF00068431018416018480268142068431018ED
:10CF0000816015484068002824D000BF17E0600603
:10CF1000060E282E00D316E00F4801681420604347
:10CF20000858B1006A4650500B480168142060430D
:10CF300008184168701C80001150601CC4B206487B
:10CF4000007AA042E3DC00BF620003486946436800
:10CF50000220984728B070BD602B002030B5A9B0E2
:10CF600000240025A02101A8FBF7A0F900BF25E0BF
:10CF70006006050E00F01AFD1F490A68142161437E
:10CF8000505000211C480268142060431018416072
:10CF9000194802681420604310188160282D0BD2B4
:10CFA00015480168142060430858A90001AA505090
:10CFB0000021681C80001150601CC4B20E48007A29
:10CFC000A042D5DC0C484068002813D00A48007AFB
:10CFD0004000282806D30848282201A943680220D7
:10CFE000984707E00448007A4200034801A94368D3
:10CFF0000220984729B030BD602B0020FFB585B0D6
:10D0000005460E461F46002004900390002402901F
:10D0100001900097681C80004149085A0490002D37
:10D0200005D0681E800040184088039003E0A800E7
:10D030003B49085A039003990E98884205D30499F6
:10D040000E98884201D80E9C08E0012E01D1049C64
:10D0500004E0002E01D1039C00E00E9C31480068E2
:10D06000052805D22F480068401C2E49086053E06F
:10D0700000202C49086005210798FBF767F802900B
:10D080000298002844D028480068A04215D22648BB
:10D090000068201A019002990198FBF757F8019057
:10D0A00021480168019808181F490860084600686F
:10D0B000A04217D90846046014E01B480068001B12
:10D0C000019002990198FBF741F801901648016818
:10D0D0000198081A1449086008460068A04201D265
:10D0E00008460460104800680090002E14D10E48D5
:10D0F00000686330B84201D300970DE064210A480C
:10D1000000686330FBF722F864214843009003E095
:10D110000548046000680090009809B0F0BD000068
:10D12000121A0200DC000020E400002008B5FFF71E
:10D130009DFD01287ED1FFF787FD8949884216D2DF
:10D140000F2088498871C87108468078002801D16D
:10D150000520487083488078052802D10020814945
:10D16000487000207F4948728872087047E0FA20B2
:10D170007C498871C8717C49088803F023FD7A488E
:10D180008078002815D17749087008468079C870E2
:10D190000846C079487100208870487088727248CB
:10D1A00000886421484371490860FA206D4908717C
:10D1B00025E001206B4908700846807A022805D1D5
:10D1C000012088720020C870487118E06548807A94
:10D1D000002814D10220634988720846407888707C
:10D1E00008468079C8700846C07948715E48008852
:10D1F000642148435D490860FA205A490871FFF7E5
:10D2000023FD5749884277D3564880785549497855
:10D21000884229DD544800886421484351490090E0
:10D22000C979504B5B79CA1A4E4988784F490B68C7
:10D23000002100E086E0FFF7E1FE4C490860002095
:10D240004849C870087108464079401C4871084632
:10D250004079C979884255DB002042494871084627
:10D260008078401E88704DE03E4880783D4949787E
:10D27000884227DA3C4800886421484339490090B5
:10D280008979384BDB78CA1A3649887837490B6870
:10D290000121FFF7B3FE354908600020314948718C
:10D2A00008710846C078401CC8700846C078897963
:10D2B000884227DB00202B49C87008468078401C34
:10D2C00088701FE0002027494871C870FA20087153
:10D2D0002548008864214843224900900979FA23AF
:10D2E0005A1A2049887821490B680221FFF786FEE7
:10D2F0001E49086006E0FFE71B4800886421484398
:10D300001A49086018488078002803D1012015497F
:10D31000487223E002F094FF732803DB02201149D6
:10D3200048721BE002F08CFF702803DC00200D49DE
:10D33000487213E00B48407A01280FD100200949B8
:10D3400048720BE000200749087008468079C870D1
:10D350000846C079487100204872887208BD0000F4
:10D36000D60B00006C200020D8000020E000002038
:10D370000020044988704870C870487148728872EB
:10D38000704700006C20002000200649088088704B
:10D39000054988704870FA20C870487100204872AA
:10D3A00088727047D80000206C200020F8B5002457
:10D3B00000250026002703F00DFB044603F01CFBAC
:10D3C0000546FFF753FC01282ED105211A48FDF729
:10D3D00001FF552804D1002018498870088027E0F3
:10D3E000012D04D1002015498870088020E001201B
:10D3F000124988701248844202DB201A84B200E08D
:10D4000000240A212046FAF7B7FE052901DB601D3A
:10D4100084B20C48844200DD04460A212046FAF713
:10D42000ABFE0649088003E00020044988700880AC
:10D43000FFF77CFEF8BD000080080020D800002027
:10D44000AA0A0000C60700001CB500200090019049
:10D4500000F0ACFA0B49086000200B49096808602D
:10D460000A48006800280CD00749096808680A21A2
:10D47000FAF76CFE0090012269460520034B1B68F9
:10D4800098471CBD10080020040800200C0800204C
:10D490000020084948800849088008490880084950
:10D4A000087008498872084908804880012008717E
:10D4B000704700002C0000201C0000201E000020EF
:10D4C000200000206408002024000020F8B503F0AC
:10D4D00063FA074603F072FA0090FFF7C7FB0128D2
:10D4E00060D10521C548FDF775FE552802D000988A
:10D4F000012807D10020C2490870C2490880C249EA
:10D50000887256E0BE480078002810D10120BC493E
:10D5100008703D462846E917890F091889030D0C44
:10D52000BA48854200DD0546B648058041E0B64868
:10D53000807A4000B4490F520846867A0EE07000A7
:10D54000B1490D5A701E4000085A7100AE4A50523F
:10D55000701E400011460D52701EC6B2002E08DD2E
:10D560007000A949095A701E4000A74A105A81420A
:10D57000E5DBA548807A401CA34988720846807A7A
:10D58000052816DB002088720846C5882846E9175A
:10D59000890F09188D109D48854200DD0546994880
:10D5A000058006E000209649087096490880964953
:10D5B00088729448058896480088A84257DA9448AB
:10D5C0000088281A84B292480079012827D190480F
:10D5D0004088A0420BDA8E4840880A308C49488047
:10D5E00008464088A04204DD0846448001E088489F
:10D5F00044808748448803212046FAF7BDFD84B261
:10D60000192C00DA19248248008800198049088002
:10D6100008460088A84201DD08460580CDE07C4828
:10D620004088142805DD7A484088143878494880B5
:10D6300002E000207649488075484488032120464E
:10D64000FAF79AFD84B2192C03DA012070490871A7
:10D65000B3E06F480088A04205DD6D480088001BDC
:10D660006B490880A9E0002069490880A5E0684866
:10D670000088A84259DD66480088401B84B264488F
:10D680000079012827D162484088142805DD6048C8
:10D69000408814385E49488002E000205C49488098
:10D6A0005B48448803212046FAF766FD84B2192CB2
:10D6B00003DA0220564908717FE0554800880019B6
:10D6C00053490880084600885049884275DD08465D
:10D6D0004F49088071E04E484088A0420BDA4C4820
:10D6E00040880A304A49488008464088A04204DD04
:10D6F0000846448001E04648448045484488032168
:10D700002046FAF739FD84B2192C00DA1924404872
:10D7100000882919884202DA3D4805804DE03C48DE
:10D720000088001B3A49088047E0394844880321B3
:10D730002046FAF721FD84B2192C3EDD344840889A
:10D74000142805DD3248408814383149488002E009
:10D7500000202F4948802E48448803212046FAF7AC
:10D760000BFD84B22A480079012813D1192C03DA61
:10D7700002202749087120E0254800880019244923
:10D780000880084600882149884216DD084620495D
:10D79000088012E0192C03DA01201D4908710CE001
:10D7A0001B480088A04205DD19480088001B184965
:10D7B000088002E00020164908801648008850289A
:10D7C00004DC134800881349088016E010480088DC
:10D7D00010490988884204DD0D4800880D490880F9
:10D7E0000BE00B4800880B490988081A84B2502CBA
:10D7F00003DB0748008807490880F8BD800800203F
:10D80000200000201C00002064080020E02E000002
:10D81000240000201E00002010B50446642044436C
:10D82000A1212046FAF792FC0446204610BD0000D4
:10D8300010B501200F49087000200F4909680860E1
:10D840000D49096848600C490968886000F07EF954
:10D85000FFF7FAFDFFF782FB08480068002807D0B1
:10D8600001220548016808310020044B1B689847D5
:10D8700010BD0000DD070020D8070020D4070020DD
:10D8800010B5184800681849884229D1174800681F
:10D89000002804D0154800688047154908701548CD
:10D8A0000068002804D013480068804712490870B7
:10D8B00012480068002804D01048006880471049CA
:10D8C000088010480068002805D00E48006880478E
:10D8D0000D49088002E00D480B49088000F078F8F7
:10D8E00010BD0000E807002078563412C40700205D
:10D8F000DC070020C8070020DE070020CC0700203E
:10D90000E0070020D0070020E207002010270000D9
:10D9100010B50023174C2360174C2370174C23704D
:10D92000174C2370174C2380174C2380174C2370FF
:10D93000174C13682360174C53682360164C936888
:10D940002360164CD3682360154C136923600028AC
:10D950000CD0144B1860134C0B682468A360002390
:10D96000104C246823600F4C246863600E4B014CFC
:10D97000236010BDE8070020E4070020DC0700203A
:10D98000DE070020E0070020E2070020DD0700207E
:10D99000C4070020C8070020CC070020D0070020C3
:10D9A000D4070020D80700207856341205480068B4
:10D9B0000549884203D10548006880687047002007
:10D9C000C043FBE7E807002078563412D807002050
:10D9D00070B50024002500263048007801285CD16D
:10D9E0002F480078002858D12E480078012854D1BB
:10D9F0002D4805882D490988694308462C49FAF7BE
:10DA0000A5FB85B2E1200001854207D819216943B1
:10DA100008460921FAF79AFB044600E0244C254801
:10DA200000680068001923490968086021480068F7
:10DA30000068204909684968884207D31D48006882
:10DA400000681C4909684968461A0AE019480068D4
:10DA500040680021C943081A164909680968401836
:10DA6000461C1548864218D3344601462046FAF72C
:10DA70006DFB04460F48006841680F486043081872
:10DA80000C490968486001200C4908700948006881
:10DA90008068001907490968886070BDDC070020AC
:10DAA000DD070020DE070020E0070020E20700205D
:10DAB00010270000D8070020A0860100E4070020FE
:10DAC00000220C4B1A600C4B0A681A600B4B4A6818
:10DAD0001A600B4B8A681A600A4BCA681A600A4BB4
:10DAE0000A691A60002801D0084A1060084A014BF0
:10DAF0001A607047E8070020C4070020C80700200C
:10DB0000CC070020D0070020D4070020D807002031
:10DB10007856341210B50A48006800280ED009481B
:10DB2000007801280AD10020064908700122064821
:10DB3000016808310020024B1B68984710BD0000A7
:10DB4000D4070020E4070020D80700201CB50020DF
:10DB5000009001900024FFF729FF04460E4800685A
:10DB6000046000200C49096848600B490968886016
:10DB70000A48006800280DD0074800680068009037
:10DB80000548006840680190022269460120034B65
:10DB90001B6898471CBD0000EC070020F007002020
:10DBA000F8B505460C4616460027002D17D00E483E
:10DBB0000560FFF7FBFE07462068B84203D90A4814
:10DBC0000068076003E008492068096808600649A2
:10DBD0006068096848600449A0680968C86003482B
:10DBE000066000F005F8F8BDEC070020F007002003
:10DBF00070B500240025FFF7D9FE04460F480068E1
:10DC00000068A04200D903E00C4800680068251AAB
:10DC10000A48006840684019084909688860074850
:10DC20000068806805490968C968884205D90348C1
:10DC30000068C06801490968886070BDEC07002071
:10DC40000148006880687047EC070020002801D078
:10DC5000024A1060024A116070470000EC07002081
:10DC6000F00700200549002005E00A1D135C044A66
:10DC70001354421CD0B22028F7DB70470006500036
:10DC8000142B002001461048026814204843101845
:10DC900082680D480368142048431818C0688242FF
:10DCA0000BD909480268142048431018C268064876
:10DCB000036814204843181882600348026814203F
:10DCC0004843101880687047602B002010B5002171
:10DCD0000022002005E01B4B1C5C1B4B1C54431C0A
:10DCE000D8B20628F7DB1221002006E0174B1C5C97
:10DCF000154B9B1D1C54431CD8B28842F6DB0020F8
:10DD000006E0134B1C5C104B18331C54431CD8B258
:10DD10000628F6DB002006E00E4B1C5C0A4B1E3387
:10DD20001C54431CD8B20628F6DB0422002005E070
:10DD30000024054B24331C54431CD8B29042F7DB1B
:10DD400010BD000059070020E82A00205F070020CE
:10DD5000530700204D07002038B5044600200090EE
:10DD6000009401226946FF202130FBF7CFF938BD2E
:10DD700008B50020009002226946FF204130FBF7E1
:10DD800003F8684600780F49C87168464078087201
:10DD90000846C0790C4948730A48007A88730948D4
:10DDA000407AC8730748807A0874002008730749CE
:10DDB0000860074908600749086007490860074983
:10DDC000087008BD68220020E809002088000020B3
:10DDD0008C0000209000002094000020980000207B
:10DDE00008B50020009002226946FF204130FAF772
:10DDF000CBFF684600781249C871684640780872BF
:10DE000000201049086048600872487288720C4807
:10DE1000C07948730A48007A88730948407AC87301
:10DE20000748807A0874002008730749086007498A
:10DE3000086007490860074908600749087008BD7D
:10DE400068220020E8090020880000208C000020C3
:10DE500090000020940000209800002038B5002495
:10DE60000025002000900121F948FDF7B3F955285D
:10DE70000AD002F005FEF749487302F015FEF54995
:10DE800088730120087308E0F348C079F1494873AA
:10DE9000F148007A8873002008730621EC48FDF7EA
:10DEA00099F9552830D002F033FE002808D002F04E
:10DEB0002FFE401C002803D00120E649087502E02F
:10DEC0000020E449087502F005FE002808D002F0A1
:10DED00001FE401C002803D00120DE49C87402E086
:10DEE0000020DC49C87402F013FE002808D002F0BC
:10DEF0000FFE401C002803D00120D649087507E01A
:10DF00000020D449087503E00020D249C874087580
:10DF1000D048407B00282BD1D0490860D048006809
:10DF2000D049884208D8CE480068401CCC490860D7
:10DF30000020C84948736CE0C748C079022812D055
:10DF4000C548C07903280ED00121C148FDF742F928
:10DF5000552803D00320BF4948735AE0BE48C07912
:10DF6000BC49487355E0BC48C079BA49487350E091
:10DF7000B848407B01282CD10020B9490860B74837
:10DF80000068B849884208D8B4480068401CB349C2
:10DF900008600120AF4948733BE0AF48C0790228D0
:10DFA00012D0AD48C07903280ED00121A848FDF752
:10DFB00011F9552803D00320A649487329E0A64843
:10DFC000C079A449487324E0A348C079A1494873A3
:10DFD0001FE0A048407B022805D10020A04908602E
:10DFE0009E49086015E09B48407B032808D100202B
:10DFF0009B4908609949086003209649487308E0E6
:10E00000002097490860954908609348C079914974
:10E0100048739048807B00282BD19349086093482F
:10E0200000689049884208D890480068401C8F4991
:10E0300008600020874988736CE08748007A0228CE
:10E0400012D08548007A03280ED001218048FDF7C0
:10E05000C1F8552803D003207E4988735AE07E48D2
:10E06000007A7C49887355E07B48007A7949887347
:10E0700050E07848807B01282CD100207B49086043
:10E08000794800687749884208D877480068401C7A
:10E090007549086001206F4988733BE06E48007A3B
:10E0A000022812D06C48007A03280ED0012168485B
:10E0B000FDF790F8552803D003206649887329E0BE
:10E0C0006548007A6349887324E06348007A6149AF
:10E0D00088731FE05F48807B022805D100206349D8
:10E0E00008606149086015E05A48807B032808D120
:10E0F00000205E4908605C49086003205549887328
:10E1000008E0002059490860574908605248C07922
:10E11000504988734F48407B4F49C979884205D19F
:10E120004C48807B4C49097A884251D04948407B11
:10E130004949C979884202D001204649C8734548F7
:10E14000807B4549097A884202D001204149087400
:10E150004048407B022803D03E48407B032817D12B
:10E160003C48407B3C49C979884211D03948407BC2
:10E170003949C8710846C179684601703648017A44
:10E180006846417002226946FF204130FAF7BEFF1F
:10E190003048807B022803D02E48807B032817D18B
:10E1A0002C48807B2C49097A884211D02948807BF1
:10E1B000294908720846C179684601702648017AE3
:10E1C0006846417002226946FF204130FAF79EFFFF
:10E1D00002F060FC044602F073FC054601211C4875
:10E1E000FCF7F8FF552807D100201A490872487239
:10E1F000086048608872B9E0FF2C01D0FF2D77D10C
:10E20000FF2C3FD1FF2D3DD0002012490872012084
:10E210004872174808601748684348604868662194
:10E22000F9F794FF0B494860084640681249884254
:10E2300002D908460749486002F070FF112803DB45
:10E2400002F06CFF192819DD0120024988728DE067
:10E2500080080020E8090020682200208C000020AF
:10E26000880000207017000094000020900000201B
:10E27000DE030000BE0A0000AC26000000205D495D
:10E28000887273E0FF2C29D0FF2D27D10120594936
:10E290000872002048725848486058486043086037
:10E2A00008686621F9F752FF52490860084600687D
:10E2B0005349884202D908464E49086002F026FEBA
:10E2C000112803DB02F022FE172803DD0120494953
:10E2D00088724BE000204749887247E0484845492A
:10E2E0000860486000208872087248723EE0FFE7CC
:10E2F000012040490872487240486043086008683D
:10E300006621F9F723FF3B490860084600683C494D
:10E31000884202D908463749086038486843354979
:10E32000486048686621F9F711FF3249486008469D
:10E3300040683349884202D908462E49486002F0B5
:10E34000E5FD11280BDB02F0E1FD172807DC02F0E8
:10E35000E5FE112803DB02F0E1FE192803DD0120B0
:10E360002449887202E00020224988722148407BBB
:10E37000002802D11F49C87315E01E48407B0128C0
:10E3800002D11C49C8730EE01A48407B022802D112
:10E390001849C87307E01748407B032803D1154983
:10E3A000C873174808601348807B002802D11149C0
:10E3B000087415E00F48807B012802D10D490874CC
:10E3C0000EE00C48807B022802D10A49087407E05D
:10E3D0000848807B032803D1064908740848486030
:10E3E0000448406807490860024800680649086018
:10E3F00038BD0000E8090020DE030000BE0A00006E
:10E40000AC2600009C000020A0000020FFB583B0D7
:10E4100006460D46174600240020029000BF142037
:10E42000784380190190002E57D00198002854D0CD
:10E430002B4806602A49069848600846077200BFC4
:10E4400045E0FFF7B3FA0290200129580298814273
:10E4500004D820012858401C002806D120490298E1
:10E460000A6814216143505006E0200129581C48D5
:10E470000268142060431150200140194068401C7C
:10E48000002807D1002116480268142060431018A4
:10E49000416008E0200140194168114802681420D9
:10E4A0006043101841602001401981680C480268DF
:10E4B000142060431018C16020014019017B0848F6
:10E4C00002681420604310180161601CC4B2044843
:10E4D000007AA042B5DC00F005F807B0F0BD0000FE
:10E4E000602B002070B5002400250026FFF75EFA9F
:10E4F000054600BF4EE02A480168142060430858D2
:10E50000A84239D8264801681420604308582E1ABA
:10E510002348016814206043081840688119204886
:10E52000026814206043101881601D48016814209F
:10E530006043081881681A48026814206043101864
:10E54000C068814224D91648016814206043081825
:10E550000069002803D02046FEF7B6FC18E01048FA
:10E560000168142060430818C1680D48026814202F
:10E570006043101881600BE0094801681420604373
:10E580000818406806490A681421614351188860D8
:10E59000601CC4B20248007AA042ACDC70BD00002E
:10E5A000602B002010B500BF14244C432318002812
:10E5B00005D0002B03D0024C20606260217210BD98
:10E5C000602B0020F8B505460E461446002D04D0F9
:10E5D000012D10D0022D1CD114E01048FAF7DAFA00
:10E5E0000F4908700D48F9F779FE07466421F9F7DD
:10E5F000ADFD30600EE0A004020C31462020FAF799
:10E60000C3FB07E0A004020C31466020FAF7BCFB14
:10E6100000E000BF00BF0020F8BD00005A2200202B
:10E62000F500002070B506460C461546002E04D0B5
:10E63000012E1AD0022E26D11EE02068002802D119
:10E64000FAF730F910E064222168514308460F4977
:10E65000F9F74EFE00200E490870012264210B4894
:10E66000FAF700FC0A4908700EE0A804020C2146E3
:10E670002020FAF74BFD07E0A804020C2146602099
:10E68000FAF744FD00E000BF00BF70BD4C2200203F
:10E69000F400002000B5B5B0502121A8F9F706FE1E
:10E6A00014211CA8F9F702FE00201B90142116A8C3
:10E6B000F9F7FCFD00201390149015901290402162
:10E6C00002A8F9F7F3FD002001904D4908600122EE
:10E6D00021A9FFF777FF2198401C002801D11B904A
:10E6E00001E021981B9047481690474817904748EB
:10E6F00018900020199046481A9016AA1BA9454860
:10E70000FFF706F9022222A90120FFF75BFF2298FA
:10E71000401C002801D1139001E022981390229808
:10E72000401C002801D1149001E0229814903A482E
:10E73000159013A939481A9AFFF732FA042224A92E
:10E740000220FFF73FFF2498401C002801D10290CF
:10E7500001E0249802902598401C002801D10390E4
:10E7600001E0259803902E48049001216846017528
:10E77000881E06902B490891012102A80177881E66
:10E780000A9028490C9101210AA80173881E0E9055
:10E790002449109101210EA80173042202A92248E4
:10E7A0001A9BFFF733FE01221CA9FF202130FAF744
:10E7B000EBFA18A8007CFF2808D101201B498871BA
:10E7C0000122891DFF202130FAF7A0FC02221CA99A
:10E7D000FF204130FAF7D8FA18A8007CFF2809D1A9
:10E7E0000021684601714171022201A9FF204130D8
:10E7F000FAF78CFC0E480249086035B000BD0000F5
:10E80000F80000206DCC000061CC000055CC000069
:10E8100025E60000E021002076841E00EC21002087
:10E820000F2700009F860100FC21002068220020A5
:10E83000A33AA55A00B585B014216846F9F736FD0C
:10E8400000200F4908600F4800900F4801900F48C2
:10E850000290002003900E48049069460D48FFF78F
:10E860002FF90D480499FFF7F1F904210B48049A98
:10E87000FFF798FE0A480249086005B000BD000095
:10E88000F80000206DCC000061CC000055CC0000E9
:10E8900025E60000E0210020EC210020FC210020E2
:10E8A000A33AA55A00200C4908800C4908800C495D
:10E8B000088001200B49087000200B4908730B49A0
:10E8C000088048800120087100200749488008809E
:10E8D000074908607047000034000020360000201F
:10E8E0003C0000203E000020700800204000002076
:10E8F00038000020F8B502F089F8064602F090F8DA
:10E900000746FEF7B3F9012865D10521AB48FCF7AE
:10E9100061FC552807D10020A9490870A949088041
:10E92000A94988805FE0012F07D10020A449087021
:10E93000A4490880A449888055E0A14800780028AF
:10E9400008D101209E49087035460A2068439D4938
:10E95000088048E09C48007B41009B48801D46524F
:10E96000801F047B11E061009748801D455A601E9E
:10E9700041009548801D415A62008152601E41004D
:10E980009148801D4552601EC4B2002C0ADD610012
:10E990008D48801D415A601E42008B48801D805A60
:10E9A0008142E0DB8848007B401C874908730846A9
:10E9B000007B032807DB00200873084605890A202E
:10E9C0006843804908807F4800887F49888001200B
:10E9D0007B49087007E00020794908707949088070
:10E9E00079490873888077480088784908607448B6
:10E9F0000078002815D0084600686C214843734908
:10EA00000860642171480068F9F7A0FB6F4908604D
:10EA1000084600686E49884206D908466B49086076
:10EA200002E000206949086068480068694909886F
:10EA3000884203D2654800680F2804D263480088E2
:10EA4000644908800AE06348008860490968401A00
:10EA50000F2803D35D4800885E4908805A48008823
:10EA6000401C59490880084600880A282CDB0020F1
:10EA700008805948008857490988884203DA0120EC
:10EA80005649087108E0544800885249098888426C
:10EA900002DD02205149087150480079012840D117
:10EAA0004C4800884C49098888420DDB4948018858
:10EAB00049480088FF309130814206DD4648008891
:10EAC000FF3073304449088077E04248018842486B
:10EAD00000889630814205DD3F48008878303E4905
:10EAE00008806AE03B4801883B4800883230814218
:10EAF00005DD394800881E30374908805DE035481B
:10EB00000188354800880A30814205DD3248008896
:10EB10000A303149088050E02E4800882E4908808C
:10EB20004BE02E480079022847D12A4800882A491C
:10EB30000988884239DA27480088FF309130264911
:10EB40000988884206DA24480088FF387338224949
:10EB500008802AE01F48008896301F4909888842AB
:10EB600005DA1D48008878381B4908801DE01948DF
:10EB70000088323018490988884205DA164800882A
:10EB80001E381549088010E0124800880A301249E2
:10EB90000988884205DA104800880A380E4908803A
:10EBA00003E00C4800880C4908800B48008808499D
:10EBB000884202DB084608490880F8BD800800202A
:10EBC0003E000020340000207008002038000020A3
:10EBD000C60700003C000020360000204000002056
:10EBE00000200849088008490880084908804880B2
:10EBF0000120087100200649488008800549086006
:10EC000070470000360000203C000020400000203B
:10EC100070080020380000200020034908700349D4
:10EC20000870034988777047A4000020A5000020E1
:10EC3000000A002070B500250024FEF717F801280F
:10EC40004FD103212A48FCF7C5FA552807D10020E7
:10EC500028490870284908702849887746E02648DE
:10EC60000078002807D101F071FF224908700120C7
:10EC7000214908703AE001201F49087001F066FF41
:10EC80001E49897F1D4A50541046847F08E01B4866
:10EC9000055D601E1949085C0855601E0D54C4B21C
:10ECA000002C06DD1548015D601E144A105C81428F
:10ECB000EDDB1248807F401C104988770846807F32
:10ECC0001E2813DB00208877897B0C4AD27B8918A9
:10ECD0000A4A127C88180321F9F74EFA0549087090
:10ECE00004E00020034908700349087070BD00006B
:10ECF00080080020A4000020A5000020000A0020B9
:10ED0000F0B5A9B004460E46002500270020289043
:10ED1000A0216846F9F7CAFAFEF748FE26490A68B4
:10ED2000142161435050244801681420604308189E
:10ED3000C068B0420CD22048016814206043081813
:10ED4000C1681D480268142060431018416005E046
:10ED50001948016814206043081846601648406846
:10ED6000002826D0002517E06806070E282F00D3BC
:10ED700016E011480168142068430858B9006A4633
:10ED800050500D4801681420684308184168781CE9
:10ED900080001150681CC5B20748007AA842E3DC25
:10EDA00000BF6A0004486946436802209847012072
:10EDB0002890289829B0F0BD602B002010B500F0F5
:10EDC000F9FD00F0D7F810F057FE00F00DFB00F051
:10EDD00001F810BD70B541480078912800D070BD91
:10EDE00000F0BEF8012876D13D4800883D490880F2
:10EDF00008468078F021884320303A4988700846D8
:10EE00008078000900013549097A0907090F08438C
:10EE1000344988703148807A401E304988720846EB
:10EE20000089401C088108460089C988884216DA92
:10EE300008202C49887200240EE028484188284880
:10EE4000001D415C2748C01C015524484088401CD7
:10EE500022494880601CC4B2072CEEDB2DE01F481D
:10EE600000891E49C98888421CD11C4800791B4969
:10EE70008978401AC5B2681C1A49887200240EE0CD
:10EE8000164841881648001D415C1648C01C0155B3
:10EE900012484088401C11494880601CC4B2AC42F2
:10EEA000EEDB0AE000F012FD00200C4908700C496E
:10EEB0000888092100F0B8F991E7012000F0C8FCAA
:10EEC000084A917A1088921C00F070F90549088868
:10EED000002100F0C1F800BF81E700009828002061
:10EEE00034280020C42700201B49097E002932D085
:10EEF0001949897E0C225143174A515A174A1180E9
:10EF000000200CE01449897E0C225143124A8918D2
:10EF1000891C0A5C1149891C0A54411CC8B2082882
:10EF2000F0DB0D49897E0C2251430B4A8918897AFE
:10EF30000A4A91720121D1720749097E491E064A87
:10EF400011761146897E491C91761146897E0229E7
:10EF500001DB00219176704790270020B827002020
:10EF60000349487B012802D10021014A51737047AF
:10EF7000A828002010B533484068002861D13148E6
:10EF8000007B030011F05EFE07590512212E3D4A59
:10EF900059002D480078002807D000202A49087021
:10EFA0002A490888012100F03FF947E02648007807
:10EFB000002809D000202449087025494A8808887B
:10EFC0000123091D00F040F938E01F4800780028AF
:10EFD00007D000201C4908701C490888022100F055
:10EFE00023F92BE018480078002809D000201649A2
:10EFF000087017494A8808880923091D00F024F978
:10F000001CE011480078002807D000200E49087045
:10F010000E490888092100F007F90FE00A48007836
:10F02000002809D000200849087009494A88088842
:10F030000323091D00F008F900E000BF00BF00F045
:10F0400045FC10BDA8280020982800203428002066
:10F05000D02700207047000070B504460D463448A4
:10F060000088A04263D1002D61D132480078222867
:10F070004ED004DC20283DD0212856D141E09028F4
:10F0800002D0912851D115E02A48C08801280AD120
:10F0900000202849087000F019FC27490888002141
:10F0A00000F0C2F805E0032000F0D2FBA0202149C7
:10F0B00008703BE01F4800891E49C98888420AD170
:10F0C00000201C49087000F001FC1B490888002141
:10F0D00000F0AAF80DE01748807A002806D000F06A
:10F0E000F5FB1449087B00F095FB02E0032000F0DB
:10F0F000AFFB1BE0062000F0ABFB11200D490870B0
:10F1000014E0062000F0A4FB11200A4908700DE06D
:10F1100000200849087000F0D9FB08494A8808888F
:10F120000923091D00F090F800E000BF00BF70BD8A
:10F13000AC2700209828002034280020D027002069
:10F1400070B50346184C247E022C00DB70BD164CB3
:10F15000647E0C256C43144D2B5300200AE0155C93
:10F16000114C647E0C2674430F4EA419A41C255424
:10F17000441CE0B28842F2D30B4C647E0C267443EC
:10F18000094EA419A1723446247E641C35462C769F
:10F190002C46647E641C6C762C46647E022C01DB5B
:10F1A00000246C7600BFD1E790270020F0B587B02F
:10F1B00007460D4616461A480780002406E03178B7
:10F1C0001748801C0155761C601CC4B2AC42F6DBAB
:10F1D0002C4605E0AA211248801C0155601CC4B2CF
:10F1E000082CF7DB0E480088029008216846C1739E
:10F1F0000021417301730171002406E00848801C5E
:10F20000015D04A80155601CC4B2082CF6DB01A9FD
:10F210000448FCF771F901200149887207B0F0BD7C
:10F22000AC2700209055044070B504460D46294691
:10F23000204610F043FB70BD70B504460D462946CC
:10F24000204610F049FB70BDF8B504460D46164641
:10F250001F463B4632462946204610F03EFBF8BD8D
:10F26000F8B507460E4615465C480078002804D0DD
:10F2700009213846FFF7D8FFF8BD002D01D0602DD9
:10F2800004DD09213846FFF7CFFFF5E75448078032
:10F290004580002406E031785148001D0155761C58
:10F2A000601CC4B2AC42F6DB00204C4948700846F2
:10F2B0008580FF2088727F20087308468088082890
:10F2C0002EDA0120C8800846808848800120088105
:10F2D000434800884349088008468078F0218843E5
:10F2E0004049887008468078000900013B49097947
:10F2F0000907090F08433B49887038480079401CCA
:10F300008872002407E03648001D015D3548C01CA6
:10F310000155601CC4B231488088A042F3DC4AE049
:10F320000721681CF8F728FF002907D00721284685
:10F330000830F8F721FF2949C88005E00721681C3B
:10F34000F8F71AFF2549C880062024494880012083
:10F350000881234800882349088008468078F021E6
:10F36000884310301F4988700846807800090001E2
:10F370001A4989880905090F08431A4988700846FF
:10F380004088FF2109028843144989880902FF2225
:10F390001202114008431349488008208872002453
:10F3A00007E00F48001D015D0E48001D0155601C5F
:10F3B000C4B2062CF5DB012000F04AFA094A917A22
:10F3C0001088921CFFF7F2FE90200449087005494E
:10F3D00008880021FFF740FE00BF4DE79828002075
:10F3E00034280020C427002010B5FFF77DFD144805
:10F3F000C07A002822D0124880780009002806D060
:10F40000012807D002280AD0032810D10CE000F010
:10F41000A7F90FE000F09EF800F066FA0AE000F0AD
:10F4200011F800F061FA05E000F000F902E0FFF7E2
:10F4300011FE00BF00BF00200149C87210BD0000CE
:10F44000B827002010B53F480078112800D010BD23
:10F450003D4800883D49884200D0F8E73A48807826
:10F460000007000F3749097A0907090F88420CD0B5
:10F4700000203449087000F029FA35494A88088884
:10F480000423091DFFF7E0FEE1E72E480089401C38
:10F490002C4908810846807A401E887208460089F7
:10F4A000C98888421BDA2848807A082800D0CEE72D
:10F4B00000240EE02448C01C015D224842882448F4
:10F4C000001D81541F484088401C1E494880601C14
:10F4D000C4B2072CEEDB062000F0BAF930E0194880
:10F4E000808818494988401A1749897A884203DA7E
:10F4F0001548807A082800D0A9E700240EE01248B9
:10F50000C01C015D0F4842881148001D8154601CD9
:10F51000C4B20C484088401C0A49488009484088C9
:10F52000084989888842EADB00200649087000F013
:10F53000CDF907494A8808880023091DFFF784FE92
:10F5400000BF84E798280020B82700201407000097
:10F55000D027002070B531480078802108408028ED
:10F5600000D170BD2E4800882E49884200D0F8E7AF
:10F570002B48807A082800D0F3E7294880780507CF
:10F580002D0F2D0226484088000A0543082D00DA79
:10F59000E7E700202149487006204880084685801A
:10F5A00001200881082088720020C8728988481CC0
:10F5B0000721F8F7E1FD002909D018498988084694
:10F5C00008300721F8F7D8FD1449C88007E013492F
:10F5D0008988481C0721F8F7CFFD1049C8801048DA
:10F5E00000881149088008464580002407E00C483F
:10F5F000001D015D0C48001D0155601CC4B2062CA5
:10F60000F5DB042000F024F9102004490870064AB4
:10F6100051881088FFF710FE00BFA2E7982800204D
:10F62000B827002014070000D027002010B5484854
:10F630000078A02808D046480078912804D0444893
:10F640000078A12800D010BD424800884249884275
:10F650000AD0424908880921FFF7E6FD00F036F993
:10F6600000203B490870EEE73A48807A08280AD023
:10F670003A4908880921FFF7D7FD00F027F9002053
:10F6800033490870DFE7334880780007000F00280F
:10F6900004D001282DD002284BD136E02C484078E8
:10F6A000002800D050E02B48C078002803D101206A
:10F6B0002749487003E02748C078254988722448C4
:10F6C000007891280BD023480079002803D101202D
:10F6D0001F49087303E01F4800791D4908739120F2
:10F6E0001B49087000F0F2F81949087B00F092F805
:10F6F0002AE017484078002800D025E0A1201449CE
:10F700000870032000F0A4F81EE01148407800289B
:10F7100000D019E00E480078A02809D10F490888C8
:10F720000821FFF781FD00F0D1F80020084908709A
:10F730000AE00A4908880521FFF776FD00F0C6F8BF
:10F7400000200349087000BF00BF00BF7BE7000036
:10F7500098280020B8270020140700003428002033
:10F7600010B52848007880210840802800D110BDBD
:10F7700024480078002805D023480088234988427F
:10F7800000D0F4E72048807A1F4989780907090FDB
:10F79000884203DD1C48807A082800D0E7E71A4831
:10F7A00080780007000F002805D0174880780007F0
:10F7B000000F072800DDDAE71348008814490880A5
:10F7C000114880780007000F4880002407E00E48A9
:10F7D000C01C015D0E48001D0155601CC4B20C48E0
:10F7E0004088A042F3DC00200649087000F06EF863
:10F7F00007494A8808880023091DFFF725FD00BF37
:10F80000B5E7000098280020B82700201407000062
:10F81000D02700207F2805DC7D21C90041430A4A0A
:10F8200091600DE0F12808DBF92806DC0107090FDB
:10F8300064225143044A916002E00449024A916003
:10F840000221014A51737047A828002018F00100D6
:10F8500000B5030011F0F6F90729050B11171D2358
:10F8600029000121144A11731449516022E0022138
:10F87000114A1173114951601CE003210E4A1173A2
:10F880000F49516016E004210B4A11730D49516074
:10F8900010E00521084A1173002151600AE0062199
:10F8A000054A11730849516004E00021024A1173AE
:10F8B000516000BF00BF00BDA8280020A861000063
:10F8C000F824010028230000F0490200002001492B
:10F8D00008737047A8280020024909880918014ABE
:10F8E00011807047A828002010B52E4800781028F5
:10F8F00018D12D48408860280ADD2C4880780009FE
:10F900000001801C2949887022202649087025E0C2
:10F910002648807800090001244988702020214968
:10F9200008701BE01F480078112816D11D48807A06
:10F93000002800D010BD1B484078002800D0F9E70F
:10F940000820184988721948807800090001174971
:10F95000887020201349087000E0EBE71448134931
:10F96000088008468078F021884330300F4988703D
:10F970000846C0780020C870084600791420087135
:10F98000032088720220FFF763FF084A917A1088EB
:10F99000921CFFF70BFC054908880021FFF75CFB70
:10F9A00000BFC7E798280020D0270020C4270020E8
:10F9B00094070000244A118852888A4242D0224A81
:10F9C00052888A4204DA204A52888A1A90B207E0A2
:10F9D0001D4A52880023DB439A1A521C521890B2D7
:10F9E000194A5180127B002A10D0174A5268002A07
:10F9F0000CD0154A5268824205D9134A5268121A2D
:10FA0000114B5A6002E000220F4B5A600E4A527BA3
:10FA1000022A17D10C4A9268002A0CD00A4A92682E
:10FA2000824205D9084A9268121A074B9A6002E08E
:10FA30000022054B9A60044A9268002A02D10122F2
:10FA4000014B5A7370470000A828002010B506F03B
:10FA5000D5F810BD00BF704710B5044621460320FD
:10FA6000400205F0F7FF10BD10B5802103204002D1
:10FA700005F084FF10BD000010B50224024805F017
:10FA8000CDFF0446204610BD0106000010B5002140
:10FA9000014805F073FF10BD0106000010B50446D3
:10FAA0002146024805F0D6FF10BD00000106000007
:10FAB00010B58021014805F061FF10BD010600006E
:10FAC00000B548220249034804F07DFE00BD000055
:10FAD0004C1F0020401F002070B516480088401CB5
:10FAE0001449088001F03CF8044613488079A0428C
:10FAF00004D011498C71084604F012FE0E4804F03F
:10FB000059FEA04202DD0C4804F00AFE002C0FD082
:10FB100001F048F905462946074804F068FE012C23
:10FB200006DD01F087F905462946034804F05FFE2B
:10FB300070BD0000D4000020401F00202E48007837
:10FB4000401C2D4908702D480078401C2B49087036
:10FB50002B480078401C2A4908702A480068401C3D
:10FB60002849086008460068FF219131884202D97F
:10FB700000202449086020480078C82802D90020C5
:10FB80001D4908701D480078842802D900201B49AF
:10FB900008701B480078502802D9002018490870C6
:10FBA000194818490968405C1849087018481249F2
:10FBB0000978405C17490870174810490978405C7B
:10FBC0001649087016480E490978405C15490870B6
:10FBD000154809490978405C1449087014480649D9
:10FBE0000978405C13490870134803490978405C60
:10FBF0001249087070470000830700208407002026
:10FC000085070020880700203F1E02007C07002097
:10FC1000CF1F02007D070020972002007E070020F2
:10FC2000E3210200800700201B2102007F07002043
:10FC30003322020081070020FB22020082070020FD
:10FC400010B58200054BD218525C012A04D1002263
:10FC50008300024C1B195A5410BD000014270020C9
:10FC600010B50446204600F055FA204600F002F890
:10FC700010BD000010B50446B348007800287DD1BF
:10FC8000B2480088B249884278DAB2480078002841
:10FC90004FD0B1480078002803D0AC480088AF4965
:10FCA0000880AF480078002818D1A8480188AB48E0
:10FCB00000880A30814206D30120A9490870A34870
:10FCC0000088A6490880A1480088A449098888427C
:10FCD0001CDA9E480088A149088017E09F480188E7
:10FCE0009A4800880A30814206D300209C49087057
:10FCF000964800889949088094480088974909885F
:10FD0000884203DD9148008894490880944800782F
:10FD1000002858D193480078042803D08E480078F2
:10FD2000002807D089480088822803DA05208D49F9
:10FD30000870A3E08B480078032803D08648007839
:10FD4000002809D081480088FF211931884203DA50
:10FD500004208449087091E082480078022803D08A
:10FD60007D48007800280AD078480088FF21AF310C
:10FD7000884204DA03207B4908707FE0E2E079489A
:10FD80000078012803D074480078002809D06F4813
:10FD90000088AF218900884203DA02207149087087
:10FDA0006CE070480078002803D06B480078002889
:10FDB00064D066480088E121890088425EDA01202B
:10FDC000684908705AE066480078012856D16548AD
:10FDD0000078012803D060480078002809D05B48EB
:10FDE0000088E1218900884203DB00205D4908701A
:10FDF00044E05C480078022803D057480078002887
:10FE000009D052480088AF218900884203DB0120D5
:10FE10005449087032E053480078032803D04E4814
:10FE20000078002809D049480088FF21AF31884276
:10FE300003DB02204B49087020E04A480078042880
:10FE400003D045480078002809D040480088FF21A9
:10FE50001931884203DB0320424908700EE0414813
:10FE60000078052803D03C480078002806D03748A1
:10FE70000088822802DB04203A490870FCF7E4FE7F
:10FE80003349463988425DD33748006800193649FE
:10FE9000086031480078002808D000202E490870FA
:10FEA000314908602F4800783049087000F062FD41
:10FEB00000281FD12C4800682D49884239D30020E2
:10FEC000294908602948007826490978884205DAD6
:10FED00026480078401C254908702AE0234800780D
:10FEE00020490978884224DD20480078401E1F49B7
:10FEF00008701EE01C4800681E49884219D3002083
:10FF0000194908601948007816490978884205DAC5
:10FF100016480078401C154908700AE0134800781C
:10FF200010490978884204DD10480078401E0F49C6
:10FF300008700E4800780B490978884202D10020E9
:10FF40000949086010BD00000B00002002000020DD
:10FF50001C0C0000120000200800002004000020FB
:10FF60000A000020060000201800002007000020E2
:10FF7000C05D0000407E050000200B4908700B4961
:10FF8000087001200A4908700A49087000200A49CF
:10FF900008700A4908700A4908800A4908800A4915
:10FFA00008800A49087070470600002007000020FA
:10FFB00008000020090000200A0000200B0000209B
:10FFC0000C0000200E000020100000201200002075
:10FFD00000200B4908700B49087001200A4908707D
:10FFE0000A49087000200A4908700A4908700A493D
:10FFF00008800A4908800A4908800A490870704741
:020000040001F9
:100000000600002007000020080000200900002052
:100010000A0000200B0000200C0000200E00002031
:100020001000002012000020F8B50646002700242A
:1000300000250020009031480078002809D00320D6
:10004000F9F784FA002804D00320F9F773FA2C4951
:1000500008802C4800880A284AD3002029490880B3
:1000600029480078282829D20320F9F763FA07469F
:10007000002407E060002549085AB84200DD05E089
:10008000601CC4B2204800788442F3DB00BF1E48E5
:10009000057808E0681E40001C49085A69001B4AA0
:1000A0005052681EC5B2A542F4DC600017490F52D9
:1000B00015480078401C1449087019E00020009091
:1000C0000F2407E060001149095A009808180090B1
:1000D000601CC4B2192CF5D30A210098F8F736F841
:1000E0000749088000200849087001200849087065
:1000F00004480088801903490880F8BD09000020E1
:10010000020000201600002000000020140800203B
:1001100012000020394909881E2928DA0021384AAE
:100120001180384A118038490988384A914207DCE1
:1001300037490978002914D033490988914210DCE5
:100140000121344A11700021334A1170334A117071
:100150002F4A11700121324A11700021314A117069
:100160004BE0294909880918274A118045E02349AD
:100170000988264A643291422ADB0021224A1180F2
:10018000204A11801E490988204A914207DC2049F3
:100190000978002916D01A490988914212DC0221F7
:1001A0001C4A117000211C4A117005211B4A117054
:1001B0000021174A11700121194A11700021194AB2
:1001C00011701AE00E49098809180D4A118014E0CF
:1001D00000210D4A11800A4A11800A4909880B4AF8
:1001E000914205DD00210B4A1170094A117004E0AB
:1001F000044909880918034A118070470200002049
:10020000100000200C0000200E000020B80B0000A1
:10021000090000200B00002006000020070000203D
:10022000080000200A000020014800787047000004
:100230006C2000200148407A704700006C200020AC
:1002400010B5642102480068F7F780FF80B210BD46
:10025000E000002001488078704700006C200020FA
:10026000F8B50023002500950024002200BF94E08B
:1002700001259D40ACB20D8825400095009DA5420A
:100280006FD11A468D79012D0DD1464D03263602C8
:10029000AD192D5C012696403543424E03273F029F
:1002A000F61935540CE03F4D03263602AD192D5C8E
:1002B00001269640B5433B4E03273F02F6193554BD
:1002C000CD78002D4ED1374D60352D5CCE78002E87
:1002D00001D1012600E000269640B543314E60363C
:1002E00035548D78002D2ED12E4D19267601AD195D
:1002F0002D5C8E78002E01D1012600E0002696406C
:10030000B543284E19277F01F61935540D79002D74
:100310000ED1244D50352D5C0E79002E01D10126D1
:1003200000E000269640B5431E4E5036355423E07B
:100330001C4D50352D5C0E7996403543EEB2194D6B
:1003400050352E5418E0174D19267601AD192D5C45
:100350008E7896403543134E19277F01F619355490
:100360000AE018E00F4D60352D5CCE78964035439D
:10037000EEB20C4D60352E544D79012D0AD1094D48
:1003800030352D5C012696403543EEB2054D3035B3
:100390002E5400E000BF5D1CABB2082B00DA67E70B
:1003A000F8BD000000000440FFB5074615461E4694
:1003B00000243846019900F01FF8002802D00120DF
:1003C00004B0F0BD00240CE00A2060430949085C39
:1003D000B04204D12946204600F05EF807E0601CD8
:1003E00084B20A2060430349085C0028ECD100BFB6
:1003F0000020E5E7D80100200246002A03D1402969
:1004000001DD01207047032A03D1022901DD01200B
:10041000F8E7042A03D1202901DD0120F2E7052AAB
:1004200003D1202901DD0120ECE70C2A03D110299A
:1004300001DD0120E6E70D2A05D1012903DD402970
:1004400001DA0120DEE70E2A03D1202901D10120A3
:10045000D8E70020D6E7000010B5064A03231B02A8
:10046000D218125C8A43034B032424021B191A542A
:1004700010BD00000000044010B5064A03231B0213
:10048000D218125C0A43034B032424021B191A548A
:1004900010BD00000000044070B502460020B1E02D
:1004A0000A2353435A4C1B195B1C440004191B19A3
:1004B0009B788B427DD10A235343554C1B195B1CFF
:1004C000440004191B195B78082B33D10A235343CA
:1004D0004F4C1B195B1C440004191B574D4C4E4DCF
:1004E0006419E35C012423430A245443484D6419EE
:1004F000641C450045196457464D474EAD192B55B0
:100500000A235343424C1B195B1C440004191B571C
:10051000404C35466419E35C022423430A245443C7
:100520003B4D6419641C450045196457394DAD199C
:100530002B5564E00A235343354C1B195B1C4400C4
:1005400004191B195B78092B34D10A235343304C0F
:100550001B195B1C440004191B572E4C2E4D6419AB
:10056000E35C402423430A245443294D6419641C4A
:10057000450045196457274D274EAD192B550A23C1
:100580005343234C1B195B1C440004191B57214C7B
:1005900035466419E35C8024A3430A2454431C4D6C
:1005A0006419641C4500451964571A4DAD192B5543
:1005B00025E025E00A235343154C1B195B1C44001E
:1005C00004191B57134C144D6419E35C0A2454435B
:1005D0000F4D6419641C45004519641965780124A0
:1005E000AC402343DCB20A235343094D5B195B1C27
:1005F000450045195B57074D074EAD19EC5404E013
:10060000431CD8B2032800DA4AE700BF70BD0000DF
:10061000D80100200000044075080000F8B500244F
:10062000FCF724FB012861D100F064FB0446FF22A3
:100630000721002003F05AF8012C21D100F048FCDA
:1006400000280ED000F068FB054600F059FB064676
:1006500001200346024629460090304605F02CFD55
:1006600050E000F059FB054600F04AFB0646012029
:100670000023024629460090304605F01DFD41E06A
:10068000022C21D100F024FC00280ED000F044FB05
:10069000054600F035FB0646012003460246294682
:1006A0000090304605F008FD2CE000F035FB0546D3
:1006B00000F026FB0646002001231A46294600903A
:1006C000304605F0F9FC1DE000F002FC054600F0A4
:1006D00023FB064600F014FB0746012003462A468A
:1006E00031460090384605F0E7FC0BE00020034659
:1006F00002460146009005F0DFFC0022072110466B
:1007000002F0F4FFF8BD0000FEB50024FCF7AEFADD
:1007100001287DD15B480078012815D1FCF786F8C7
:1007200000BF0EE0182C0AD0152C08D00D2C06D0D6
:100730001A2C04D0FF222146002002F0D7FF601CB3
:10074000C4B2242CEEDB9CE0FCF77EFA4E498842D2
:100750007ED34E480078032805DA4C480078401CC8
:100760004A49087011E000204849087000F0CEFAAC
:10077000064600F0E5FA07460A21F7F7E7FC0546CA
:100780003246294601200BF055FA00F00FFD0646CF
:1007900000F098FC0A210290F7F7D8FC054600F01B
:1007A000B5FA07463246294609F0D2F9FFF736FF77
:1007B00000F08AFA05462946012007F00DFD00F0F9
:1007C000B9FA0646FF21F531F7F7D6FCC5B229463E
:1007D000012006F02DFCFFF727FD0546FFF730FD51
:1007E0000646FFF737FD07462B46324639460120BD
:1007F00005F03CFF00F0C4F80546294601200BF047
:10080000BFFC00F085FC054600F07AFB064600E0E0
:100810002AE000F083FC074600F078FB00233A460C
:10082000014600960195029001200AF01FFFFF2269
:100830000321002002F05AFFFF220421002002F0D1
:1008400055FF00F033FC054600F02AFC064600E0A8
:1008500007E000F031FC07462A46314607F0F2FE79
:100860000FE0FCF75BF80CE0FCF736F9002406E03B
:1008700000222146104602F039FF601CC4B2242C2D
:10088000F6DBFEBD0D010020D60B0000720000203B
:100890000149086070470000B00700200248006866
:1008A000401C014908607047AC070020F3B581B0D7
:1008B000064600200E49086000F01EF8044600F0CD
:1008C0001BF805462F1B3046029903F0B3FF00903A
:1008D0000AE000F011F805462F1B064800680028C2
:1008E00002D004480068804700988742F1D3FEBDDB
:1008F000AC070020B00700200148006870470000E6
:10090000AC0700200B490978012901D101200FE033
:1009100008490978022901D1022009E0054909782E
:10092000032901D1042003E00121024A11700120B2
:10093000704700003D07002010B5094B1B8899B295
:100940000A12C8B2D3433133064C2370C343233356
:10095000637013465633A37003467133E37010BDC2
:1009600074070020430700200148008870470000FA
:100970001C0000200148008870470000340000205F
:100980000148007870470000A4000020014800786A
:1009900070470000A500002010B500220521064880
:1009A000FAF706FC0402012205210348FAF700FCCD
:1009B000201880B210BD00008008002010B506226B
:1009C00005210348FAF7F4FBC006C00F10BD000074
:1009D0008008002010B5042205210648FAF7E8FB3C
:1009E0000402052211460348FAF7E2FB201880B200
:1009F00010BD00008008002010B506220521024825
:100A0000FAF7D6FBC01110BD8008002010B50222F5
:100A100005210248FAF7CCFB10BD00008008002039
:100A200010B5062205210348FAF7C2FB8006C00F65
:100A300010BD00008008002010B5042202210348E8
:100A4000FAF7B6FBC007C00F10BD000080080020F9
:100A500010B5052202210348FAF7AAFBC007C00F10
:100A600010BD00008008002010B5002204210348BA
:100A7000FAF79EFB4006400F10BD000080080020E2
:100A800010B5042201210248FAF792FB801110BD33
:100A90008008002010B5002201210248FAF788FBE7
:100AA00010BD00008008002010B505220121034878
:100AB000FAF77EFB8007800F10BD00008008002041
:100AC00010B5012211460248FAF772FB10BD000072
:100AD0008008002010B5002206210C48FAF768FBB8
:100AE0000402012206210948FAF762FB20180402D9
:100AF000022206210548FAF75BFB201804020322B4
:100B000006210248FAF754FB201810BD8008002087
:100B100010B5042206210C48FAF74AFB040205220C
:100B200006210948FAF744FB201804020622114660
:100B30000548FAF73DFB2018040207220621024867
:100B4000FAF736FB201810BD8008002010B50222ED
:100B500003210248FAF72CFB10BD0000800800209A
:100B600010B5032200210248FAF722FB10BD000055
:100B70008008002010B5002211460248FAF718FB41
:100B800010BD00008008002010B50422002102489A
:100B9000FAF70EFB10BD00008008002010B50122FE
:100BA00000210248FAF704FB10BD00008008002075
:100BB00010B5052200210248FAF7FAFA10BD00002C
:100BC000800800200146322915DA3E488078012845
:100BD00003DD01203B4A507070E03A4880780028DD
:100BE00005DD2F296ADC0020364A507066E00020BF
:100BF000344A507062E03E2917DA322915DB314859
:100C00008078022803DD02202E4A507056E02D48DD
:100C10008078012805DD3B2950DC0120294A5070ED
:100C20004CE00120274A507048E0502917DA3E294D
:100C300015DB24488078032803DD0320214A507007
:100C40003CE020488078022805DD4D2936DC022072
:100C50001C4A507032E002201A4A50702EE062297D
:100C600017DA502915DB17488078042803DD0420A3
:100C7000144A507022E013488078032805DD5F296C
:100C80001CDC03200F4A507018E003200D4A5070FE
:100C900014E073290FDA62290DDB0A4880780428F2
:100CA00005DD70290ADC0420064A507006E00420A5
:100CB000044A507002E00520024A50700148407812
:100CC000704700006C200020014800787047000049
:100CD0000700002000B50249024803F02BFD00BDCB
:100CE000D4000020401F0020014800787047000019
:100CF0000101002001480078704700000001002039
:100D00000148007870470000050100200148007983
:100D100070470000682200200148407870470000BA
:100D200005010020014880797047000068220020FA
:100D30000020704701480088704700001E00002016
:100D400010B50024FFF7E2FF00280AD10A48008806
:100D50000A49884202DB0846074908800648048899
:100D600008E005480088FCF757FD84B20448844237
:100D700000DB0446204610BD36000020C6070000F8
:100D8000CE040000002005490988054A914202DB93
:100D90001146024A11800149088870473600002038
:100DA000C6070000F8B50027002500260024FFF73D
:100DB000E1FE0546FFF7F2FE0646F020284000114E
:100DC0000A2805DBF02028400011C01C044303E082
:100DD000F02028400011044324022807000F0A28AD
:100DE00004DB2807000FC01C044302E02807000FA3
:100DF00004432402F020304000110A2805DBF020D3
:100E000030400011C01C044303E0F02030400011CA
:100E1000044324023007000F0A2804DB3007000FC8
:100E2000C01C044302E03007000F04432746384645
:100E3000F8BD0000F8B50027002500260024FFF7C4
:100E4000A3FE0546FFF7B4FE0646F0202840001139
:100E50000A2805DBF02028400011C01C044303E0F1
:100E6000F02028400011044324022807000F0A281C
:100E700004DB2807000FC01C044302E02807000F12
:100E800004432402F020304000110A2805DBF02042
:100E900030400011C01C044303E0F020304000113A
:100EA000044324023007000F0A2804DB3007000F38
:100EB000C01C044302E03007000F0443002C01D1A2
:100EC0000248F8BD27463846FBE70000FFFF000058
:100ED00001480078704700007D0700200148007835
:100EE000704700007F0700200148C07B704700006A
:100EF000E80900200148C07C70470000E809002094
:100F00000148007A70470000E809002010B500246D
:100F10006421044800683230F7F718F984B220469B
:100F200010BD00009C00002070B500240748006838
:100F3000FBF7BCFF05466421F7F708F984B20448C3
:100F4000844200DD0446204670BD0000A000002061
:100F5000DE03000010B5002400F014F8012800D1D1
:100F60000CE000F00FF8022802D1FF24373405E02E
:100F70000A2103480088F7F7FFF884B2204610BD25
:100F80000200002001480078704700000B0000209C
:100F9000002005490968002903D003490968086849
:100FA00000E002487047000090010020307500000A
:100FB00010B50024044804F031FD002801D00124BC
:100FC00000E00024204610BD0407000010B50024F6
:100FD000044804F023FD002801D0012400E000248F
:100FE000204610BD0507000010B50024044804F099
:100FF00015FD002801D0012400E00024204610BD8A
:101000000707000010B50024062004F007FD0028A3
:1010100001D0012400E00024204610BD10B50024BA
:10102000052004F0FBFC002801D0012400E000248E
:10103000204610BD10B50024044804F0EFFC002841
:1010400001D0012400E00024204610BD0607000066
:1010500010B50024044804F0E1FC002801D001246C
:1010600000E00024204610BD0305000010B5002458
:10107000044804F0D3FC002801D0012400E000243F
:10108000204610BD040500000148807A704700002A
:10109000E80900200148006870470000F8000020BF
:1010A0000148807870470000240A00200148406809
:1010B00070470000240A0020014840787047000073
:1010C000240A002070B50024FFF720FE002803D179
:1010D000FCF7B6FD04460DE0FFF718FE012806D127
:1010E000FCF7AEFD0546FCF797FB044602E0FCF773
:1010F000A7FD0446204670BD0148007C70470000F3
:10110000E80900200148007D70470000E809002040
:101110000148407A70470000E809002010B500241B
:101120006421044800683230F7F710F8C4B2204652
:1011300010BD00009C00002070B500240748006826
:10114000FBF7B4FE05466421F7F700F884B20448C3
:10115000844200DD0446204670BD00009C00002053
:10116000DE03000070B50BF013FB0546002D01D126
:10117000012400E00024204670BD00000148007BEF
:1011800070470000E80900200148407B70470000DC
:10119000E80900200148807B70470000E809002032
:1011A00001480078704700000401002070B5002459
:1011B000FFF7ACFD002803D1FCF764FD04460FE007
:1011C000FFF7A4FD012807D10020FCF75BFD0546D1
:1011D000FCF722FB044603E00020FCF753FD044625
:1011E000204670BD01480078704700003E00002096
:1011F00070B505460024032D00D170BD002D01D02F
:10120000012D1BD181210320800204F0B7FB802136
:10121000134804F0B3FB32211248FFF747FB0024C8
:1012200009E0A200104BD2189178A200985A04F05D
:10123000A5FB601CC4B23B2CF3DB0FE0022D0DD1EB
:10124000002409E0A200094BD2189178A200985A14
:1012500004F094FB601CC4B23B2CF3DB00BFCCE772
:1012600002060000A08601005C140200481502007E
:10127000F8B5002100240023002200BF0AE0012568
:101280008D40ABB205881D402C469C4200D10A46D9
:101290004D1CA9B21029F2DB0588FF2D1FDC284D5B
:1012A0006D7E0688B543264E757635462D7E0688BA
:1012B000B543234E357635466D7E8678F607F60FB4
:1012C000964035431E4E757635462D7E867802272C
:1012D0003E40760896403543194E357622E0184D4B
:1012E000ED7E0688B543164EF5763546AD7E06880A
:1012F000B543134EB5768578ED07ED0F1646083EDB
:10130000B5400F4EF67E35430D4EF57685780226B4
:1013100035406D081646083EB540094EB67E354349
:10132000074EB5760025009505E000BF6D462D7887
:101330006D1CEEB200966D462D78012DF5D9F8BDE5
:10134000206B0440C107C90F002905D00021394A8C
:101350001171002238490A7102210140002905D08B
:101360000021344A1172002233490A7204210140DB
:10137000002905D000212F4A117300222E490A733B
:1013800008210140002905D000212A4A11740022B9
:1013900029490A7410210140002905D00021254A5D
:1013A0001175002224490A7520210140002905D029
:1013B0000021204A117600221F490A76402101406F
:1013C000002904D000221B494A711B494A7180211F
:1013D0000140002904D0002216494A7216494A7277
:1013E000FF2101310140002904D0002211494A7334
:1013F00011494A73012149020140002904D0002209
:101400000C494A740C494A7401218902014000299F
:1014100004D0002207494A7507494A750121C902CB
:101420000140002904D0002202494A7602494A7646
:10143000704700000060004000610040C107C90F14
:10144000002905D001223C490A7100213B4A117153
:1014500002210140002905D0012237490A720021EA
:10146000364A117204210140002905D00122324977
:101470000A730021314A117308210140002905D067
:1014800001222D490A7400212C4A117410210140B7
:10149000002905D0012228490A750021274A117523
:1014A00020210140002905D0012223490A7600218C
:1014B000224A117640210140002905D001221E490F
:1014C0004A7100221D494A7180210140002905D03E
:1014D000012219494A72002218494A72FF2101313A
:1014E0000140002905D0012213494A730022134903
:1014F0004A73012149020140002905D001220E4909
:101500004A7400220D494A740121890201400029D0
:1015100005D0012208494A75002208494A7501216F
:10152000C9020140002905D0012203494A76002260
:1015300002494A76704700000061004000600040A8
:1015400010B50C480078002803D00B4A5068916809
:10155000884708484078002803D0084A50689168B6
:10156000884704488078002803D0054A506891686D
:10157000884710BD0060004028030020A804002018
:101580002806002010B508480079002803D0074A33
:1015900010695169884704484079002803D0044AFB
:1015A00050689168884710BD006000402803002003
:1015B000B404002010B50848007A002803D0074A78
:1015C000D069116A88470448407A002803D0044A49
:1015D00050689168884710BD0060004028030020D3
:1015E000C004002010B50848007B002803D0074A3B
:1015F000906AD16A88470448407B002803D0044A97
:1016000050689168884710BD0060004028030020A2
:10161000CC04002010B50848007C002803D0074AFD
:10162000506B916B88470448407C002803D0044AE3
:1016300050689168884710BD006000402803002072
:10164000D804002010B50848007D002803D0074AC0
:10165000106C516C88470448407D002803D0044A30
:1016600050689168884710BD006000402803002042
:10167000E404002010B50848007E002803D0074A83
:10168000D06C116D88470448407E002803D0044A7E
:1016900050689168884710BD006000402803002012
:1016A000F004002010B50848407F002803D0074A06
:1016B0005068916888470448007F002803D0044A96
:1016C000906DD16D884710BD00600040FC04002083
:1016D0002803002010B508484078002803D0074AA6
:1016E00050689168884704480078002803D0044A6D
:1016F000506E916E884710BD2060004008050020A4
:101700002803002010B509480079002803D0084AB2
:10171000106F516F88470548001D4078002803D09E
:10172000044A50689168884710BD0000206000405E
:10173000280300201405002010B5034AD06F78322A
:101740009168884710BD00002803002010B5024AA8
:1017500050689168884710BDAC03002010B5094857
:10176000007C002803D0084A5068916888470548E3
:1017700010304078002803D0044A506891688847A8
:1017800010BD000020600040B80300203805002094
:1017900010B5024A50689168884710BDC403002004
:1017A00010B5024A50689168884710BDD0030020E8
:1017B00010B50948007F002803D0084A5068916896
:1017C000884705481C304078002803D0044A5068F8
:1017D0009168884710BD000020600040DC030020B5
:1017E0005C05002010B50C480078002803D00B4A97
:1017F00050689168884708484078002803D0084A14
:1018000050689168884704488078002803D0054ACA
:1018100050689168884710BD40600040E803002090
:1018200068050020E806002010B50D480079002862
:1018300003D00C4A5068916888470948001D4078D9
:10184000002803D0084A5068916888470448001D62
:101850008078002803D0054A50689168884710BDF9
:1018600040600040F403002074050020F4060020CE
:1018700010B50D48007A002803D00C4A50689168D2
:101880008847094808304078002803D0084A506843
:1018900091688847044808308078002803D0054ABA
:1018A00050689168884710BD4060004000040020E7
:1018B000800500200007002010B50D48007B00289F
:1018C00003D00C4A50689168884709480C3040782A
:1018D000002803D0084A50689168884704480C30B3
:1018E0008078002803D0054A50689168884710BD69
:1018F000406000400C0400208C0500200C070020F4
:1019000010B50D48007C002803D00C4A506891683F
:101910008847094810304078002803D0084A5068AA
:1019200091688847044810308078002803D0054A21
:1019300050689168884710BD40600040180400203E
:10194000980500201807002010B5024A50689168D9
:10195000884710BD2404002010B50948007E0028E7
:1019600003D0084A50689168884705481830407885
:10197000002803D0044A50689168884710BD0000D1
:101980004060004030040020B005002010B5094838
:10199000007F002803D0084A5068916888470548AE
:1019A0001C304078002803D0044A5068916888476A
:1019B00010BD0000406000403C040020BC05002039
:1019C00010B508480078002803D0074A506891688D
:1019D000884704484078002803D0044A506891683A
:1019E000884710BD6060004048040020C805002002
:1019F00010B509480079002803D0084A506891685A
:101A000088470548001D4078002803D0044A5068E4
:101A10009168884710BD00006060004054040020B9
:101A2000D405002010B50948007A002803D0084AE0
:101A3000506891688847054808304078002803D0EE
:101A4000044A50689168884710BD000060600040FB
:101A500060040020E005002010B5024A506891683B
:101A6000884710BD6C04002010B5024A5068916888
:101A7000884710BD7804002010B50948007D002873
:101A800003D0084A50689168884705481430407868
:101A9000002803D0044A50689168884710BD0000B0
:101AA00060600040840400200406002010B509484E
:101AB000007E002803D0084A50689168884705488E
:101AC00018304078002803D0044A5068916888474D
:101AD00010BD00006060004090040020100600204F
:101AE00010B50948007F002803D0084A5068916863
:101AF000884705481C304078002803D0044A5068C5
:101B00009168884710BD0000606000409C04002080
:101B10001C06002010B5FE4800688079002806D019
:101B200001286ED002286DD003286CD104E2F84859
:101B30000068407903000FF085F80A0614BC2BBC3E
:101B400047BC67BC9BBC0BF0B1F80020F0490968AA
:101B5000C873EF4800684079401CED490968487136
:101B6000AEE0EC490969EA4A1268D27A885C0BF067
:101B700015F9E74800684079401CE5490968487153
:101B8000E34800684079401CE1490968487197E0E2
:101B900001F014FF002810D10BF000F9DC480068B8
:101BA0004079401CDA4909684871D9480068407991
:101BB000401CD7490968487105E00BF0A1F80020E6
:101BC000D349096848717BE001F0F8FE002811D183
:101BD00001200BF0E3F8CE4800684079401CCC4966
:101BE00009684871CA4800684079401CC8490968BA
:101BF000487105E00BF084F80020C5490968487178
:101C00005EE05FE0FEE0A3E101F0D8FE002828D10D
:101C1000BF490968C97A24225143BF4A126889180A
:101C2000BB4A1268D27B885C0BF0B8F8B8480068F1
:101C3000C07B401CB6490968C873B5480068C07BC2
:101C4000242814D3B24800684079401CB049096880
:101C50004871AF4800684079401CAD490968487137
:101C600005E00BF04DF80020A9490968487127E00C
:101C700001F0A4FE002815D1A5480068C07A401CD8
:101C8000A3490968C872A2480068C07AA1490978C6
:101C9000884207DB00209E490968C87201209C49E0
:101CA000096888710BF02CF800209949096848717F
:101CB00006E00BF025F8002095490968487100BF3F
:101CC00000BF4FE192480068407903000EF0BAFF70
:101CD000080513912A91479170910AF0E7FF0020BF
:101CE0008B490968C8738A4800684079401C884954
:101CF0000968487184E087490969854A1268D27A7F
:101D0000885C0BF04BF8824800684079401C8049A1
:101D1000096848717E4800684079401C7C49096820
:101D200048716DE001F04AFE002811D126200BF029
:101D300035F8774800684079401C75490968487152
:101D4000734800684079401C71490968487105E092
:101D50000AF0D6FF00206E490968487150E001F092
:101D60002DFE00281DD101200BF018F868480068EE
:101D7000C07B401C66490968C87365480068C07B21
:101D8000242814D3624800684079401C60490968DF
:101D900048715F4800684079401C5D490968487196
:101DA00005E00AF0ADFF002059490968487127E0B5
:101DB00001F004FE002815D155480068C07A401C87
:101DC00053490968C87252480068C07A5149097875
:101DD000884207DB00204E490968C87202204C493E
:101DE000096888710AF08CFF002049490968487128
:101DF00006E00AF085FF002045490968487100BFE8
:101E000000BFAFE042480068407903000EF01AFFBF
:101E10000805138B2A8B478B638B0AF047FF002042
:101E20003B490968C8733A4800684079401C384902
:101E3000096848717EE037490969354A1268D27AE3
:101E4000885C0AF0ABFF324800684079401C30499A
:101E5000096848712E4800684079401C2C4909687F
:101E6000487167E001F0AAFD002811D125200AF091
:101E700095FF274800684079401C2549096848714A
:101E8000234800684079401C21490968487105E0F1
:101E90000AF036FF00201E49096848714AE001F047
:101EA0008DFD002810D10AF079FF194800684079AB
:101EB000401C174909684871154800684079401C62
:101EC00013490968487105E00AF01AFF002010491B
:101ED000096848712EE001F071FD002815D10C4809
:101EE0000068C07A401C0A490968C872084800683E
:101EF000C07A08490978884207DB0020044909684C
:101F0000C87203200249096888710AF0F9FE05E0E9
:101F100000080020982B0020FC0700200020124918
:101F20000968487106E00AF0EBFE00200E490968D6
:101F3000487100BF00BF15E000200B490968887197
:101F4000094909684871062007490968C87009E00D
:101F50000AF0D6FE00200449096848710249096860
:101F6000887100BF00BF10BD0008002010B56A488E
:101F70000068407903000EF065FE090610C627C60A
:101F800044C6608EC6000AF091FE6348006840793E
:101F9000401C614909684871BCE0604909695E4AB2
:101FA0001268D27A885C0AF0F9FE5B4800684079D2
:101FB000401C594909684871574800684079401CDD
:101FC000554909684871A5E001F0F8FC002811D1D5
:101FD0004F200AF0E3FE504800684079401C4E490B
:101FE000096848714C4800684079401C4A490968B2
:101FF000487105E00AF084FE0020474909684871ED
:1020000088E001F0DBFC002810D10AF0C7FE42484E
:1020100000684079401C4049096848713E480068A2
:102020004079401C3C490968487105E00AF068FEA7
:1020300000203949096848716CE001F0BFFC0028B4
:1020400022D135480068C07A401C33490968C872FB
:1020500031480068C07A3149097888420FDB002096
:102060002D490968C8722C4800684079401C2A49EB
:1020700009684871002028490968486208E0002082
:1020800025490968487103E000202349096848711F
:102090000AF036FE3EE020480068407C002816D05A
:1020A0001E48C068002803D01C48C1681920884712
:1020B000002019490968486217490968487116499A
:1020C00009688871052014490968C8701AE0124827
:1020D0000068406A282807D20F480068406A401C00
:1020E0000D49096848620DE000200B490968486203
:1020F0000949096848710849096888710520064935
:102100000968C87006E00AF0FBFD00200249096872
:10211000487100BF00BF10BD00080020982B0020B0
:1021200010B50024F7480068807A01287ED1F54870
:102130000068C07900287AD0F248006880790028C9
:1021400004D0012874D0022873D191E1ED480068D1
:10215000007B24286ED2EB480068C07901287AD130
:10216000002475E0E7480068C07A24214843E64926
:1021700009684018E3490968097B415CE148006847
:10218000C07A24225043E14A12688018DD4A12685E
:10219000127B805C814229D0DA480068C07A242111
:1021A0004843DA4909684018D6490968097B415C07
:1021B000D4480068C07A24225043D34A1268801859
:1021C000D04A1268127B8154CE480068407B242894
:1021D00005D3CC480068007BCA4909684873C948E0
:1021E0000068007BC7490968887308E0C548006833
:1021F000407B242803D20120C24909688871C14864
:102200000068007B401CBF4909680873BD4800682E
:10221000007B242808D3BB480068407B242803D2D5
:102220000120B84909688871B64805E0D3E1CDE1DD
:1022300069E0BAE138E00EE00068007B242804D2AF
:10224000B04800688079012800D103E0601CC4B266
:10225000242C87D356E0002413E0AA480068C07AF3
:1022600024214843A94909684018015DA548006830
:10227000C07A24225043A44A126880180155601C79
:10228000C4B2242CE9D300209E4909684873232056
:102290009C490968887301209A490968887124203B
:1022A0009849096808732DE0002096490968087369
:1022B00094480068C07A401C92490968C8729148E5
:1022C0000068C07A92490978884217DB8D48006817
:1022D000007C012804D102208A490968887106E03F
:1022E000002088490968887186490968C8710020FA
:1022F00084490968C87283490968087400208149C3
:102300000968487161E17F480068407903000EF078
:1023100099FC080513A62AA651A68EA60120794984
:10232000096808740AF0C2FC764800684079401CCD
:1023300074490968487199E075490969714A1268D8
:10234000D27A885C0AF02AFD6E4800684079401C09
:102350006C49096848716B4800684079401C6949BC
:102360000968487182E001F029FB00281BD165490A
:102370000968497B491CC8B20AF010FD6148006831
:10238000407B60490968C8735E4800684079401C1A
:102390005C49096848715B4800684079401C5949AC
:1023A0000968487105E00AF0ABFC0020554909684E
:1023B00048715BE001F002FB00282BD1514909680C
:1023C000C97A24225143504A126889184D4A12682A
:1023D000D27B885C0AF0E2FC4A480068C07B401C63
:1023E00048490968C87347480068C07B454909687F
:1023F000897B88421ADD434800684079401C414986
:10240000096848713F4800684079401C3D490968A7
:1024100048710BE00AF074FC3A480068407B394987
:102420000968C87300203749096848711EE001F047
:10243000C5FA00280CD13349096888712420314934
:102440000968C8732F49096848732E490968887359
:102450000AF056FC00202B490968487106E00AF092
:102460004FFC002027490968487100BF00BFACE05D
:1024700024480068407903000EF0E4FB08050F8E45
:10248000268E4C8E688E0AF011FC1E48006840793A
:10249000401C1C490968487185E01D490969194AB1
:1024A0001268D27A885C0AF079FC16480068407994
:1024B000401C144909684871124800684079401C62
:1024C0001049096848716EE001F078FA002811D1CE
:1024D00025200AF063FC0B4800684079401C09493C
:1024E00009684871074800684079401C0549096837
:1024F000487105E00AF004FC0020024909684871AF
:1025000051E0000000080020FC070020F807002030
:10251000982B002001F052FA002810D10AF03EFC5E
:10252000644800684079401C624909684871614804
:1025300000684079401C5F490968487105E00AF06D
:10254000DFFB00205B49096848712CE001F036FA96
:1025500000281AD157480068C07A401C55490968BC
:10256000C87254480068C07A5349097888420CDB25
:10257000002050490968C8724E49096888714D4960
:10258000096848714B490968C8710AF0B9FB002015
:1025900048490968487106E00AF0B2FB0020454945
:1025A0000968487100BF00BF0FE00AF0A9FB0020D6
:1025B0004049096848713F49096888713D4909687F
:1025C00008733C490968C87200BF71E000203949AE
:1025D000096888726CE037480068807A022867D101
:1025E00034480068007A00285ED03248006840799C
:1025F000002804D001280CD0032846D11BE00AF0A3
:1026000055FB2C4800684079401C2A4909684871EC
:1026100049E000200AF0C2FB264800684079401CCF
:10262000244909684871234800684079401C2149C1
:102630000968487137E00AF003FB002812D11D48F1
:1026400000684078401C1B490968487019480068B8
:102650004078032812D301F055FA00201549096883
:1026600048700BE00020134909680872AA2011493C
:102670000968887000200F49096848700AF040FB1B
:1026800000200C49096848710DE00AF039FB002070
:10269000084909684871074909684870AA2005492E
:1026A0000968887000BF03E0002002490968887249
:1026B00010BD000000080020982B0020F8B504464B
:1026C0000D4600260C2060431D49085C002801D0FF
:1026D0000120F8BD0C2060431949401885600C208A
:1026E000604340188068002801D10120F1E70121F2
:1026F0000C206043124A115400222046E317DB0EDF
:102700001B185B115B01E31A9B000E4FDB19E717E7
:10271000FF0E3F197F11DA550EF0C6FA002220464F
:10272000E317DB0E1B185B115B01E31A9F00064BDE
:10273000FB18E717FF0E3F197F11DA553046C8E73F
:1027400028030020006000400061004000BFFEE759
:1027500010B51B480088401C1949088008460088AD
:10276000184988422BDD18480078002827D00846F1
:10277000134908801448007801280CD113480078C8
:10278000012808D1002012498870084602F014FF81
:1027900000200E4908700C48007802280CD10D4822
:1027A0000078012808D1002009498870084602F005
:1027B00003FF00200749087000200349087010BD7E
:1027C000FC000020DC0500000001002002010020C8
:1027D000050100200301002070470000002001498E
:1027E00008807047FC000020F0B505460E461746ED
:1027F00000243A463146284600F05EFE00BF42E023
:1028000000202101394A126850522101374A1268CA
:102810008918488000212001344A1268801881807C
:102820002001324A12688018C18020012F4A1268A4
:102830008018017220012D4A12688018417220010F
:102840002A4A1268801881722001284A126880186A
:10285000C17200202101254A1268891808730021DD
:102860002001224A126880184173002021011F4A6A
:10287000126889188873002120011C4A1268801888
:10288000C173601CC4B21A484078A042B8DC64200E
:102890001849096808807D20C000164909684880E9
:1028A00015481449096888807D200001114909688C
:1028B000C88010490968088110480E490968488194
:1028C0000F480C490968888140000A490968C88195
:1028D0003220084909680882FF20F5300549096857
:1028E0004882044909688882F0BD0000C0070020C2
:1028F000B4070020BC0700204C0400001027000093
:102900003075000038B5002404E000201349085554
:10291000601C84B2282CF8D30121684641700170F4
:102920006A460F490D48FFF75FFF7D21C90032203D
:1029300000F0B2F90B490C4800F0CCF909486430BA
:1029400000F05EF90748C83000F06AF9074800F067
:102950007DF9074800F090F938BD0000742200208E
:10296000301A020028230000B80B00005424000095
:102970001027000010B524480078002803D101205A
:10298000214908703EE020480078012810D11F48F6
:102990000078012808D100201D498870084602F0FF
:1029A0000BFE00201949087002201749087029E021
:1029B00015480078022810D116480078012808D15F
:1029C000002013498870084602F0F6FD00201149E6
:1029D000087003200C49087014E00B4800780328A5
:1029E00003D10520084908700CE007480078052845
:1029F00003D005480078062804D100200249087059
:102A00000549087010BD00000001002002010020EF
:102A1000050100200301002004010020F8B5002476
:102A2000002500263548007800281ED1344800785B
:102A3000002803D101203249087016E030480078A0
:102A4000012803D102202E4908700EE02C4800789E
:102A5000022803D103202A49087006E0284800789C
:102A6000032802D100202649087024480078012854
:102A70000ED101241725002622480123324629467B
:102A80000090204601F038FF01201F49087034E013
:102A90001A48007802280FD101243B250026194846
:102AA000401C0123324629460090204601F024FFB5
:102AB00001201649087020E01048007803280DD145
:102AC000FEF724F9002803D101201149087102E022
:102AD00000200F4908710EF087F80EE007480078D3
:102AE000052803D106200549087006E00348007850
:102AF000062802D1052001490870F8BD0001002018
:102B00000101002005010020020100200301002036
:102B10006822002010B5044623000EF093F80961E6
:102B200006101A1B1C1D5F606400FAF78DF82F4910
:102B3000884201D3FFF772FFFFF750FE54E0FAF727
:102B400083F82A49884201D3FFF714FFFFF746FEB6
:102B50004AE049E048E047E0FAF776F8234988423E
:102B600039D301F075FE22480078032814D121489A
:102B70000078002810D1FEF7D5F8002806D10120F2
:102B80001D4988718879FBF7E7F805E000201A49AC
:102B900088718879FBF7E0F815480078012805D19D
:102BA00014480078002801D1FAF7D8F911480078C4
:102BB000052803D10120114908700AE00D4800786A
:102BC000062803D102200D49087002E000200B49BD
:102BD00008700BF0A3FDFFF701FE05E004E003E041
:102BE000FFF7B6FD00E000BF00BF10BDD60B000030
:102BF00001010020000100206822002004010020C3
:102C000001460020054A126852898A4201DC0120EF
:102C100002E0024A1268118170470000BC070020E0
:102C200001460020084A126812898A4201DB01200D
:102C300009E0054A126892898A4201DC012002E01B
:102C4000014A126851817047BC07002001460020EC
:102C5000084A126852898A4201DB012009E0054ACC
:102C60001268D2898A4201DC012002E0014A12681E
:102C700091817047BC07002001460020054A126878
:102C800092898A4201DB012002E0024A1268D18166
:102C900070470000BC070020024600200C4B1B6858
:102CA0001B8A934201DD012010E08A4201DB0120F2
:102CB0000CE0074B1B689B888B4201DC012005E080
:102CC000034B1B681A80024B1B6859807047000039
:102CD000BC070020024600200C4B1B681B8A934255
:102CE00001DD012010E08A4201DB01200CE0074BEE
:102CF0001B685B88934201DB012005E0034B1B68E6
:102D00009A80024B1B68D98070470000BC070020E6
:102D100070B5044600250C206043FE490968401840
:102D20004068002807D00C216143FA4A12688918CC
:102D30004868804705460C206043F6490968085CEE
:102D4000002873D10C206043F2490968401880685C
:102D5000002874D02001F04909684018C07A022880
:102D60000AD1032D08D10C206043EA4A126880186A
:102D700081680120884762E02001E749096840181E
:102D8000C07A02280AD1042D08D10C206043E14A00
:102D90001268801881680220884750E02001DE49CF
:102DA00009684018C07A02280AD1052D08D10C20E4
:102DB0006043D84A126880188168032088473EE043
:102DC0002001D54909684018C07A02280AD1062D89
:102DD00008D10C206043CF4A126880188168042013
:102DE00088472CE02001CC4909684018C07A0228A5
:102DF0000AD1072D08D10C206043C64A12688018FA
:102E00008168052088471AE02001C34909684018F5
:102E1000C07A02280BD1082D09D10C206043BD4A8D
:102E20001268801881680620884708E00DE00C20B1
:102E30006043B84A126880188168002088472001E2
:102E4000B54909684018C5720CE30C206043B149CC
:102E50000968085C012873D10C206043AD490968FA
:102E600040188068002874D02001AB4909684018D8
:102E7000C07A03280AD1022D08D10C206043A54A4C
:102E80001268801881680120884762E02001A24909
:102E900009684018C07A04280AD1022D08D10C20F4
:102EA00060439C4A1268801881680220884750E07D
:102EB0002001994909684018C07A05280AD1022DD5
:102EC00008D10C206043934A12688018816803205F
:102ED00088473EE02001904909684018C07A0628DA
:102EE0000AD1022D08D10C2060438A4A126880184A
:102EF0008168042088472CE0200187490968401830
:102F0000C07A07280AD1022D08D10C206043814ADB
:102F1000126880188168052088471AE020017E49E0
:102F200009684018C07A08280BD1022D09D10C205D
:102F30006043784A1268801881680620884708E054
:102F40000DE00C206043734A1268801881680020ED
:102F500088472001704909684018C57282E20C2038
:102F600060436C490968085C0228F7D1002D7DD1C7
:102F7000200169490968085A68490968098A88422C
:102F800075DA200164490968085A0A3081B22001C3
:102F9000614A1268115220015F490968085A5F4965
:102FA0000968098A884231DB20015B4909684018B9
:102FB00040885A4909680988884227DB2001564918
:102FC00009684018408855490968498888421DDCCD
:102FD00000202101504A12688918488020014E497A
:102FE00009684018807A0028B8D10C20604349490C
:102FF0000968401880680028B0D00C206043454A1A
:10300000126880188168012088472BE2200142491C
:103010000968085A41490968098A88429EDB2001EB
:103020003D490968401840883C49096889888842B8
:1030300094DB2001384909684018408837490968FD
:10304000C98888428ADC00202101334A1268891825
:1030500048802001304909684018807A0028D4D17E
:103060000C2060432B490968401801E063E00BE045
:1030700080680028C9D00C206043264A1268801856
:10308000816802208847EDE100202101224A126870
:10309000891848802101204A12688918C8720021C5
:1030A00020011D4A12688018C18020011A4A126846
:1030B000801841722001184A1268801881721848DD
:1030C00001782001144A1268801801720020210141
:1030D000114A12688918888021010F4A12688918DC
:1030E000087321010C4A12688918487321010A4AA1
:1030F00012688918887300212001074A1268801815
:10310000C1730C2060430349096840188068002897
:10311000B9D007E0B8070020C0070020BC07002096
:10312000B40700200C206043CF4A126880188168E1
:103130000020884796E1012DA5D12001CB490968DF
:103140004018C07AA84225D000212001C74A126841
:103150008018418000202101C44A12688918C88063
:103160002001C24909684018C572C1480078210190
:10317000BE4A12688918487200202101BB4A1268B1
:1031800089188880BA4801782001B84A12688018E6
:10319000017267E12001B54909684018007AB44915
:1031A0000978884220D0B24800782101AF4A1268DD
:1031B000891808722001AD4909684018407AAC4965
:1031C0000978884209D02001A849096840188088F8
:1031D0002101A64A12688918C88000212001A34A4B
:1031E00012688018818012E02001A0490968401807
:1031F0008088A04988420AD220019C490968401869
:1032000080880A302101994A126889188880200133
:103210009649096840184088964988420AD2200198
:1032200092490968401840880A3021018F4A126883
:103230008918488020018D4909684018407A8C49D6
:103240000978884205D001202101884A126889182E
:1032500088722001854909684018408886490968B4
:103260000988884204DB00212001804A126811523B
:1032700020017E4909684018807A00287ED10C2000
:1032800060437949096840188068002877D0200198
:103290007649096840184088774909680989884251
:1032A00014DB2001714909684018007B00280DD10A
:1032B0000C2060436C4A126880188168032088479C
:1032C00001202101694A12688918087320016749A1
:1032D000096840184088684909684989884214DBB0
:1032E0002001624909684018407B00280DD10C205C
:1032F00060435D4A12688018816804208847012075
:1033000021015A4A126889184873200157490968EF
:1033100040184088584909688989884214DB20018F
:10332000524909684018807B00280DD10C20604369
:103330004D4A1268801881680520884701202101C4
:103340004A4A126889188873200148490968401858
:10335000408849490968C989884210DB20014349EE
:1033600009684018C07B00287CD10C2060433E4A8D
:103370001268801881680620884701E007E03BE07A
:1033800001202101394A12688918C8736AE02001B6
:10339000364909684018407A01282ED1344800780F
:1033A00002282AD12001314909684018C0883249D1
:1033B0000968498A884255DB20012C490968401870
:1033C00080882D490968898A88424BDB0C2060433C
:1033D0002549096840188068002843D00C206043C4
:1033E000214A12688018816807208847002021013F
:1033F0001E4A12688918487234E020011B49096886
:103400004018407A02282DD119480078012829D186
:103410002001164909684018C08817490968898A37
:1034200088421FDB20011149096840188088124931
:103430000968498A884215DB0C2060430A490968FB
:103440004018806800280DD00C206043064A12689E
:10345000801881680820884700202101034A1268EB
:103460008918487270BD0000B8070020C00700200E
:10347000B4070020F0FF0000BC07002010B50024B6
:1034800000BF04E02046FFF743FC601CC4B20248C2
:103490004078A042F6DC10BDB407002010B500242F
:1034A000044802F0BBFA002800D000E001242046C6
:1034B00010BD00000304000010B5074B14781C7009
:1034C00054785C70054B1960054B1860034618333F
:1034D000044C236010BD0000B4070020B807002092
:1034E000BC070020C007002010B50446012C09D1FC
:1034F000FF220C21002000F0F9F80121022004F045
:10350000DBFF08E000220C21104600F0EFF800215C
:10351000022004F0D1FF10BD10B50024042108489A
:10352000F7F758FE552801D1012407E0042001F0E7
:1035300077F8002801D0002400E00124204610BDC7
:103540008008002010B50446012C09D1FF221C215F
:10355000002000F0CBF80121062004F0ADFF08E0C8
:1035600000221C21104600F0C1F80021062004F0C2
:10357000A3FF10BD10B50024062001F051F800286B
:1035800001D0012400E00024204610BD10B50446FF
:10359000012C09D1FF221721002000F0A7F80121FA
:1035A000042004F089FF08E000221721104600F0F3
:1035B0009DF80021042004F07FFF10BD0020044985
:1035C000097A002901D0012000E0002070470000A6
:1035D000240A002010B50446022C1CD100220D2123
:1035E000104600F083F8FDF773FC002809D0FF2295
:1035F0000B21002000F07AF801210D2004F05CFF7F
:1036000058E000220B21104600F070F800210D2038
:1036100004F052FF4EE0032C1CD100220B21104677
:1036200000F064F8FDF754FC002809D0FF220D21BA
:10363000002000F05BF801210D2004F03DFF39E08F
:1036400000220D21104600F051F800210D2004F059
:1036500033FF2FE0042C0ED1FF220D21002000F0BB
:1036600045F800220B21104600F040F801210D2002
:1036700004F022FF1EE0012C0ED100220D21104685
:1036800000F034F8FF220B21002000F02FF8012178
:103690000D2004F011FF0DE000220D21104600F076
:1036A00025F800220B21104600F020F800210D2003
:1036B00004F002FF10BD000010B500240A48007895
:1036C000012801D101240CE0FCF7B4FD012801D14F
:1036D000032406E0FCF7AEFD022801D1022400E03D
:1036E0000424204610BD00000D01002010B5064B3B
:1036F0001B78834207DD242905D224234343034C4E
:1037000024681B195A5410BD982B0020F80700207C
:1037100010B574480068407903000DF093FA0B0768
:1037200011D325D35A6D77D38DA8D30009F0BEFAF3
:103730006C4800684079401C6A4909684871CFE0CC
:1037400069494969087809F029FB664800684079A9
:10375000401C644909684871624800684079401C0F
:10376000604909684871BBE000F028F9002811D1D0
:103770007F2009F013FB5B4800684079401C5949E1
:1037800009684871574800684079401C55490968E4
:1037900048711DE0534800684078401C5149096851
:1037A000487050480068407803280BD300204D49EA
:1037B00009684870AA204B49096888700320494964
:1037C0000968C87009F09CFA0020464909684871E8
:1037D00086E000F0F3F8002807D1424800684079FD
:1037E000401C40490968487103E000203D490968D0
:1037F000487109F085FA73E009F058FA3948006811
:103800004079401C37490968487169E0364949697F
:103810000978491CC8B209F0C1FA324800684079F9
:10382000401C3049096848712E4800684079401CA6
:103830002C490968487153E000F0C0F800280FD106
:1038400009F006FA274909688870012009F07AFA18
:10385000244800684079401C22490968487105E005
:1038600009F04EFA00201F490968487138E01D48E8
:103870000068807818280CD102201A49096808705D
:103880000020184909684870042016490968C87062
:1038900011E0144800684078401C124909684870DB
:1038A000104800684078032805D300F02BF9002069
:1038B0000C490968487009F023FA00200949096891
:1038C00048710DE009F01CFA0020064909684871AA
:1038D000044909684870AA2002490968887000BF35
:1038E00000BF10BD00080020982B002010B5314803
:1038F00000684079002804D001280CD0032848D162
:103900001DE009F0D3F92B4800684079401C294993
:10391000096848714BE028490969087809F03EFABE
:10392000244800684079401C2249096848712148B0
:1039300000684079401C1F490968487137E000F071
:103940003DF800280CD101201A49096808700020B0
:10395000184909684870042016490968C87011E0C0
:10396000144800684078401C1249096848701148A2
:1039700000684078032805D300F0C4F800200D4902
:103980000968487009F0BCF900200A4909684871C3
:103990000DE009F0B5F900200649096848710549AC
:1039A00009684870AA2003490968887000BF00BFF1
:1039B00010BD000000080020982B002010B509F071
:1039C0003FF904461F4800680078002838D01D4899
:1039D0000068C078042833D3002C09D1002119488D
:1039E0000068C07A8200174800681430815027E0D0
:1039F00014480068C07A81001248006814304058AA
:103A00001149884211D20F480068C07A81000D48E0
:103A1000006814304058401C0A490968C97A8A0075
:103A200008490968143188500AE000F06BF8002159
:103A300004480068C07A820002480068143081504F
:103A4000204610BD00080020B80B000000B587B06C
:103A50000120694608710A4802900A4803900A4802
:103A600004900A4805900A48069070210948F4F726
:103A70001DFC01A9074800F00FF807B000BD0000C9
:103A8000BD3D0100FD5B0100C50D02009D1A020055
:103A90009C1A0200DC220020F8B506460F460024DE
:103AA00000253946304600F0EFF900BF14E000254C
:103AB0000EE00021242060430B4A12688018415513
:103AC00024206043094A126880184155681CC5B219
:103AD000242DEED3601CC4B205480078A042E6DC79
:103AE00000F010F8F8BD0000F8070020FC070020E7
:103AF000982B0020012002490968087170470000D6
:103B00000008002010B500F073F90020034909688F
:103B1000087002490968C87010BD00000008002044
:103B200007480068C078062808D105480068C079B1
:103B3000002803D1012002490968C87170470000BC
:103B40000008002010B555480068C07803000DF04B
:103B500079F808671D1A1714110E05665048406859
:103B6000002803D04E4841680020884793E000F0C9
:103B7000E5F890E000F0C6F88DE000F0D1F88AE0BA
:103B8000FFF7B4FE87E0FFF7C3FD84E044484068D8
:103B9000002803D042484168012088473F48006818
:103BA000407C00281AD03E48C068002803D03C481A
:103BB000C168C820884700203849096848623748EA
:103BC00000680078002804D0042034490968C870CF
:103BD00024E0022031490968C8701FE02F480068BE
:103BE000406A401C2D49096848622C480068406AB8
:103BF0007D21C900884211D3002028490968486204
:103C0000264800680078002804D004202349096869
:103C1000C87003E0022021490968C8703BE000BF7A
:103C20001F484068002803D01D484168002088478D
:103C30001A480068407C002813D01948C068002842
:103C400003D01748C168C820884700201349096875
:103C5000486212480068C078401C10490968C87062
:103C600018E00E480068406A401C0C490968486228
:103C70000A480068406A7D21C90088420AD30020B2
:103C800006490968486205480068C078401C034935
:103C90000968C87000BF00BF10BD00000008002008
:103CA000982B002010B515480068C078072824D04C
:103CB000012012490968487408E01148806800280A
:103CC00002D00F4988688047FFF73CFF0B48006827
:103CD000C0780628F1D109480068007A0028ECD1A4
:103CE00006480068C0790028E7D104480068807A57
:103CF0000028E2D101490968487410BD000800207D
:103D0000982B002010B5054800680078012802D1E2
:103D1000FDF700FF01E0F5F7E3FC10BD000800200F
:103D200010B5054800680078012802D1FEF71EF999
:103D300001E0F6F7B3F810BD0008002010B51D48EB
:103D40000068807A002829D11A480068007A002883
:103D500003D0022017490968887216480068C079A4
:103D6000002803D0012013490968887211480068AF
:103D70000079012812D100200E49096808710D4907
:103D80000968887207200B490968C8700A484068AA
:103D9000002803D00848416800208847054800688B
:103DA0000078012802D1FEF7BBF901E0F6F750F9DF
:103DB00010BD000000080020982B002010B504461C
:103DC0002146084801F046FE07480078002805D142
:103DD000002C03D032210548FCF768FD024804702E
:103DE00010BD0000010300000E01002050C30000C0
:103DF0000020244909684870AA202249096888706F
:103E000000202049096848621E49096808711D4957
:103E1000096848711B49096888711A490968C8719D
:103E200018490968087217490968887215490968AC
:103E3000C872144909680873242012490968487334
:103E40001049096888730F490968C87300200D4933
:103E5000096808740B49096848740A490968887434
:103E600008490968C874074909684861002105487C
:103E70000068816103480068C1610248006801620E
:103E8000704700000008002010B50A780D4B18603C
:103E9000034628330C4C2360242353430446283420
:103EA0001B190A4C23600A4C4B6863608B68A36043
:103EB000CB68E3604B6963610B6923610B78237006
:103EC00010BD000000080020F8070020FC070020BB
:103ED000982B002007480068C078062808D10548BC
:103EE0000068007A002803D101200249096808729D
:103EF000704700000008002010B50446012C09D1CD
:103F0000FF2220210020FFF7F1FB0121084604F0E9
:103F1000D3FA08E0002220211046FFF7E7FB00213A
:103F2000012004F0C9FA10BD10B50024032000F0F0
:103F300077FB002801D0012400E00024204610BDBA
:103F400010B50446032C0ED1FF2215210020FFF7E7
:103F5000CDFB002214211046FFF7C8FB01210E20E3
:103F600004F0AAFA39E0022C1CD1FCF7B1FF0028BA
:103F700009D0FF2214210020FFF7B8FB01210E20F9
:103F800004F09AFA08E0002214211046FFF7AEFB75
:103F900000210E2004F090FA002215211046FFF7B0
:103FA000A5FB1AE0012C0ED1FF2214210020FFF7FF
:103FB0009DFB01210E2004F07FFA002215211046FE
:103FC000FFF794FB09E0002215211046FFF78EFB56
:103FD000002214211046FFF789FB10BD10B5002404
:103FE000F8F732FE094988420DD3FCF7CBFF0028D1
:103FF00007D1FCF769FE012801DD032404E0022457
:1040000002E0022400E00124204610BDD60B00008F
:1040100010B50446012C09D1FF221D210020FFF715
:1040200065FB0121002004F047FA08E000221D2171
:104030001046FFF75BFB0021084604F03DFA10BD77
:1040400010B50024022000F0EBFA002801D0012472
:1040500000E00024204610BD10B50446012C09D113
:10406000FF221E210020FFF741FB0121092004F05F
:1040700023FA08E000221E211046FFF737FB00213B
:10408000092004F019FA10BD70B50024002500269F
:10409000FCF7D2FC0546FCF7DBFC0646022108488B
:1040A000F7F798F8552800D108E0012E01D1002437
:1040B00004E0012D01D1012400E00024204670BD60
:1040C0008008002010B50446012C09D1FF221F21D1
:1040D0000020FFF70BFB0121082004F0EDF908E0B8
:1040E00000221F211046FFF701FB0021082004F0E9
:1040F000E3F910BD70B500240025FCF727FD054647
:1041000003211A48F7F766F8552806D10120184907
:10411000088000201749088023E0164800880128FD
:1041200011D114490880FCF72BFC762803DA012012
:104130000F49088015E0FCF723FC782811DB0020EC
:104140000B4908800DE001200A490880FCF718FCA3
:10415000762803DA01200649088002E0002004499D
:10416000088003480488204670BD000080080020B5
:104170002C0100202E01002010B50446012C09D18D
:10418000FF2221210020FFF7B1FA0121072004F0CE
:1041900093F908E0002221211046FFF7A7FA002139
:1041A000072004F089F910BD10B50024FCF7DAFFF0
:1041B000012801D1012400E00024204610BD10B5E3
:1041C0000446012C09D1FF2216210020FFF78EFAA8
:1041D0000121032004F070F908E0002216211046A6
:1041E000FFF784FA0021032004F066F910BD10B532
:1041F0000024052000F014FA002801D0012400E07A
:104200000024204610BD10B50446012C09D1FF2220
:1042100019210020FFF76AFA0121052004F04CF96A
:104220003CE0022C17D1FCF753FE002809D0FF22F6
:1042300019210020FFF75AFA0121052004F03CF96A
:104240002CE0002219211046FFF750FA002105202A
:1042500004F032F922E0032C17D1FCF73FFE0028CE
:1042600009D0FF2219210020FFF740FA0121052083
:1042700004F022F912E0002219211046FFF736FA65
:104280000021052004F018F908E000221921104649
:10429000FFF72CFA0021052004F00EF910BD0000F4
:1042A00010B50024FCF73EFD012839D10421404817
:1042B000F6F790FF552803D101203E49087032E0FF
:1042C000FCF7D2FB01280BD0FCF7CEFB022807D06D
:1042D000FCF7CAFB032803D0FCF7C6FB052803D173
:1042E0000120344908701EE0FCF7BEFB042803D10E
:1042F00002203049087016E0FCF7B6FB062803D10F
:1043000003202C4908700EE0FCF7AEFB002803D018
:10431000FCF7AAFB072806D100202649087002E016
:1043200000202449087024480078022813D123482B
:104330000078002807D1FCF7CBFD002803D01D48EA
:1043400000781D490870FCF7C3FD1C490870FCF794
:10435000BFFD044616E018480078032812D117481C
:104360000078002807D1FCF7B9FD002803D01148D8
:10437000007811490870FCF7B1FD10490870FCF78E
:10438000ADFD04460C48007802280ED00A4800789B
:1043900003280AD0074800780749087008460078C3
:1043A000002801D0012400E00024204610BD0000B8
:1043B000800800203001002031010020320100205F
:1043C00010B50446012C0ED1FF221B210020FFF75F
:1043D0008DF900221A211046FFF788F901210A20E1
:1043E00004F06AF81EE0022C0ED1FF221A210020F0
:1043F000FFF77CF900221B211046FFF777F9012116
:104400000A2004F059F80DE000221A211046FFF7A7
:104410006DF900221B211046FFF768F900210A20E0
:1044200004F04AF810BD000010B5002410480078D0
:10443000012801D1012418E0FCF756FD022803D021
:10444000FCF75AFE02280FD1FCF71EFE012809D105
:10445000FCF750FD012803D0FCF754FE012801D1E0
:10446000012402E0022400E00224204610BD0000E6
:104470000D01002010B5F8F7F9FB0446204610BDE9
:1044800010B540210448F3F711FF044B08220449FA
:10449000014800F013F910BD9C2200207544010072
:1044A0003C1A020070B506465C488068002804D0BB
:1044B0005A4988688047054600E000250024A6E0A8
:1044C000564841680C20604308184088A84207D02D
:1044D000524841680C2060430818408802287DD16A
:1044E0004E4841680C2060430818806800280CD0B2
:1044F0004A494A680C2161435118886880474749F6
:104500000968E2008918487009E0444841680C20B5
:104510006043095C41480068E200801841703F48F0
:104520000068E100401840783C490968E200895C75
:1045300088420FD039480068E10040184178374878
:104540000068E2008154002034490968E2008918BB
:1045500048605AE031480068E100401841782F482F
:1045600042680C2060431018407881421FD12B48CC
:104570000068E10040184168284842680C20604308
:104580001018808881420BD824480068E100401848
:104590004068801921490968E2008918486034E0C0
:1045A00001201E490968E200891848802DE01B4857
:1045B0000068E10040184168184842680C206043D8
:1045C0001018C08881420DD814480068E1004018D6
:1045D0004068811911480068E20000E009E0801895
:1045E000416012E000200D490968E2008918488006
:1045F0000BE0002009490968E20089184880002181
:1046000006480068E20080184160601C84B20348DC
:104610008089A04200DD53E770BD0000502B0020D0
:104620000146064A92898A4205DD044A1268CB0097
:10463000D218508800E0002070470000502B002066
:10464000002000BF14E00D494A680C214143511875
:10465000498801290AD10021084A1268C300D218EA
:104660005180064A1268C300D2185160411C88B2BA
:10467000024989898142E6DC70470000502B002006
:10468000002000BF13E00C494A680C214143511837
:104690004988002909D1084A1268C300D2185180FC
:1046A000054A1268C300D2185160411C88B2024901
:1046B00089898142E7DC7047502B0020F0B5044621
:1046C0000020164DAB6069602C60AA8100BF1FE01E
:1046D000124D6E680C254543755D104E3668C70057
:1046E000F61975700D4D6E680C254543755D0B4EC2
:1046F0003668C700F5550025084E3668C700F6191C
:104700007580064E3668C700F6197560451CA8B25C
:10471000024DAD898542DBDCF0BD0000502B00204E
:104720000146002901D1022070470020087148711C
:1047300000BFF9E710B503460C46002B01D0002C52
:1047400001D1002010BD184600F034F8002800D137
:10475000F8E72088FF21F53188420ADB002020801D
:10476000187A401CC0B218725979884201DB187956
:104770001872197A890018684058E3E710B50346A3
:104780000C46002B01D1022010BD184600F012F893
:10479000002800D1F8E7197907E08A0018688058E6
:1047A000A04201D10120EFE7491C58798842F4DC8E
:1047B0000020E9E70146002900D1704748790A79CD
:1047C000801AC0B2F9E70346002B01D0002901D1BD
:1047D00002207047012A01DA0120FAE71960DA7134
:1047E0000020187198715871187200BFF1E730B548
:1047F00004460D46002C01D1032030BD002D01D10F
:104800000420FAE76079401CE179884201DB01204D
:10481000F3E729462046FFF7B1FF002801D0022028
:10482000EBE761798900206845506079401C607130
:104830000020E2E770B505460E46002E05D0314651
:104840002846F3F783FC044600E02C46204670BD62
:1048500010B5FCF787FC012817D10C480078012817
:1048600013D00A48007803280FD0094800780028A0
:104870000BD1FCF78DFB0749884202D108F0F5F80F
:1048800003E07D20000108F0F7F810BD01010020D1
:10489000000100208813000008B5002000900122CC
:1048A0006946FF202130F4F76FFA68460078054921
:1048B0008871002004490870044908700449087090
:1048C00008BD000068220020000100200201002035
:1048D0000301002008B50020009001226946FF2056
:1048E0002130F4F751FA0020024908716846007837
:1048F000887108BD6822002070B5049C257891421B
:1049000016DD01280AD18D4206DAFF26F61AAE42DC
:104910000ED3EE18F5B20BE0154609E0022807D1D8
:10492000954204DD9D4203DBEE1AF5B200E00D4630
:10493000257070BD00BF00BF00BF00BF00BF00BF3B
:1049400000BF00BF00BF00BF00BF00BF00BF00BF6F
:1049500000BF00BF00BF00BF00BF00BF00BF00BF5F
:1049600000BF00BF00BF00BF00BF00BF00BF00BF4F
:1049700000BF00BF00BF00BF00BF00BF00BF00BF3F
:1049800000BF00BF00BF00BF00BF00BF00BF704737
:104990000D4A4168516081699161C168D160416A85
:1049A0005162016A11620168116041695161816857
:1049B0009160C169D16101691161816A91620021CF
:1049C000024A1170704700006C2B0020F407002091
:1049D00010B5FFF735FEF7F78BFFF8F74DF910BD6F
:1049E00010B5F6F741FDF7F783FFFFF749FE0AF030
:1049F00009F90AF0A5F9FBF7BFFAFAF70DF9FFF785
:104A00004BFFF8F7B5FCF6F7FBFAF9F7B1F95521CA
:104A10000448F6F769FDF8F7E1F9F9F723F9FBF730
:104A20004FF810BD8C0800201CB5F6F733FD0020B0
:104A300033490870FCF7DCFB08F0E8F80CF090FA5A
:104A4000F7F7DAF8F9F7CCF9F6F72AFDF8F7C6F92F
:104A5000F9F708F9F5F74EFEF6F73AF9E1204002CA
:104A60000CF05AF800F0B8FAF6F7CAFA08F0CEFAE5
:104A7000F7F73EFFF9F716FFF8F70AFDF8F784FCA1
:104A8000FFF7FEFCFDF73EFFFEF7E0FFFFF70AF938
:104A9000F9F700FEFBF79CFAFAF7BEF8194A1A4933
:104AA00001200AF013FA0022114601200AF052F9FF
:104AB00008F01CF80AF08CF80AF042F9FFF70AFF38
:104AC000002012498871487108710120887048706F
:104AD0001420087007226846F3F7CFFB019900986D
:104AE00001F008F80221012000F0E0FEFAF7E8FFEB
:104AF000F8F77AF8012006490870064908701CBDCD
:104B00000D0100200090D003EC04000020010020E3
:104B100086000020870000207047000010B5044682
:104B2000552C03D105494869804702E003490868CC
:104B3000804700200249087010BD00006C2B002047
:104B4000F407002010B54648007803000CF07AF80E
:104B50000A06111B26303B4650517381414840687C
:104B6000002802D03F494868804701203C4908702E
:104B700000BF3C488068002804D03A4988688047D4
:104B80003749087069E03748C068002802D03549C5
:104B9000C868804703203249087000BF3148006967
:104BA000002804D02F49086980472D49087054E037
:104BB0002C484069002802D02A49486980470020D3
:104BC0002749087049E027488069002802D0254914
:104BD0008869804706202249087000BF2148C069C3
:104BE000002804D01F49C86980471D49087034E077
:104BF00000BF1B48007807280AD11A48006A00281D
:104C000002D01849086A804709201549087011E048
:104C10001348007808280AD11248406A002802D0B8
:104C20001049486A804709200D49087002E00020B9
:104C30000B49087000BF0A480078002808D00948CE
:104C4000806A002804D00749886A804704490870B0
:104C500003E000200249087000BF00BF10BD000043
:104C6000F40700206C2B00207047000010B50020D6
:104C70000CF00EFA09F0A4F809F0F8F809F00EF9B2
:104C800000F008FDF6F7C4F80220FCF7B1FA0020A6
:104C900006490870FFF706F8FEF72CFFFEF752FFF3
:104CA000F5F794FE10200AF027FD10BDC401002086
:104CB00010B50124F7F7DAFF012801D1052407E038
:104CC000F7F7BCFF0349884201D2012400E0022427
:104CD000204610BD8813000010B5062408F03EFCE5
:104CE000002800D1002408F03FFC012803D008F080
:104CF0003BFC072800D90924204610BD10B5F6F763
:104D000087F80022114601200AF056F900213C489C
:104D1000F6F7EAFB00203B490880002400BF00F0C2
:104D20006DFF32217D200001FBF7C0FD00203649D8
:104D300008700AE00022344801781046FEF7D6FCDD
:104D400031480078401C304908702F4800782428EA
:104D5000F0DB00202D49087009E000212B48007885
:104D600009F03EFD29480078401C28490870274872
:104D700000780D28F1DBFEF7E5FEF5F7FDFC08F005
:104D80003FFB23480078401C214908700846007802
:104D9000052812D300200870FEF7C2FE1D480078D7
:104DA0000A2805D300201B490870FFF793F804E098
:104DB00018480078401C1749087008F0D5FB0128F6
:104DC000ADD908F0D1FB0728A9D200200F490870FF
:104DD00008E00E48007809F01DFD0C480078401CE2
:104DE0000A490870094800780D28F2DBF5F770FFD2
:104DF00055210348F6F778FBF7F7F6FE204610BD7D
:104E00008C080020840000202901002027010020B8
:104E1000280100202A01002010B503240BE000F037
:104E2000EDFE012000F0FAFD002802D100F032FD75
:104E300001E0042400E0F2E700BF204610BD0000BE
:104E400010B500202C4908600120FCF7D1F907F0CB
:104E5000DDFEF6F7D1FEF7F7C1FFF8F703FF0CF020
:104E60007FF8F5F747FCF9F7E5FCF5F731FF08F0B7
:104E7000D7FAF8F77DFFF6F7F7FAF6F711FBF9F72F
:104E800011FDF9F7ADFEF8F703FBFFF7F9FAFDF7AF
:104E900039FDFFF7F5FBFFF7FFFCFEF7D7FDFEF747
:104EA00001FF00F099F8E12040020BF035FEF6F723
:104EB000A7F8FBF78DF8F9F7AFFE104A104901206B
:104EC0000AF004F800221146012009F043FF09F01E
:104ED0007FFE09F035FF0221012000F0E7FCFAF720
:104EE000EFFD07F025FEF7F77FFE0120054908706A
:104EF0000549087010BD00004C0000200090D00350
:104F0000EC040000860000208700002010B5072078
:104F1000400200F083FD012812D114480068C8281F
:104F200008D300201249086000210720400200F049
:104F300091FD19E00D480068401C0C49086013E021
:104F40000B480068022805D809480068401C084939
:104F5000086009E000200649086004490860012152
:104F60000720400200F076FD10BD0000CC000020BC
:104F7000D000002070B506460D4614460E48066067
:104F80000E4805600E49206808600E496068086098
:104F90000D49A06808600D49206908600C49E06867
:104FA00008600C496069086005480068002802D064
:104FB00003480068804770BDC0000020C800002082
:104FC000A8000020AC000020B0000020B4000020A9
:104FD000B8000020BC00002000B587B00C4801904C
:104FE0000C4802900C4803900020049005900B4858
:104FF000069000200A49086048600A490860486035
:1050000001AA0121C9020848FFF7B4FF07B000BD9B
:105010002D500100D9530100615301008552010058
:1050200038120020300A002040170020012070476D
:10503000F3B5C3B00446449E0020009057E002E060
:10504000641C761E00BF022E05D32078EB28F7D112
:1050500060789028F4D1072E00D24AE0A778FD1C92
:10506000B54200D945E0A81E205C0002691E615CC3
:1050700008434290042D38D9291FA01C0BF08AFF49
:105080004299884226D11D480068002804D0B91EE4
:10509000E01C1A4A1268904719480068002824D07A
:1050A000E178684601712079811168464171207963
:1050B0008106890E68468171381FC1B26846C17188
:1050C000C279611D02A8F3F7D8F801A80C49096854
:1050D00088470AE00020009002E00098401C009001
:1050E0000098A842F9D3002000906419761B072E7F
:1050F000A5D200BF4498801B45B0F0BDB40000208D
:10510000BC000020F7B5C0B0154600260027E81DFA
:10511000FF210131884202DD002043B0F0BDEB21C8
:105120006846017090214170281DC1B268468170A7
:105130000021C1704098C1B2684601710524002663
:1051400005E04198805D69460855641C761CAE42B6
:10515000F7DBA11E00A802300BF01CFF0746381237
:1051600069460855641C0F55641C064800680028F1
:1051700005D021466846034A12689047CDE70020D3
:10518000CBE70000AC00002070B50024002500260D
:105190001B4840681A490968884200D170BD184808
:1051A000406817490968884205D91548406814497C
:1051B0000968451A07E01248006811494968401A11
:1051C000012189020D1AFF2D01D9FF2600E02E468C
:1051D00000240DE00A4801680830405C0949085580
:1051E00007480088401C8005800D05490860641C44
:1051F000B442EFD3314603480BF0EAFC00BFCDE7E1
:10520000381200204016002070B500251A480068AA
:10521000002830D0194A1288FF230133991A184AFE
:105220001268164B1B88D018134A1268904705461F
:10523000002D20D0114800884019104908800846E8
:1052400001880F480068FFF7F3FE0446002C0DDDCF
:105250000A480088844209DA08480088021B084886
:105260000068011906480068F3F707F8034800884A
:10527000001B0249088070BDB0000020C40000205F
:10528000C000002038B50446002000903049086076
:10529000A07810280CD120792E4908700846007893
:1052A000012853D1002211462020FFF72BFF4DE0AB
:1052B000A078122803D120792649087246E0A07808
:1052C000052803D12079234988723FE0A07802287D
:1052D0001DD120791F4948720846407A012806D11D
:1052E0000090012269460420FFF70CFF2EE01948C8
:1052F000407A02282AD100BFBFF34F8F16481749C2
:10530000C860BFF34F8F00BF00BF00BFFDE7A078AC
:1053100001281BD12079332803D101200D49487081
:1053200005E02079352802D100200A4948706079CB
:1053300008498870607A0006217A09040843E179F7
:1053400009020843A17908430249486038BD0000BA
:10535000CC000020240A00200400FA0500ED00E043
:1053600070B503460022002400251A484068194EF3
:105370003668B04201D1002070BD16484068154E15
:105380003668B04205D913484068124E3668841B0F
:1053900007E0104800680F4E7668801B0126F60271
:1053A000341AA14201D9254600E00D4600220CE046
:1053B000084806680830805D985406480088401CFC
:1053C0004005400D034E3060521CAA42F0D32846DF
:1053D000D2E70000300A002070B503460022002406
:1053E00015484068144D2D68A84208D312484068FB
:1053F000114D2D68401B0125AD022C1A04E00E480A
:1054000000680D4D6D68441BA14201D9012070BD9B
:1054100000220CE09D5C0848466808308555083835
:105420008088401C8005800D034D6860521C8A42B4
:10543000F0D30020EBE700003812002010B502483E
:10544000FFF7A6FA10BD0000241B02000021014A4C
:105450001175704740600040014600BFF0200840D1
:1054600000110A23584302460807000F8018C0B2F3
:1054700070470146002204E0501CC2B208460A38B8
:10548000C1B20A29F8DA1007000E0843704700007D
:1054900010B5044601218020F6F7BAF8607A012899
:1054A00005D14248C078102108434049C870607A4D
:1054B000A22805D13E48007F802108433C49087757
:1054C000607A3B49087700203A4948770846407F90
:1054D0002178084337494877E07B002805D0084603
:1054E000407F20210843334948773248407FC00835
:1054F000C000A17A08432F4948770846807FF721EA
:1055000008402C498877E078FFF7B3FF2949887471
:10551000A078FFF7AEFF2749C8746078FFF7A9FFAE
:10552000244908752078002805D10846007D217996
:10553000084320490875E079FFF79BFF1D498875EE
:105540006079FFF796FF1B494875A079FFF791FF37
:105550001849C875207AFFF78CFF16490876084667
:10556000807F4006400E8877E07A002806D0084603
:10557000807F402108430F49887703E00D48807FF2
:105580000C498877A07BFFF774FF0A498876607B17
:10559000FFF76FFF0749C876207B08770846807FB2
:1055A000102188430349887710BD00002004024081
:1055B00060040440404F044010B504461B48807FFF
:1055C00001210843194988772078FFF752FF1749CE
:1055D00008756078FFF74DFF1449C874A078FFF78D
:1055E00048FF1249887420780C2806DD0846407F61
:1055F000082108430D49487709E00C48407F0B49D2
:1056000048770846007DE17808430849087507484F
:10561000807F400840000549887700BF0348807FAD
:10562000022108400028F9D110BD0000404F04407D
:1056300010B500201449087616200BF029FB002134
:10564000124801761248407F80210843104948776C
:105650000846807F012108430D49887700BF0C4828
:10566000807F022108400028F9D00948807F400847
:1056700040000749887700BF0548807F0221084025
:105680000028F9D110BD000040600040406100409A
:10569000404F044010B50020074908700021202029
:1056A000F5F7B6FF0121054801750020044908758A
:1056B00015200BF0D5FA10BD0050044040610040A9
:1056C0004060004070B504460D46002C14D0002DFB
:1056D00012D0042D10D800F013F800280CD10026A9
:1056E00008E00649885D22460121F3F733FEA41C39
:1056F000701CC6B2AE42F4DB70BD0000A01A0200FE
:1057000000200549897DC907C90F002901D0012062
:1057100000E00020704700000050044030B585B024
:1057200005460C46002003900490009001900290E2
:10573000072C0BDC0120A04081B268468181012149
:10574000C17303A90220FAF78BFD3EE0082C01D0BB
:10575000092C0BD10120A04081B268468181012132
:10576000C17303A90120FAF77BFD2EE00A2C03D0B8
:105770000B2C01D00D2C0BD10120A04081B268462A
:1057800081810121C17303A90020FAF769FD1CE0A2
:105790000C2C01D00F2C0BD10120A04081B2684607
:1057A00081810121C17303A90E20FAF759FD0CE094
:1057B0000E2C0AD10120A04081B2684681810121CE
:1057C000C17303A90C20FAF74BFD00216846017054
:1057D000C17041700121817000210171C1720D21E0
:1057E0008172FF21017200214172F3F717FE034914
:1057F0001520FCF763FF05B030BD00004D540100DB
:1058000010B500201049087515200BF029FA002169
:105810000E4801751520002809DB00BF00BFC20635
:10582000D20E012191400A4A116000BF00BF00BFA3
:10583000084880798011032805D006480078802127
:1058400008430449087010BD4060004040610040BA
:1058500000E100E00050044010B5F3F7D9FE10BDA0
:1058600010B501231A4600211846F5F785FE0122DE
:1058700011461046F5F7ECFEF2F724FC03480BF056
:1058800061FB02480249086010BD00000090D0038F
:105890007807002000BF044800690421084302493A
:1058A000086130BF00BF704700ED00E0F3B585B080
:1058B0000546002400270026002003900490EEB245
:1058C0002804070E0F2F54DA082E52DA002009E0C0
:1058D0000C214143284A515AA94201D1044603E010
:1058E000411CC8B21728F3D300BF0120B04086B2D4
:1058F0000C20604320494018C3780C2060434018B6
:105900008278F8B231460190FAF74EFD68468681FA
:10591000012181730021C17302214174F8B203A9EE
:10592000FAF79EFC0C216143134A8918C888FBF7DB
:1059300085FD0C20604310494018C18868460181EC
:1059400069460698887202A8FBF792FC0C22624313
:10595000094BD21891680C226243D21804201056C9
:10596000FCF7ACFE0C216143034A8918C888FBF799
:10597000E9FC07B0F0BD0000BC1C0200FEB5054606
:105980000C460020C0430290EFB22804060E0F2EF2
:1059900042DA082F40DA0120B840694608808020AA
:1059A0002040002816D101208870A007800F02280F
:1059B00001D1487109E0A007800F012802D1694692
:1059C000487102E0002069464871F0B26946FAF772
:1059D00047FC1FE00020694688700E202040002808
:1059E00000D000BF10202040002802D16946087175
:1059F00002E0012069460871E007C00F002802D1CB
:105A00006946887102E0012069468871F0B26946F2
:105A1000FAF726FC002002900298FEBD30B5014640
:105A2000CAB20C04230E00200F2B0FDA082A0DDA5D
:105A300001249440A2B2064C03252D026419E45CB3
:105A40001440002C01D0012000E0002030BD0000F7
:105A500000000440F8B504460F460020C043009003
:105A6000E6B22004050E0F2D11DA082E0FDA012000
:105A7000B04086B2002F04D1E8B23146FAF7ECFC10
:105A800003E0E8B23146FAF7F7FC002000900098F6
:105A9000F8BD00001649897F01221143144A91770D
:105AA00000BF1349897F022211400029F9D0104913
:105AB000897C81700E49C97C41700D49097D017056
:105AC0000B498A7D8271497D01710949CA7D427104
:105AD0000A7EC271897F49084900054A917700BF53
:105AE0000349897F022211400029F9D17047000043
:105AF000404F044003B585B0002001900290039010
:105B00000490002168464173817E01A8C1706846F7
:105B1000417E01A881706846017E4171002101A883
:105B20000171082168460171817D01A8C171684633
:105B3000C17D4172417D01A881716846017D01A846
:105B40000172002168468173C17301A881730C2121
:105B500041734121684601740021C17401A8FFF717
:105B600097FC18200249888200F004F807B000BDB5
:105B7000204F044010B5FFF75BFD10BD70B5044623
:105B80000D46601E0D49884200D90124002C00D129
:105B9000012440200A4908700846007860430949FA
:105BA00048610321081F0BF08BF80020054988612C
:105BB000072008610448056070BD0000FFFFFF007A
:105BC000A001002000E000E09C0100200020C04374
:105BD000002809DBC206D20E01219140054A11605E
:105BE000BFF34F8FBFF36F8F00BF002002490861E2
:105BF0008861704780E100E000E000E010B50BF044
:105C000005F810BD1A20084908722B2048723C2064
:105C100088724D20C8727F20044909680860AC2052
:105C2000034948707047000000040240A4010020AE
:105C30000010024010B504460F488088002800D1AB
:105C400010BD0D480088182250430B4A08328118B5
:105C500018222046F2F711FB07490988481C172132
:105C6000F2F78AFA88B20449088008468088401E04
:105C700088800120E4E70000A424002010B51C481F
:105C80000078012812D11B480078642809DB022023
:105C900019494871087100201649087014490870A4
:105CA00004E014480078401C12490870134800783A
:105CB00001281CD112480078012804D10020104985
:105CC0000870104908700F48007832280ADBF7F78F
:105CD000CDF800210C48F5F747FB55210B48F5F7A7
:105CE00003FC04E007480078401C0649087010BD1A
:105CF0004107002040070020300700203A0700201D
:105D00003C0700203B070020800800208C08002072
:105D1000F8B504460D46002700200090032000033C
:105D2000204000130090102C04D0122C02D01148F7
:105D3000844217D122202840222806D127073F0F6E
:105D400039460098F4F7C2FC064612202840122873
:105D50000ED12007000F471C39460098F4F7B6FC17
:105D6000064605E02107090F0098F4F7AFFC064648
:105D70003046F8BD10100000F8B504460D46002668
:105D800000270120000320400713102C04D0122C00
:105D900002D00F48844215D122202840222805D164
:105DA0002607360F31463846F9F74AFF12202840B9
:105DB00012280CD12007000F461C31463846F9F74F
:105DC0003FFF04E02107090F3846F9F739FFF8BD16
:105DD00010100000FFB58BB01C4600200790069005
:105DE00005903848049010210B980840002801D0F5
:105DF000022707E040210B980840002801D0012726
:105E000000E00027002C04D01498047001200890B2
:105E100001E010200890002548E0002C08D025461D
:105E20006000294A115A0C98F2F790F9079006E0A1
:105E30006800254A115A0C98F2F788F907903E46F7
:105E400030E0711C0798F2F781F9400806900D9830
:105E5000F2F7D2FA03900D9A0699881AF2F7CCFA63
:105E600018490190F2F74DFA02900399F2F786FA79
:105E700005900598F2F7C7FA490049080391029086
:105E80000498F2F7C0FA4900490801910090039B79
:105E9000029AF2F7CDFA03D20A9509960598049072
:105EA000701CC6B27F2ECCDD681CC5B20898854236
:105EB000B3DB14990A9808701499099848700498EB
:105EC0000FB0F0BD0000C842D01D02000246412ABA
:105ED0002ED010DC212A2AD006DC102A45D0122A26
:105EE0004BD0202A59D11CE0222A26D0232A2AD09E
:105EF000402A52D116E081235B01D01A9A4228D061
:105F000008DC422A1AD0432A1ED02548101800283F
:105F100043D13AE0012822D020281BD021283CD1AF
:105F20001EE000BF1F4803890B43038136E000BF1A
:105F30001C4843890B43438130E000BF19488389E3
:105F40000B4383812AE000BF1648C3890B43C381FA
:105F500024E000BF144883880B4383801EE000BF09
:105F60001148C3880B43C38018E00E4843890B4394
:105F7000438103890B43038110E00A48C3890B4323
:105F8000C38183890B43838108E00748C3880B439F
:105F9000C38083880B43838000E000BF00BF70474D
:105FA000F0EFFFFF0011044000140440F0B5054677
:105FB0000E46412D30D010DC212D2CD006DC102DCA
:105FC00051D0122D56D0202D62D11CE0222D2AD086
:105FD000232D30D0402D5BD116E081214901681A74
:105FE0008D4230D008DC422D1ED0432D24D02A48CB
:105FF000281800284CD144E001282CD0202823D098
:10600000212845D128E000BF244F3888314600F0D0
:1060100049F804463DE000BF204F7888314600F043
:1060200041F8044635E000BF1C4FB888314600F007
:1060300039F804462DE000BF184FF888314600F0CB
:1060400031F8044625E000BF154F3888314600F08E
:1060500029F804461DE000BF114F7888314600F052
:1060600021F8044615E00D4F7888314600F01AF803
:1060700004460EE0094FF888314600F013F8044654
:1060800007E0074F7888314600F00CF8044600E03E
:1060900000BF00BF2046F0BDF0EFFFFF001104403D
:1060A000001404400246002013460B40002B01D090
:1060B000012000E000207047FFB581B00E46174672
:1060C000012F07D1F748407D00090001C01DF549A7
:1060D000487505E0F348407D00090001F149487525
:1060E000049801287ED10A210198F2F72FF805467D
:1060F000ED48445DE007C00F002807D0E948007C68
:1061000000090001C01DE749087405E0E548007C6E
:1061100000090001E349087402202040002807D04C
:10612000E048C07BF02188437030DE49C87305E049
:10613000DC48C07BF0218843DA49C8730420204042
:10614000002807D0D748807C00090001C01DD54930
:10615000887405E0D348807C00090001D149887427
:1061600008202040002807D0CE48407CF0218843FA
:106170007030CC49487405E0CA48407CF02188431F
:10618000C849487410202040002807D0C548407CEA
:1061900000090001C01DC349487405E0C148407CA6
:1061A00000090001BF49487420202040002807D082
:1061B000BC48007CF02188437030BA49087405E07F
:1061C000B848007CF0218843B6490874402020403C
:1061D000002808D0B348807CF02188437030B14952
:1061E000887406E08BE0AF48807CF0218843AD499D
:1061F00088740A210198F1F7A9FF0D46AA48445D69
:10620000E007C00F002807D0A648807BF021884314
:106210007030A449887305E0A248807BF021884350
:10622000A049887302202040002807D09D48807B29
:1062300000090001C01D9B49887305E09948807BD7
:10624000000900019749887304202040002807D0E6
:106250009448007DF021884370309249087505E02C
:106260009048007DF02188438E4908750820204021
:10627000002807D08B48007D00090001C01D894916
:10628000087505E08748007D00090001854908750B
:1062900010202040002807D08248C07CF02188438D
:1062A00070308049C87405E07E48C07CF021884386
:1062B0007C49C87420202040002807D07948C07B42
:1062C00000090001C01D7749C87305E07548C07B0F
:1062D000000900017349C87340202040002807D0FE
:1062E0007048C07C00090001C01D6E49C87454E0AC
:1062F0006C48C07C000900016A49C8744DE06948D7
:10630000007C00090001674908740846C07BF02141
:1063100088436449C8730846807C0009000188747A
:106320000846407CF02188435E4948740846407C1A
:106330000009000148740846007CF021884359494F
:1063400008740846807CF0218843564988740846C2
:10635000807BF0218843534988730846807B00097D
:10636000000188730846007DF02188434D49087577
:106370000846007D0009000108750846C07CF02130
:1063800088434849C8740846C07B00090001C873A7
:106390000846C07C00090001C8740A9801287DD114
:1063A0000A213046F1F7D2FE05463F48445DE0073A
:1063B000C00F002807D03B48407B00090001C01DEA
:1063C0003849487305E03748407B000900013549EA
:1063D000487302202040002807D03248007BF0217B
:1063E000884370302F49087305E02E48007BF02168
:1063F00088432C49087304202040002807D02948EE
:10640000807DF021884370302649887505E0254855
:10641000807DF0218843234988750820204000288A
:1064200007D02048807D00090001C01D1D498875E6
:1064300005E01C48807D000900011A49887510207C
:106440002040002807D01748407DF0218843703055
:106450001449487505E01348407DF02188431149EF
:10646000487520202040002807D00E48407BF021AE
:10647000884370300B49487305E00A48407BF0219F
:106480008843084948734020204000280ED0054822
:10649000C07D00090001C01D024900E092E0C875FE
:1064A0000AE0000078200020F41702006D48C07D4B
:1064B000000900016B49C8750A213046F1F746FE14
:1064C0000D466948445DE007C00F002807D06548C5
:1064D000C07AF021884370306249C87205E0614893
:1064E000C07AF02188435F49C8720220204000280A
:1064F00007D05C48C07A00090001C01D5949C87224
:1065000005E05848C07A000900015649C8720420C5
:106510002040002807D05348407E00090001C01DDC
:106520005049487605E04F48407E000900014D493A
:10653000487608202040002807D04A48007EF021F5
:10654000884370304749087605E04648007EF021D0
:1065500088434449087610202040002807D041484D
:10656000007E00090001C01D3E49087605E03D4857
:10657000007E000900013B490876202020400028C9
:1065800007D03848007B00090001C01D3549087359
:1065900005E03448007B00090001324908734020BF
:1065A0002040002807D02F48C07DF021884370305C
:1065B0002C49C87554E02B48C07DF02188432949F7
:1065C000C8754DE02748407B000900012549487304
:1065D0000846007BF0218843224908730846807DE5
:1065E000F02188431F4988750846807D0009000115
:1065F00088750846407DF02188431A494875084649
:10660000407BF0218843174948730846C07D000944
:106610000001C8750846C07AF02188431149C87244
:106620000846C07A00090001C8720846407E000989
:10663000000148760846007EF02188430949087623
:106640000846007E0009000108760846007B000924
:10665000000108730846C07DF02188430149C875D0
:1066600005B0F0BD78200020F4170200FFB581B01E
:106670000E461746019801287ED10498002826D19D
:10668000FA480078012822D0F6F7DEFAF849884265
:106690001DD3FAF71DFC00280DD0F648807DF021AF
:1066A00088437030F34988750846C07C00090001B2
:1066B000C01DC87418E0EF48807DF0218843ED4983
:1066C00088750846C07C00090001C8740CE0E948E0
:1066D000807DF02188437030E64988750846C07C8B
:1066E00000090001C01DC874E248C07CF021884345
:1066F0007030E049C8740846007EF021884370304D
:10670000DC4908760846807D00090001401C887538
:106710000846407DF02188431030D6494875084628
:10672000407D00090001401C48750846007DF021AD
:1067300088431030CF4908750846007D00090001E4
:10674000401C087533000AF07DFA062E261E140C34
:10675000042FC848007D00090001C01DC549087507
:1067600000BFC448007DF02188437030C1490875DE
:1067700000BFC048407D00E0ADE100090001C01D40
:10678000BC49487500BFBB48407DF021884370304C
:10679000B849487500BFB748807D00090001C01D99
:1067A000B449887500BF00E000BF00BF049800280E
:1067B0005ED1AE48007801285AD0F6F745FAAC49C8
:1067C000884255D3AB48C07FF0218843A949C87798
:1067D0000846807F0009000188770846407FF02145
:1067E0008843A44948770846007FF0218843A1499F
:1067F00008770846C07DF02188439E49C875084641
:10680000C07F00090001C8770846807FF0218843D7
:10681000984988770846407F00090001C01D4877E5
:106820000846807EF0218843924988760846807E1B
:106830000009000188760846407E0009000148767C
:106840000846007E0009000108760846007F00091E
:10685000000108770846C07EF02188438549C87644
:106860000846407EF0218843703082494876B8E17E
:1068700064213846F1F76AFC0546012D07D17D48B1
:10688000C07FF021884370307A49C87705E07948A5
:10689000C07FF02188437749C8770A213846F1F74D
:1068A00055FC0A210090F1F751FC0D46642F02D3EC
:1068B0007148445D01E07148445DE007C00F002865
:1068C00007D06C48807F00090001C01D69498877A6
:1068D00005E06848807F000900016649887702204A
:1068E0002040002807D06348407FF0218843703063
:1068F0006049487705E05F48407FF02188435D4963
:10690000487704202040002807D05A48007FF02113
:10691000884370305749087705E05648007FF021DA
:1069200088435449087708202040002807D0514860
:10693000C07DF021884370304E49C87505E04D4850
:10694000C07DF02188434B49C875102020400028A5
:1069500007D04848C07F00090001C01D4549C877DD
:1069600005E04448C07F000900014249C877202063
:106970002040002807D03F48807FF02188437030B6
:106980003C49887705E03B48807FF02188433949BE
:10699000887740202040002807D03648407F0009F3
:1069A0000001C01D3349487705E03248407F0009A7
:1069B0000001304948770A213846F1F7C7FB0D46F8
:1069C0002D48445DE007C00F002807D02948807E8D
:1069D000F021884370302749887605E02548807E7D
:1069E000F02188432349887602202040002807D0E0
:1069F0002048807E00090001C01D1E49887605E000
:106A00001C48807E000900011A4988760420204035
:106A1000002807D01748407E00090001C01D154915
:106A2000487605E01348407E000900011149487688
:106A300008202040002807D00E48007E00090001F1
:106A4000C01D0C49087605E00A48007E00090001D7
:106A50000849087610202040002811D00548007F02
:106A600000090001C01D034908770FE00D01002057
:106A7000D60B00004C210020F4170200071802007A
:106A80005948007F0009000157490877202020401D
:106A9000002807D05448C07EF02188437030524906
:106AA000C87605E05048C07EF02188434E49C8763C
:106AB00040202040002807D04B48407EF0218843EA
:106AC0007030494948768CE04748407EF021884341
:106AD0004549487685E04448807D000900014249E7
:106AE00088750846407DF02188433F49487508462F
:106AF000407D0009000148750846007DF02188436B
:106B0000394908750846007D0009000108750846E6
:106B1000C07C00090001C8740846807DF0218843CC
:106B2000314988750846C07CF02188432E49C874D5
:106B30000846007EF02188432B4908760846C07F2E
:106B4000F02188432849C8770846807F0009000162
:106B500088770846407FF0218843234948770846D4
:106B6000007FF0218843204908770846C07DF02146
:106B700088431D49C8750846C07F00090001C877D1
:106B80000846807FF0218843174988770846407F70
:106B90000009000148770846807EF02188431249A9
:106BA00088760846807E0009000188760846407E87
:106BB0000009000148760846007E000900010876B9
:106BC0000846007F0009000108770846C07EF021D2
:106BD00088430549C8760846407EF021884302492B
:106BE000487605B0F0BD00004C21002010B50146EC
:106BF000002200200A0EFE4B985CC307DB0F002B1F
:106C000007D0FC4BDB7FF024A3437033F94CE377D0
:106C100005E0F84BDB7FF024A343F64CE377022337
:106C20000340002B07D0F34BDB7F1B091B01DB1D4F
:106C3000F04CE37705E0EF4BDB7F1B091B01ED4CCC
:106C4000E37704230340002B07D0EA4B9B7F1B090B
:106C50001B01DB1DE74CA37705E0E64B9B7F1B097F
:106C60001B01E44CA37708230340002B09D0E14B20
:106C700020335B781B091B01DB1DDE4C2034637065
:106C800007E0DC4B20335B781B091B01D94C203417
:106C9000637010230340002B09D0D64B20331B78A0
:106CA000F024A3437033D34C2034237007E0D14B3E
:106CB00020331B78F024A343CE4C203423702023B0
:106CC0000340002B09D0CB4B20331B781B091B0141
:106CD000DB1DC84C2034237007E0C64B20331B78E3
:106CE0001B091B01C34C2034237040230340002B9D
:106CF00007D0C04B9B7FF024A3437033BD4CA377D8
:106D000005E0BC4B9B7FF024A343BA4CA377FF2341
:106D10001B040B401A0CB64B985CC307DB0F002B0F
:106D200007D0B44B1B7F1B091B01DB1DB14C237724
:106D300005E0B04B1B7F1B091B01AE4C23770223E0
:106D40000340002B07D0AB4BDB7EF024A343703312
:106D5000A84CE37605E0A74BDB7EF024A343A54CCB
:106D6000E37604230340002B07D0A24B9B7EF02444
:106D7000A34370339F4CA37605E09E4B9B7EF0248B
:106D8000A3439C4CA37608230340002B07D0994BC8
:106D90005B7FF024A3437033964C637705E0954BFB
:106DA0005B7FF024A343934C637710230340002BB5
:106DB00007D0904B5B7F1B091B01DB1D8D4C63775C
:106DC00005E08C4B5B7F1B091B018A4C63772023FA
:106DD0000340002B07D0874B1B7FF024A343703365
:106DE000844C237705E0834B1B7FF024A343814C25
:106DF000237740230340002B07D07E4BDB7E1B090B
:106E00001B01DB1D7B4CE37605E07A4BDB7E1B0927
:106E10001B01784CE376FF231B020B401A0A744BCC
:106E2000985CC307DB0F002B07D0724B1B7EF0244E
:106E3000A34370336F4C237605E06E4B1B7EF0242A
:106E4000A3436C4C237602230340002B07D0694BED
:106E50001B7E1B091B01DB1D664C237605E0654B81
:106E60001B7E1B091B01634C237604230340002B6C
:106E700007D0604BDB7D1B091B01DB1D5D4CE375FF
:106E800005E05C4BDB7D1B091B015A4CE3750823B5
:106E90000340002B07D0574B9B7E1B091B01DB1DBA
:106EA000544CA37605E0534B9B7E1B091B01514CB0
:106EB000A37610230340002B07D04E4B5B7EF024BB
:106EC000A34370334B4C637605E04A4B5B7EF02462
:106ED000A343484C637620230340002B07D0454B47
:106EE0005B7E1B091B01DB1D424C637605E0414BB9
:106EF0005B7E1B091B013F4C637640230340002B44
:106F000007D03C4BDB7DF024A3437033394CE37551
:106F100005E0384BDB7DF024A343364CE375CAB261
:106F2000334B985CC307DB0F002B07D0314B1B7D25
:106F3000F024A34370332F4C237505E02D4B1B7DAC
:106F4000F024A3432B4C237502230340002B07D0CE
:106F5000284B1B7D1B091B01DB1D264C237505E0FF
:106F6000244B1B7D1B091B01224C2375042303406A
:106F7000002B07D01F4BDB7C1B091B01DB1D1D4CAD
:106F8000E37405E01B4BDB7C1B091B01194CE3740C
:106F900008230340002B07D0164B9B7CF024A3430F
:106FA0007033144CA37405E0124B9B7CF024A34374
:106FB000104CA37410230340002B07D00D4B5B7DB6
:106FC000F024A34370330B4C637505E0094B5B7DE4
:106FD000F024A343074C637520230340002B0BD000
:106FE000044B5B7D1B091B01DB1D024C637509E033
:106FF000F41702002C2100200C4B5B7D1B091B01A8
:107000000A4C637540230340002B07D0074BDB7C01
:10701000F024A3437033054CE37405E0034BDB7CA1
:10702000F024A343014CE37410BD00002C21002088
:1070300000B501287ED1FE4AD278F0239A437032FF
:10704000FB4BDA701A46127912091201D21D1A711D
:107050001A461279F0239A437032F54B1A711A4688
:10706000527912091201D21D5A711A465279F0232F
:107070009A437032EE4B5A711A46D27912091201B4
:10708000D21DDA711A46D279F0239A437032E84B56
:10709000DA711A46527A12091201D21D5A721A4630
:1070A000527AF0239A437032E14B5A721A46927A1E
:1070B000F0239A437032DE4B9A721A469278F0238C
:1070C0009A437032DA4B9A701A46D27A1209120138
:1070D000D21DDA721A46527812091201D21D5A7064
:1070E0001A46D27AF0239A437032D14BDA721A469A
:1070F000203AD27FF0239A437032CD4B203BDA778F
:10710000CB4A127B12091201D21D20331A731A4680
:10711000203A927F12091201D21D203B9A77C44A6D
:10712000127BF0239A437032C14B1A731A46203AED
:10713000127F00E0F2E1F0239A437032BC4B203B17
:107140001A77BB4A527B12091201D21D20335A739F
:107150001A46203AD27E12091201D21D203BDA765D
:10716000B44AD278F0239A437032B24BDA701A469E
:10717000127B12091201D21D1A731A4612791209D2
:107180001201D21D1A711A46927AF0239A43703274
:10719000A84B9A721A461279F0239A437032A54B83
:1071A0001A711A46527912091201D21D5A711A46E1
:1071B000927912091201D21D9A711A46127A120995
:1071C0001201D21D1A721A46127AF0239A437032B3
:1071D000984B1A721A46527A12091201D21D5A722B
:1071E000934A927912091201521C914B9A711A46D4
:1071F0009279F0239A4310328D4B9A711A46127A83
:1072000012091201521C1A721A46127AF0239A437A
:107210001032874B1A721A46927A12091201521CC6
:107220009A721A46D27812091201521CDA701A4662
:10723000927812091201521C9A701A465278F02361
:107240009A4310327A4B5A701A461278F0239A43B6
:107250001032774B1A701A46127812091201521C1A
:107260001A701A46203AD27F12091201521C203B92
:10727000DA771A46927FF0239A4310326C4B203B08
:107280009A771A46527FF0239A431032684B203B7C
:107290005A771A46527F12091201521C5A771A461F
:1072A000127F12091201521C1A771A46D27EF0235D
:1072B0009A4310325E4B203BDA761A46927EF023D8
:1072C0009A4310325A4B203B9A765A4A127BF0234B
:1072D0009A431032574B1A731A46D27AF0239A43C4
:1072E0001032544BDA721A46D27A12091201521C29
:1072F000DA721A46927A12091201521C9A721A46CE
:10730000527AF0239A4310324A4B5A721A465279F3
:10731000F0239A431032474B5A711A46D279F02320
:107320009A431032434BDA710B0009F08BFC19F3CE
:10733000E9DFD5CBC1B7ADA3998F87786E645A507A
:10734000463E362E261E160EF5003A4AD279F02316
:107350009A437032374BDA7100BF364A5279F023C4
:107360009A437032334B5A7100BF324A527AF0233B
:107370009A4370322F4B5A7200BF2E4A927A1209EA
:107380001201D21D2B4B9A7200BF2A4AD27A1209DF
:107390001201D21D274BDA7200BF264AD27AF0239F
:1073A0009A437032234BDA7200BF224A127BF023D9
:1073B0009A4370321F4B1A7300BF1D4A203A927EC7
:1073C000F0239A4370321A4B203B9A7600BF184A3A
:1073D000203AD27EF0239A437032154B203BDA7666
:1073E00000BF134A203A127F12091201D21D104B1E
:1073F000203B1A7700BF0E4A203A527F1209120131
:10740000D21D0B4B203B5A7700BF094A203A527FCE
:10741000F0239A437032064B203B5A7700BF044A50
:10742000203A927FF0239A437032014B203B03E0D5
:10743000982000206C2100209A7700BFDC4AD27F80
:1074400012091201D21DDA4BDA7700BFD84A203276
:10745000127812091201D21DD54B20331A7000BFC9
:10746000D34A20321278F0239A437032D04B203323
:107470001A7000BFCE4A20325278F0239A437032FD
:10748000CB4B20335A7000BFC94A20329278120980
:107490001201D21DC64B20339A7000BFC44A20325D
:1074A000D27812091201D21DC14B2033DA7000BF0D
:1074B000BF4A2032927A12091201D21DBC4B2033EE
:1074C0009A7200BFBA4A2032127AF0239A4370327D
:1074D000B74B20331A7200BFB54A2032127A120914
:1074E0001201D21DB24B20331A7200BFB04A2032B3
:1074F0009279F0239A437032AD4B20339A7100BFDA
:10750000AB4A2032927912091201D21DA84B2033C6
:107510009A7100BF01E0FFE700BF47E1A44A2032B3
:10752000D278F0239A43A24B2033DA701A461279AC
:10753000120912011A711A461279F0239A439C4BD0
:1075400020331A711A465279120912015A711A46D9
:107550005279F0239A43964B20335A711A46D279C6
:1075600012091201DA711A46D279F0239A43904B2C
:107570002033DA711A46527A120912015A721A46E7
:10758000527AF0239A438A4B20335A721A46927ADF
:10759000F0239A43864B20339A721A469278F0234E
:1075A0009A43834B20339A701A46D27A12091201F9
:1075B000DA721A465278120912015A701A46D27AB1
:1075C000F0239A437A4B2033DA72794AD27FF02340
:1075D0009A43774BDA771A462032127B120912014E
:1075E00020331A73724A927F12091201203B9A7754
:1075F0001A462032127BF0239A436D4B20331A73C4
:107600006B4A127FF0239A43694B1A771A4620324D
:10761000527B1209120120335A73654AD27E120935
:107620001201203BDA76634AD278F0239A43614B09
:10763000DA701A46127B120912011A731A4612796D
:10764000120912011A711A46927AF0239A43594B81
:107650009A721A461279F0239A43564B1A711A46B7
:107660005279120912015A711A46927912091201BD
:107670009A711A46127A120912011A721A46127A6D
:10768000F0239A434B4B1A721A46527A120912018E
:107690005A72474A2032927912091201444B203320
:1076A0009A711A469279F0239A43414B20339A718A
:1076B0001A46127A120912011A721A46127AF02325
:1076C0009A433B4B20331A721A46927A12091201DE
:1076D0009A721A46D27812091201DA701A46927812
:1076E000120912019A701A465278F0239A43304BCD
:1076F00020335A701A461278F0239A432C4B2033C9
:107700001A701A461278120912011A70284AD27F8A
:1077100012091201203BDA771A46927FF0239A432E
:10772000234B9A771A46527FF0239A43204B5A777D
:107730001A46527F120912015A771A46127F12090D
:1077400012011A771A46D27EF0239A43184BDA7642
:107750001A46927EF0239A43154B9A76154A127B6D
:10776000F0239A43134B1A731A46D27AF0239A43A2
:10777000104BDA721A46D27A12091201DA721A46DC
:10778000927A120912019A721A46527AF0239A4397
:10779000084B5A721A465279F0239A43054B5A7194
:1077A0001A46D279F0239A43024BDA7100BD0000E9
:1077B000782000206C210020F7B582B006461746DD
:1077C000002500200190002E7ED1F9F793FA0528BC
:1077D0005FD1F9F77DFB00280DD0FA484079F02100
:1077E00088437030F74948710846807800090001E5
:1077F000C01D88700AE0F3484079F0218843F149C0
:10780000487108468078000900018870ED48C07909
:1078100000090001EB49C8710846807900090001A0
:107820008871084640790009000148710846007ACD
:10783000F0218843E34908720846007A00090001F4
:1078400008720846C079F0218843DE49C8710846AD
:10785000C07800090001C87008468078F02188438C
:10786000D849887008464078F0218843D549487047
:107870000846407800090001487008460079000970
:10788000000108710846C078F0218843CD49C870CE
:1078900029E2CC484079F02188437030C9494871C9
:1078A0000846807800090001C01D88700846C0792C
:1078B00000090001C871084680790009000188713B
:1078C00008464079000900E034E0000148710846AC
:1078D000007AF0218843BB4908720846007A000903
:1078E000000108720846C079F0218843B549C87183
:1078F0000846C07800090001C87008468078F02169
:107900008843B049887008464078F0218843AD49E3
:107910004870084640780009000148700846007920
:107920000009000108710846C078F0218843A54984
:10793000C870ADE7012E5FD1F9F7CAFA00280DD063
:10794000A0484079F021884370309E49487108462C
:10795000807800090001C01D88700AE099484079CC
:10796000F021884397494871084680780009000152
:1079700088709448C079000900019249C87108468E
:1079800080790009000188710846407900090001EA
:1079900048710846007AF02188438A4908720846EF
:1079A000007A0009000108720846C079F021884376
:1079B0008449C8710846C07800090001C8700846AB
:1079C0008078F02188437F49887008464078F0210C
:1079D00088437C4948700846407800090001487097
:1079E000084600790009000108710846C078F021B6
:1079F00088437449C870EAE3022E7DD1F9F77AF919
:107A000005287AD1F9F764FA002877D0012F76D1CA
:107A10000A210398F0F79AFB0546F9F789F900283F
:107A200002D16948445D01E06848445DE007C00F49
:107A3000002807D06348C07900090001C01D6149D2
:107A4000C87105E05F48C079000900015D49C8714F
:107A500002202040002807D05A4880790009000100
:107A6000C01D5849887105E0564880790009000119
:107A70005449887104202040002807D0514840799B
:107A800000090001C01D4F49487105E04D4840798B
:107A9000000900014B49487108202040002807D008
:107AA0004848007AF021884370304649087205E062
:107AB0004448007AF021884342490872102020404F
:107AC000002807D03F48007A00090001C01D3D4949
:107AD000087205E03B48007A000900013949087244
:107AE0002020204000280BD03648C079F021884360
:107AF00070303449C87109E0AEE242E1F4E0A4E03C
:107B00003048C079F02188432E49C8714020204078
:107B1000002807D02B484079F0218843703029494C
:107B2000487105E027484079F0218843254948718C
:107B30000A210398F0F70AFB0D462348445DE0074D
:107B4000C00F002807D01F48C07800090001C01DE1
:107B50001C49C87005E01B48C0780009000119499C
:107B6000C87002202040002807D016488078F021F5
:107B7000884370301349887005E012488078F021FE
:107B800088431049887004202040002807D00D4801
:107B90004078F021884370300A49487005E0094870
:107BA0004078F02188430749487008202040002889
:107BB0000ED00448407800090001C01D01494870FA
:107BC0000CE00000B8200020F417020007180200A3
:107BD000FE48407800090001FC4948701020204010
:107BE000002807D0F948007900090001C01DF749B5
:107BF000087105E0F548007900090001F3490871B2
:107C000020202040002807D0F048C078F021884389
:107C10007030EE49C87005E0EC48C078F021884328
:107C2000EA49C87040202040002807D0E748807803
:107C300000090001C01DE5498870C8E2E34880786A
:107C400000090001E1498870C1E2E0484079F02173
:107C500088437030DD49487108468078000900018A
:107C6000C01D88700846C07900090001C871084627
:107C700080790009000188710846407900090001F7
:107C800048710846007AF0218843D04908720846B6
:107C9000007A0009000108720846C079F021884383
:107CA000CA49C8710846C07800090001C870084672
:107CB0008078F0218843C549887008464078F021D3
:107CC0008843C2494870084640780009000148705E
:107CD000084600790009000108710846C078F021C3
:107CE0008843BA49C87072E2B8484079F0218843A5
:107CF000B649487108468078000900018870084636
:107D0000C07900090001C8710846807900090001A6
:107D10008871084640790009000148710846007AD8
:107D2000F0218843A94908720846007A0009000139
:107D300008720846C079F0218843A449C8710846F2
:107D4000C07800090001C87008468078F021884397
:107D50009E49887008464078F02188439B494870C6
:107D6000084640780009000148700846007900097B
:107D7000000108710846C078F02188439349C87013
:107D800025E2012F73D10A210398F0F7DFF90546A8
:107D9000F8F7CEFF002802D18D48445D01E08D4800
:107DA000445DE007C00F002807D08848C07900096B
:107DB0000001C01D8549C87105E08448C0790009EB
:107DC00000018249C87102202040002807D07F4866
:107DD000807900090001C01D7C49887105E07B485D
:107DE0008079000900017949887104202040002829
:107DF00007D07648407900090001C01D73494871D9
:107E000005E0724840790009000170494871082076
:107E10002040002807D06D48007AF0218843703058
:107E20006A49087205E06948007AF0218843674989
:107E3000087210202040002807D06448007A00090A
:107E40000001C01D6149087205E06048007A000920
:107E500000015E49087220202040002808D05B48BD
:107E6000C079F021884370305849C87106E09DE020
:107E70005648C079F02188435449C87140202040B9
:107E8000002807D051484079F021884370304F498D
:107E9000487105E04D484079F02188434B494871CD
:107EA0000A210398F0F752F90D464948445DE0076E
:107EB000C00F002807D04548C07800090001C01D48
:107EC0004249C87005E04148C078000900013F49B7
:107ED000C87002202040002807D03C488078F0215C
:107EE000884370303949887005E038488078F0213F
:107EF00088433649887004202040002807D0334842
:107F00004078F021884370303049487005E02F48B0
:107F10004078F02188432D494870082020400028EF
:107F200007D02A48407800090001C01D2749487041
:107F300005E02648407800090001244948701020D7
:107F40002040002807D02148007900090001C01D09
:107F50001E49087105E01D480079000900011B4910
:107F6000087120202040002807D01848C078F02150
:107F7000884370301549C87005E01448C078F02176
:107F800088431249C87040202040002807D00F487D
:107F9000807800090001C01D0C49887017E10B486A
:107FA0008078000900010949887010E1074840798C
:107FB000F0218843703005494871084680780009EF
:107FC0000001C01D88700846C07905E0B820002077
:107FD000F41702000718020000090001C8710846E2
:107FE0008079000900018871084640790009000184
:107FF00048710846007AF02188437649087208469D
:10800000007A0009000108720846C079F02188430F
:108010007049C8710846C07800090001C870084658
:108020008078F02188436B49887008464078F021B9
:108030008843684948700846407800090001487044
:10804000084600790009000108710846C078F0214F
:1080500088436049C870BAE0032E9FD1F8F74AFE02
:1080600005285FD1F8F734FF00280DD05948407932
:10807000F0218843703057494871084680780009DC
:108080000001C01D88700AE052484079F021884301
:1080900050494871084680780009000188704D48B1
:1080A000C079000900014B49C87108468079000970
:1080B00000018871084640790009000148710846AE
:1080C000007AF0218843434908720846007A000983
:1080D000000108720846C079F02188433D49C87103
:1080E0000846C07800090001C87008468078F02171
:1080F00088433849887008464078F02188433549DC
:108100004870084640780009000148700846007928
:108110000009000108710846C078F02188432D4904
:10812000C87054E02B480079F02188437030294909
:10813000087108464079F02188437030254948711C
:108140000846807800090001C01D88700846C07983
:1081500000090001C8710846807900090001887192
:10816000084640790009000148710846007AF0216C
:108170008843184908720846007A0009000108720D
:108180000846C079F02188431249C8710846C07872
:1081900000090001C87008468078F02188430D4925
:1081A000887008464078F02188430A49487008469C
:1081B0004078000900014870084600790009000174
:1081C00008710846C078F02188430249C87005B09C
:1081D000F0BD0000B820002070B505460C46012D0A
:1081E0007ED1B248407D00090001C01DAF494875ED
:1081F0000846007DF02188431030AC4908750846D8
:10820000007D00090001401C08750846C07CF02173
:1082100088431030A549C8740846807CF021884303
:108220001030A24988740846807C00090001401C77
:108230008874F8F7A7FE022803D0F8F7A3FE0128F8
:108240006CD19B480078012868D0F4F7FDFC99496F
:10825000884263D3F8F73CFE00282FD09348007D76
:10826000F02188437030914908750846007D000967
:108270000001C01D08750846C07CF021884370309D
:108280008A49C8740846807CF02188437030874949
:1082900088740846807C00090001C01D8874084667
:1082A000407DF02188437030804948750846407C05
:1082B000F021884370307D494874F6E07B48007DAA
:1082C000F02188431030794908750846007D00097F
:1082D0000001401C08750846C07CF021884300E07E
:1082E000B6E010307149C8740846807CF02188439C
:1082F00010306E4988740846807C00090001401CDB
:1083000088740846407DF0218843684948750846CE
:10831000407CF021884365494874C6E0F8F7D4FCF6
:10832000002825D1F4F790FC62491E3188421FD302
:10833000F8F7CEFD00280ED05C48407DF021884340
:1083400070305A4948750846407CF02188437030A7
:10835000564948741AE05548407DF02188435349F6
:1083600048750846407CF0218843504948740DE028
:108370004E48407DF021884370304C49487508468E
:10838000407CF0218843703048494874F8F79CFCE1
:1083900001282BD146480078012827D0F4F754FC57
:1083A00044491E31884221D34048407DF021884312
:1083B00070303E4948750846407CF0218843703053
:1083C0003A494874F8F784FD002807D03748007D03
:1083D000F021884370303549087566E03348007DE8
:1083E000F02188431030314908755EE0230008F021
:1083F00029FC062C241C140C042D2C48807C00091C
:108400000001C01D2949887400BF2848807CF021E4
:10841000884370302549887400BF2448C07CF0210F
:10842000884370302149C87400BF2048007D00098E
:108430000001C01D1D49087500BF1C48007DF021CA
:10844000884370301949087500BF00E000BF2CE078
:108450001648407DF0218843144948750846007D40
:10846000F0218843114908750846007D0009000184
:1084700008750846C07CF02188430C49C87408463A
:10848000807CF0218843094988740846807C000973
:10849000000188740846407D0009000148750846BF
:1084A000407CF02188430149487470BD9820002029
:1084B0000D010020B80B000030B50246002901D1A3
:1084C000002000E00720130008F0BCFB0F09141F78
:1084D0002B3743505D67727C88929FA9B500574B3C
:1084E0005B7EF024A3430401F0252C402343534C2E
:1084F0006376A1E0524B9B79F024A3430401F0255D
:108500002C4023434E4CA37196E04D4B2033DB7936
:108510001B091B010407240F2343494C2034E3713A
:108520008AE0464B2033DB7C1B091B010407240F28
:108530002343424C2034E3747EE0404B40331B78AD
:108540001B091B010407240F23433C4C40342370B8
:1085500072E03A4B2033DB7FF024A3430401F02583
:108560002C402343354C2034E37765E0334B2033F4
:108570005B7BF024A3430401F0252C4023432F4CC4
:108580002034637358E02E4B9B791B091B010407B1
:10859000240F23432A4CA3714EE0294B9B7CF024EB
:1085A000A3430401F0252C402343254CA37443E04E
:1085B000234BDB7E1B091B010407240F2343204CA4
:1085C000E37639E01D4B2033DB7F1B091B010407D9
:1085D000240F2343194C2034E3772DE0174B9B7E67
:1085E0001B091B010407240F2343144CA37623E02B
:1085F000134B20339B79F024A3430401F0252C4036
:1086000023430F4C2034A37116E00D4BDB7D1B0977
:108610001B010407240F2343094CE3750CE0074BAF
:1086200020335B7C1B091B010407240F2343034CED
:108630002034637400E000BF00BF30BD782000200C
:108640004C210020F7B582B00746154600260024CD
:10865000FE480078012804D0F4F7F6FAFC49884275
:1086600079D2FC48407CF02188437030F949487445
:108670000846807C00090001C01D88740846007D02
:1086800000090001C01D08750846007DF0218843DF
:108690007030F04908750846807CF02188437030BE
:1086A000EC4988740846C07C00090001C01DC874EC
:1086B0000846C07CF02188437030E649C8740846FB
:1086C000407C00090001C01D48740846407D000937
:1086D0000001C01D48750846407DF0218843703078
:1086E000DC4948750846007CF02188437030D94940
:1086F00008740846007C00090001C01D0874084683
:10870000C07BF02188437030D249C873FF220A2110
:108710000020FAF7EBFFFF2213210020FAF7E6FF13
:10872000FF2211210020FAF7E1FFFF221221002091
:10873000FAF7DCFFFF220E210020FAF7D7FFFF2215
:108740000F210020FAF7D2FFFF2210210020FAF7B4
:10875000CDFFF4E3FFE7039836283DD019DC082865
:108760007ED007DC801E030008F06CFA0635A8FCFA
:10877000FBFAF97E102874D006DC092872D00D2887
:1087800071D00E2870D1FDE333286ED03428F9D192
:1087900070E13F286AD00FDC3738082864D24300E4
:1087A0007B449B885B009F448A009702FF025F0026
:1087B0005F006503CB0318004E287BD006DC402801
:1087C00079D0412878D04D28DCD1BBE14F2874D036
:1087D0005028D7D14FE100BF00BF9E48407CF02118
:1087E00088439C4948740846807C000900018874CD
:1087F0000846007D00090001C01D08750846007D7F
:10880000F02188437030934908750846807CF02138
:108810008843904988740846C07C00090001C01D47
:10882000C8740846C07CF02188438A49C874084649
:10883000407C0009000148740846407D00090001A1
:1088400048750846407DF0218843824948750846AE
:10885000007CF02188437F4908740846007C06E0CC
:10886000A1E2FDE337E2D2E3FBE394E028E0000974
:10887000000108740846C07BF02188437549C8731D
:10888000FF220A210020FAF731FFFF2213210020E6
:10889000FAF72CFF00220E211046FAF727FF0022DC
:1088A0000F211046FAF722FF002210211046FAF796
:1088B0001DFF77E2ABE110E2DDE26DE000BF00BF3B
:1088C0006448407CF0218843624948740846807CB3
:1088D0000009000188740846007D00090001C01DE0
:1088E00008750846007DF0218843703059490875A5
:1088F0000846807CF0218843564988740846C07C2D
:1089000000090001C8740846C07CF0218843514921
:10891000C8740846407C0009000148740846407D40
:1089200000090001C01D48750846407DF0218843BC
:10893000484948750846007CF02188434549087439
:108940000846007C0009000108740846C07BF0213D
:1089500088434049C873FF220A21002003E055E103
:10896000EFE086E016E0FAF7C1FEFF2213210020B7
:10897000FAF7BCFE00220E211046FAF7B7FE0022DD
:108980000F211046FAF7B2FE002210211046FAF726
:10899000ADFE8EE700BF00BF2E48407CF02188432B
:1089A0002C4948740846807C00090001C01D887469
:1089B0000846007D00090001C01D08750846007DBD
:1089C000F02188437030234908750846807CF021E7
:1089D000884370301F4988740846C07C0009000134
:1089E000C8740846C07CF02188431A49C8740846F8
:1089F000407C0009000148740846407D00090001E0
:108A000048750846407DF02188431249487508465C
:108A1000007CF02188430F4908740846007C000957
:108A2000000108740846C07BF02188430949C873D7
:108A3000FF220A210020FAF759FEFF22132100200D
:108A4000FAF754FE00220E21104605E00D01002029
:108A5000D60B0000B8200020FAF748FE00220F21B4
:108A60001046FAF743FE002210211046FAF73EFEA8
:108A70001FE700BF00BFFE48407CF0218843FC494F
:108A800048740846807C00090001C01D88740846AF
:108A9000007D00090001C01D08750846007DF02119
:108AA00088437030F24908750846807CF02188437D
:108AB000EF4988740846C07C00090001C874084664
:108AC000C07CF0218843EA49C8740846407C00090C
:108AD0000001C01D48740846407D0009000148752A
:108AE0000846407DF0218843E14948750846007CEE
:108AF000F0218843DE4908740846007C0009000123
:108B000008740846C07BF0218843D949C873FF2206
:108B10000A210020FAF7EAFDFF2213210020FAF7CC
:108B2000E5FD00220E211046FAF7E0FD00220F219C
:108B30001046FAF7DBFD002210211046FAF7D6FDA9
:108B4000F6E300BFCA48407CF0218843C849487416
:108B50000846807C0009000188740846007D0009F1
:108B6000000108750846007DF02188437030C04937
:108B700008750846807CF0218843BD498874084602
:108B8000C07C00090001C8740846C07CF0218843FD
:108B90007030B749C8740846407C00090001487429
:108BA0000846407D0009000148750846407DF021D7
:108BB0008843AF4948750846007CF0218843AC499A
:108BC00008740846007C0009000108740846C07B50
:108BD000F0218843A649C873FF220A210020FAF732
:108BE00085FDFF2213210020FAF780FD00220E21CF
:108BF0001046FAF77BFD00220F211046FAF776FDAA
:108C0000002210211046FAF771FD91E300BF984849
:108C1000407CF0218843964948740846807C0009CE
:108C2000000188740846007D0009000108750846A7
:108C3000007DF021884370308D4908750846807C9E
:108C4000F02188438A4988740846C07C00090001E5
:108C5000C8740846C07CF02188438549C87408461A
:108C6000407C0009000148740846407D000900016D
:108C700048750846407DF021884370307C4948752E
:108C80000846007CF0218843794908740846007C36
:108C90000009000108740846C07BF021884374492C
:108CA000C873FF220A210020FAF720FDFF221321BA
:108CB0000020FAF71BFD00220E211046FAF716FDE0
:108CC00000220F211046FAF711FD00221021104654
:108CD000FAF70CFD2CE300BF00BF6548407CF02193
:108CE00088437030624948740846807C000900015E
:108CF000C01D88740846007D00090001C01D08756C
:108D00000846007DF02188437030594908750846AF
:108D1000807CF0218843564988740846C07C00094D
:108D20000001C8740846C07CF02188435049C874CB
:108D30000846407C0009000148740846407D00094F
:108D4000000148750846407DF02188434849487530
:108D50000846007CF0218843454908740846007C99
:108D60000009000108740846C07BF021884340498F
:108D7000C873FF220A210020FAF7B8FCFF22132152
:108D80000020FAF7B3FC00220E211046FAF7AEFCE1
:108D900000220F211046FAF7A9FC002210211046EC
:108DA000FAF7A4FCC4E200BF3148407CF0218843BC
:108DB0002F4948740846807C0009000188740846E1
:108DC000007D0009000108750846007DF0218843F8
:108DD0007030274908750846807CF0218843244973
:108DE00088740846C07C00090001C8740846C07C2D
:108DF000F021884370301E49C8740846407C000941
:108E0000000148740846407D000900014875084685
:108E1000407DF0218843164948750846007CF021C2
:108E20008843134908740846007C0009000108744F
:108E30000846C07BF02188430D49C873FF220A21F0
:108E40000020FAF753FCFF2213210020FAF74EFC12
:108E500000220E211046FAF749FC00220F2110468D
:108E6000FAF744FC002210211046FAF73FFC5FE2BB
:108E7000B820002000BFFC48407CF0218843FA491C
:108E800048740846807C0009000188740846007D0B
:108E90000009000108750846007DF0218843703004
:108EA000F14908750846807CF0218843EE498874B2
:108EB0000846C07C00090001C8740846C07CF02147
:108EC0008843E949C8740846407C00090001487499
:108ED0000846407D0009000148750846407DF021A4
:108EE00088437030E04948750846007CF02188438B
:108EF000DD4908740846007C000900010874084632
:108F0000C07BF0218843D849C873FF220A21002082
:108F1000FAF7ECFBFF2213210020FAF7E7FB00220F
:108F20000E211046FAF7E2FB00220F211046FAF755
:108F3000DDFB002210211046FAF7D8FBF8E1F8E13A
:108F4000C948407CF02188437030C74948740846BE
:108F5000807C00090001C01D88740846007D00095E
:108F60000001C01D08750846007DF0218843BE49F8
:108F700008750846807CF0218843BB498874084600
:108F8000C07C00E0A9E000090001C8740846C07C6C
:108F9000F0218843B449C8740846407C00090001A8
:108FA00048740846407D0009000148750846407D28
:108FB000F0218843AC4948750846007CF02188437D
:108FC000A94908740846007C000900010874084695
:108FD000C07BF0218843A449C873FF220A210020E6
:108FE000FAF784FBFF2213210020FAF77FFB00220F
:108FF0000E211046FAF77AFB00220F211046FAF7ED
:1090000075FB002210211046FAF770FB90E196489C
:10901000407CF0218843944948740846807C0009CC
:10902000000188740846007D0009000108750846A3
:10903000007DF02188438C4908750846807CF0212A
:109040008843894988740846C07C00090001C874B7
:109050000846C07CF02188438349C874084601E073
:109060009EE003E1407C0009000148740846407D11
:109070000009000148750846407DF02188437A497F
:1090800048750846007CF0218843774908740846F3
:10909000007C0009000108740846C07BF021884369
:1090A00070307149C87300220A211046FAF71EFB7E
:1090B000002213211046FAF719FBFF220E2100208F
:1090C000FAF714FB00220F211046FAF70FFB0022DB
:1090D00010211046FAF70AFB2AE16348407CF02190
:1090E0008843614948740846807C000900018874FF
:1090F0000846007D0009000108750846007DF02142
:109100008843594908750846807CF02188435649B0
:1091100088740846C07C00090001C8740846C07CF9
:10912000F02188435049C8740846407C000900017A
:1091300048740846407D0009000148750846407D96
:10914000F0218843484948750846007CF02188434F
:10915000454908740846007C00090001C01D0874D8
:109160000846C07BF02188433F49C87300220A218A
:109170001046FAF7BBFA002213211046FAF7B6FAA6
:1091800000220E211046FAF7B1FAFF220F2100202B
:10919000FAF7ACFA002210211046FAF7A7FAC7E056
:1091A0003148407CF02188432F4948740846807C30
:1091B0000009000188740846007D00090001087557
:1091C0000846007DF0218843274908750846807CC1
:1091D000F0218843244988740846C07C00090001B6
:1091E000C8740846C07CF02188431F49C8740846EB
:1091F000407C0009000148740846407D00090001D8
:1092000048750846407DF02188431749487508464F
:10921000007CF02188437030134908740846007CB4
:109220000009000108740846C07BF02188430E49FC
:10923000C87300220A211046FAF758FA00221321B7
:109240001046FAF753FA00220E211046FAF74EFAAA
:1092500000220F211046FAF749FAFF2210210020C0
:10926000FAF744FA64E00000B8200020FD48407C92
:10927000F0218843FB4948740846807C00090001BE
:1092800088740846007D0009000108750846007DC5
:10929000F0218843F34908750846807CF021884313
:1092A000F04988740846C07C00090001C87408466B
:1092B000C07CF0218843EB49C8740846407C000913
:1092C000000148740846407D0009000148750846C1
:1092D000407DF0218843E34948750846007CF02131
:1092E0008843E04908740846007C000900010874BE
:1092F0000846C07BF0218843DA49C87300220A215E
:109300001046FAF7F3F9002213211046FAF7EEF9A6
:1093100000220E211046FAF7E9F900220F2110462B
:10932000FAF7E4F9002210211046FAF7DFF900BF3E
:1093300000BF002F03D0CC48007A002808D1F3F7F3
:1093400083FCCA49884203D3C9480078012872D1F6
:10935000FF2211210020FAF7C9F9FF221221002073
:10936000FAF7C4F9C2480078012804D0F3F76CFC7E
:10937000BE49884216D2BF48807BF02188437030B6
:10938000BC498873084640300078F021884370302B
:10939000B849403108700846007800090001C01D36
:1093A00008702DE07D20C000854214D2B148807B3A
:1093B000F0218843AF498873084640300078F02197
:1093C00088437030AB494031087008460078000986
:1093D0000001087014E0A748807BF02188437030BA
:1093E000A4498873084640300078F0218843A14999
:1093F000403108700846007800090001C01D08705F
:109400007D20C000854205D201462846EEF79EFE2B
:10941000064604E098492846EEF798FE064694482A
:109420000078012804D0F3F70FFC9049884203D25A
:109430009248845D02E0A0E29148845DE007C00F9D
:10944000002809D08B484030C07800090001C01DB9
:1094500088494031C87007E086484030C07800092C
:10946000000184494031C87002202040002807D004
:109470008048C07900090001C01D7E49C87105E01F
:109480007C48C079000900017A49C8710420204055
:10949000002807D07748807900090001C01D754970
:1094A000887105E07348807900090001714988716D
:1094B00008202040002807D06E484079F0218843DA
:1094C00070306C49487105E06A484079F021884362
:1094D0006849487110202040002807D0654840792D
:1094E00000090001C01D6349487105E061484079E9
:1094F000000900015F49487120202040002807D062
:109500005C480079F021884370305A49087105E0C1
:1095100058480079F021884356490871402020407E
:10952000002807D053488079F02188437030514992
:10953000887105E04F488079F02188434D49887152
:109540007D20C000854213D264212846EEF7FEFD3F
:10955000064647480078012804D0F3F775FB4349D5
:10956000884202D24548845D23E04548845D20E07E
:10957000642128463230EEF7E9FD7D21C9000090D4
:10958000EEF7E4FD019164210198EEF7DFFD064658
:109590003C48854208D236480078012804D0F3F7C9
:1095A00053FB3249884202D23448845D01E034489A
:1095B000845DE007C00F002809D02E484030807835
:1095C000F021884370302B494031887007E02948EA
:1095D00040308078F021884326494031887002204D
:1095E0002040002807D02348807A00090001C01DD0
:1095F0002049887205E01F48807A000900011D4952
:10960000887204202040002807D01A48407A0009B8
:109610000001C01D1749487205E01648407A00094C
:1096200000011449487208202040002807D0114842
:10963000007AF021884370300E49087205E00D4829
:10964000007AF02188430B4908721020204000283E
:109650001AD00848007A00090001C01D05490872A7
:1096600018E00000B8200020240A0020D60B0000DB
:109670000D0100202C210020A0860100F41702001B
:109680000718020010270000FE48007A00090001B8
:10969000FC49087220202040002807D0F948C079F2
:1096A000F02188437030F749C87105E0F548C0796A
:1096B000F0218843F349C87140202040002807D09A
:1096C000F048407AF02188437030EE49487205E056
:1096D000EC48407AF0218843EA4948727D20C00076
:1096E000854219D20A212846EEF730FD0A21019061
:1096F000EEF72CFD0E460A2D08D2E348007801282B
:1097000004D0F3F7A1FAE149884202D2E048845D2F
:1097100012E0E048845D0FE0642128463230EEF725
:1097200015FD0A210090EEF711FD0A210190EEF7D8
:109730000DFD0E46D6498C5DE007C00F002809D00C
:10974000D0484030807800090001C01DCD4940312B
:10975000887007E0CB484030807800090001C94993
:109760004031887002202040002807D0C548807B07
:1097700000090001C01DC349887305E0C148807B12
:1097800000090001BF49887304202040002807D049
:10979000BC48407B00090001C01DBA49487305E080
:1097A000B848407B00090001B649487308202040B2
:1097B000002807D0B348007BF02188437030B149BE
:1097C000087305E0AF48007BF0218843AD4908737A
:1097D00010202040002807D0AA48C07A00090001C4
:1097E000C01DA849C87205E0A648C07A000900015A
:1097F000A449C87220202040002807D0A148807AC0
:10980000F021884370309F49887205E09D48807A36
:10981000F02188439B49887240202040002807D0CF
:109820009848407BF021884370309649487305E0A2
:109830009448407BF0218843924948737D20C000C2
:10984000854207D20A212846EEF780FC0E46904852
:10985000845D0BE0642128463230EEF777FC0A2164
:109860000190EEF773FC0E4689498C5DE007C00F4E
:10987000002809D0834840304078F0218843703078
:1098800080494031487007E07E4840304078F02100
:1098900088437C494031487002202040002809D08C
:1098A00078484030407800090001C01D75494031BA
:1098B000487007E073484030407800090001714962
:1098C0004031487004202040002807D06D48007CBB
:1098D000F021884370306B49087405E06948007CCA
:1098E000F02188436749087408202040002807D0E9
:1098F0006448007C00090001C01D6249087405E04D
:109900006048007C000900015E4908741020204076
:10991000002807D05B48C07BF0218843703059494C
:10992000C87305E05748C07BF02188435549C87388
:1099300020202040002807D05248C07B00090001A9
:10994000C01D5049C87305E04E48C07B00090001A6
:109950004C49C87340202040002807D04948407C2B
:1099600000090001C01D47494874ECE04548407CAF
:109970000009000143494874E5E000220A2110462D
:10998000F9F7B4FE002213211046F9F7AFFE0022CA
:1099900011211046F9F7AAFE002212211046F9F70C
:1099A000A5FE00220E211046F9F7A0FE00220F218D
:1099B0001046F9F79BFE002210211046F9F796FE9B
:1099C00030484030C078000900012E494031C8704D
:1099D0002C48C079000900014039C87108468079D7
:1099E00000090001887108464079F0218843254923
:1099F000487108464079000900014871084600791D
:109A0000F02188431F49087108468079F021884376
:109A10001C498871084640308078F02188431949F4
:109A2000403188701748807A0009000140398872F7
:109A30000846407A0009000148720846007AF02181
:109A40008843104908720846007A0009000108722C
:109A50000846C079F02188430A49C8710846407A0F
:109A6000F021884307494872084640308078000951
:109A70000001403188700348807B000900014039B3
:109A8000887309E02C2100200D010020D60B000076
:109A9000F4170200071802000846407B0009000185
:109AA00048730846007BF02188432849087308461C
:109AB000C07A00090001C8720846807AF021884304
:109AC000224988720846407BF02188431F49487329
:109AD000084640304078F02188431C4940314870A6
:109AE000084640780009000148701848007CF021C1
:109AF0008843164908740846007C00090001087470
:109B00000846C07BF02188431049C8730846C07BD3
:109B100000090001C8730846407C00090001487430
:109B20000846807BF0218843084988730846403006
:109B30000078F021884305494031087008460078D4
:109B400000090001087005B0F0BD00002C210020C4
:109B5000F7B582B007460E460121FF200830FBF71B
:109B600079FF0121FC48FBF775FFFC4800780128CC
:109B70007ED0F3F769F8FA49884279D3F7F7BAF853
:109B8000032843D1F7F7B0F8002803D0F7F7ACF873
